:100000000C94B10D0C94DC0D0C94DC0D0C94DC0DF7
:100010000C94DC0D0C94DC0D0C94DC0D0C94DC0DBC
:100020000C94DC0D0C94DC0D0C9492D60C940CD535
:100030000C94DC0D0C94DC0D0C94DC0D0C94DC0D9C
:100040000C94DC0D0C9470A80C94DC0D0C94DC0D5D
:100050000C94DC0D0C94DC0D0C94C19B0C94D5D34A
:100060000C94DC0D0C94DC0D0C94DC0D0C94DC0D6C
:100070000C94DC0D0C94DC0D0C94DC0D0C94DC0D5C
:100080000C94DC0D0C94DC0D0C94DC0D0C94DC0D4C
:100090000C9403CF0C94DC0D084AD73B3BCE016E89
:1000A00084BCBFFDC12F3D6C74319ABD56833DDACF
:1000B0003D00C77F11BED9E4BB4C3E916BAAAABEDE
:1000C000000000803F05A84CCDB2D44EB93836A907
:1000D000020C50B9918688083CA6AAAA2ABE000044
:1000E00000803F6563686F3A0020746F6F206C6F0B
:1000F0006E6720657874727573696F6E20707265B3
:1001000076656E7465640020636F6C642065787436
:10011000727573696F6E2070726576656E74656452
:10012000002D2D3A2D2D002D2D2D005344000120A2
:10013000000120000120004D323100496E69742E0B
:100140002053442D43617264004E6F2043617264FA
:10015000004D3231004368616E67652053442D4382
:10016000617264005072696E742066726F6D205304
:10017000440053746F70205072696E74005265733E
:10018000756D65205072696E7400506175736520DD
:100190005072696E7400436F6E74726F6C005072AF
:1001A00065706172650054756E6500496E666F20FA
:1001B00073637265656E00052E2E000452656672CB
:1001C000657368004D61696E004D3234004D323305
:1001D000202573004D383420582059205A204500DE
:1001E000526573746F7265204661696C73616665F0
:1001F000004C6F6164206D656D6F72790053746F90
:100200007265206D656D6F7279004D6F74696F6EE8
:100210000054656D7065726174757265004D616939
:100220006E004573746570732F6D6D004573746552
:1002300070732F6D6D005A73746570732F6D6D0040
:100240005A73746570732F6D6D0059737465707394
:100250002F6D6D005973746570732F6D6D00587339
:10026000746570732F6D6D005873746570732F6DA6
:100270006D00412D7265747261637400412D726569
:10028000747261637400416D6178206500416D6135
:1002900078206500416D6178207A00416D61782099
:1002A0007A00416D6178207900416D617820790094
:1002B000416D6178207800416D6178207800565456
:1002C000726176206D696E005654726176206D6998
:1002D0006E00566D696E00566D696E00566D6178E0
:1002E000206500566D6178206500566D6178207A32
:1002F00000566D6178207A00566D6178207900563D
:100300006D6178207900566D6178207800566D61B6
:100310007820780056652D6A65726B0056652D6AE7
:1003200065726B00567A2D6A65726B00567A2D6A7B
:1003300065726B005678792D6A65726B0056787914
:100340002D6A65726B00416363656C004163636590
:100350006C00436F6E74726F6C00507265686561FB
:10036000742041425320436F6E6600507265686589
:10037000617420504C4120436F6E66005049442DFB
:1003800043005049442D43005049442D44005049F6
:10039000442D44005049442D49005049442D490002
:1003A0005049442D50005049442D50002002204611
:1003B0006163740020022046616374002002204DB6
:1003C0006178002002204D6178002002204D696E86
:1003D000002002204D696E004F6666004F6E2000BF
:1003E0004F6666004F6E20004175746F74656D70C6
:1003F0000046616E2073706565640046616E20730F
:10040000706565640042656400426564004E6F7A01
:100410007A6C6533004E6F7A7A6C6533004E6F7A72
:100420007A6C6532004E6F7A7A6C6532004E6F7A64
:100430007A6C65004E6F7A7A6C6500436F6E7472E9
:100440006F6C0053746F7265206D656D6F7279000B
:1004500042656400426564004E6F7A7A6C65004EB6
:100460006F7A7A6C650046616E2073706565640012
:1004700046616E2073706565640054656D706572C9
:1004800061747572650053746F7265206D656D6F70
:1004900072790042656400426564004E6F7A7A6C3E
:1004A00065004E6F7A7A6C650046616E20737065E8
:1004B00065640046616E2073706565640054656D07
:1004C0007065726174757265004D6F766520417854
:1004D000697300436F6F6C646F776E00507265686C
:1004E00065617420414253005072656865617420F3
:1004F000504C4100473238004175746F20486F6D91
:1005000065004D38340044697361626C6520537432
:10051000657070657273004D61696E004D6F766530
:1005200020302E316D6D004D6F766520316D6D0080
:100530004D6F76652031306D6D005072657061725F
:1005400065004578747275646572004D6F7665203C
:100550005A004D6F76652059004D6F766520580022
:100560004D6F7665204178697300457874727564C3
:100570006572005A0059005800466C6F7700466C4F
:100580006F770046616E2073706565640046616E2A
:100590002073706565640042656400426564004EC6
:1005A0006F7A7A6C6533004E6F7A7A6C6533004EE1
:1005B0006F7A7A6C6532004E6F7A7A6C6532004ED3
:1005C0006F7A7A6C65004E6F7A7A6C65005370654D
:1005D0006564005370656564004D61696E00656314
:1005E000686F3A004572726F723A0053544F505020
:1005F00045442E20005072696E7465722073746FCA
:10060000707065642064756520746F206572726F08
:1006100072732E2046697820746865206572726F47
:100620007220616E6420757365204D3939392074EC
:100630006F20726573746172742E202854656D701A
:100640006572617475726520697320726573657473
:100650002E2053657420697420616674657220725F
:10066000657374617274696E6729004B494C4C451F
:10067000442E20005072696E7465722068616C743B
:1006800065642E206B696C6C28292063616C6C6535
:100690006421006F6B00526573656E643A2000221E
:1006A00000556E6B6E6F776E20636F6D6D616E645B
:1006B0003A202200486F74656E64206F6666736529
:1006C00074733A007A5F6D696E3A2000795F6D69E4
:1006D0006E3A2000785F6D696E3A20005A3A0059F0
:1006E0003A0020436F756E7420583A2000453A0056
:1006F0005A3A00593A00583A004649524D57415229
:10070000455F4E414D453A4D61726C696E205631E0
:100710003B20537072696E7465722F6772626C2031
:100720006D617368757020666F722067656E362024
:100730004649524D574152455F55524C3A68747480
:10074000703A2F2F7777772E6D656E64656C2D70FC
:10075000617274732E636F6D2050524F544F434F2C
:100760004C5F56455253494F4E3A312E30204D4141
:100770004348494E455F545950453A4D656E64654E
:100780006C2045585452554445525F434F554E5482
:100790003A330A0042656420646F6E652E00204281
:1007A0003A0020453A00543A0042656420486561A9
:1007B00074696E672E0048656174696E6720646FA6
:1007C0006E652E0020573A0020453A00543A004802
:1007D000656174696E672E2E2E002042403A00201B
:1007E000403A00202F0020423A00202F006F6B205B
:1007F000543A002569206D696E2C202569207365A7
:100800006300456E642066696C65206C69737400D2
:10081000426567696E2066696C65206C6973740057
:100820004E6F206D6F76652E00526573756D696E23
:1008300067207072696E74005761697420666F7208
:1008400020757365722E2E2E00536C6565702E2EEA
:100850002E000000A0400000A0400000803FFFFFED
:10086000FF256920686F757273202569206D696E98
:100870007574657300446F6E65207072696E74697B
:100880006E672066696C650053544F505045442E86
:1008900020005072696E7465722073746F70706599
:1008A000642064756520746F206572726F72732E98
:1008B0002046697820746865206572726F722061C5
:1008C0006E6420757365204D39393920746F20723C
:1008D0006573746172742E202854656D7065726141
:1008E000747572652069732072657365742E205368
:1008F0006574206974206166746572207265737412
:10090000617274696E6729006F6B004E6F204C69CD
:100910006E65204E756D626572207769746820631C
:100920006865636B73756D2C204C617374204C6922
:100930006E653A20004E6F20436865636B73756D7A
:100940002077697468206C696E65206E756D6265CC
:10095000722C204C617374204C696E653A200063E0
:100960006865636B73756D206D69736D6174636821
:100970002C204C617374204C696E653A20004C69E0
:100980006E65204E756D626572206973206E6F749E
:10099000204C617374204C696E65204E756D6265E4
:1009A000722B312C204C617374204C696E653A2097
:1009B000004D31313000446F6E6520736176696E91
:1009C000672066696C652E006F6B004D3239002020
:1009D00020506C616E6E6572427566666572427912
:1009E0007465733A20002046726565204D656D6F11
:1009F00072793A200041756720203220323031333D
:100A000000436F6D70696C65643A2000286C7761F3
:100A10006C6B6572612C205072696E7472626F74B7
:100A2000206669726D776172652900207C204175AE
:100A300074686F723A20004175672020322032308E
:100A400031332031363A34303A313400204C61733E
:100A50007420557064617465643A2000312E302E24
:100A600030004D61726C696E200020536F667477A0
:100A70006172652052657365740020576174636804
:100A8000646F67205265736574002042726F776EE1
:100A9000206F757420526573657400204578746505
:100AA000726E616C20526573657400506F77657269
:100AB0005570007374617274002200656E71756503
:100AC000696E672022002200656E717565696E6728
:100AD0002022004572726F723A004572723A204DC0
:100AE000415854454D50204245440054656D706551
:100AF00072617475726520686561746564206265F1
:100B000064207377697463686564206F66662E205D
:100B10004D415854454D5020747269676765726540
:100B200064202121004572723A204D494E54454DB2
:100B300050003A2045787472756465722073776945
:100B40007463686564206F66662E204D494E544577
:100B50004D50207472696767657265642021004595
:100B600072723A204D415854454D50003A20457814
:100B70007472756465722073776974636865642044
:100B80006F66662E204D415854454D502074726951
:100B9000676765726564202100202D20496E7661AB
:100BA0006C6964206578747275646572206E756D09
:100BB00062657220210070012C0190012701B001B3
:100BC0002201C0011D01F0011801100213013002C1
:100BD0000E016002090190020401C002FF0000033F
:100BE000FA004003F5008003F000D003EB0020047E
:100BF000E6007004E100E004DC004005D700C00519
:100C0000D2004006CD00D006C8008007C3003008DF
:100C1000BE00F008B900C009B400B00AAF00B00BC4
:100C2000AA00D00CA500000EA000500F9B00C01021
:100C300096005012910000148C00C0158700B01768
:100C40008200B0197D00D01B7800001E7300402088
:100C50006E0090226900F024640040275F00902914
:100C60005A00E02B5500102E500020304B0010325F
:100C70004600E033410090353C00103737007038B3
:100C80003200A0392D00B03A2800A03B2300603C80
:100C90001E00103D1900903D1400103E0F00703EE4
:100CA0000A00C03E0500003F000050494420417545
:100CB000746F74756E652066696E6973686564210A
:100CC0002050757420746865204B702C204B69206F
:100CD000616E64204B6420636F6E7374616E747315
:100CE00020696E746F20436F6E66696775726174F8
:100CF000696F6E2E6800504944204175746F747599
:100D00006E65206661696C6564212074696D656F2C
:100D100075740020403A006F6B20543A006F6B20CE
:100D2000423A00504944204175746F74756E6520D5
:100D30006661696C6564212054656D7065726174CB
:100D400075726520746F6F206869676800204B6456
:100D50003A2000204B693A2000204B703A200020B6
:100D6000436C617369632050494420002054753AF4
:100D70002000204B753A2000206D61783A20002039
:100D80006D696E3A200020643A2000206269617328
:100D90003A200045313A200045303A20005A3A20A6
:100DA00000593A2000583A20004D53312C4D53320F
:100DB0002050696E730A0024F404D9201BC40C5C13
:100DC0000E9804C4095F0265077101F405F900FB80
:100DD00004B30048048700C10369005803550003A9
:100DE000034500BE023A008402310053022A002962
:100DF00002250004022000E4011C00C8011900AF14
:100E000001170098011400840113007101100061A2
:100E100001100051010E0043010D0036010B002BA3
:100E2000010B0020010B00150109000C0109000352
:100E3000010800FB000800F3000800EB000700E4D5
:100E4000000600DE000600D8000600D2000600CC36
:100E5000000500C7000500C2000500BD000400B980
:100E6000000400B5000400B1000400AD000400A9B6
:100E7000000400A5000300A20003009F0004009BE3
:100E80000003009800030095000200930003009007
:100E90000003008D0002008B000300880002008622
:100EA00000020084000300810002007F0002007D38
:100EB0000002007B0002007900020077000100764A
:100EC0000002007400020072000100710002006F55
:100ED0000002006D0001006C0002006A0001006960
:100EE0000002006700010066000100650001006467
:100EF0000002006200010061000100600001005F6B
:100F00000002005D0001005C0001005B0001005A6E
:100F1000000100590001005800010057000100566F
:100F2000000100550001005400010053000000536F
:100F30000001005200010051000100500001004F6B
:100F40000001004E0000004E0001004D0001004C69
:100F50000001004B0000004B0001004A0001004965
:100F60000001004800000048000100470001004661
:100F7000000000460001004500000045000100445B
:100F80000001004300000043000100420000004255
:100F90000001004100000041000100400001003F4D
:100FA0000000003F0001003E0000003E0001003D47
:100FB0000000003D0001003C0000003C0000003C3F
:100FC0000001003B0000003B0001003A0000003A35
:100FD000000100390000003900010038000000382D
:100FE0000000003800010037000000370001003623
:100FF000000000360000003600010035000000351A
:10100000000000350001003400000034000000340E
:101010000001003300000033000000330001003203
:1010200000000032000000320001003100000031F9
:1010300000000031000100300000003000000030EE
:101040000001002F0000002F0000002F0000002FE3
:101050000001002E0000002E0000002E0001002DD7
:101060000000002D0000002D0000002D0001002CCC
:101070000000002C0000002C0000002C0001002BC0
:101080000000002B0000002B0000002B0001002AB4
:101090000000002A0000002A0000002A00010029A8
:1010A000000000290000002900000029000000299C
:1010B000000100280000002800000028000000288F
:1010C0000000002800010027000000270000002782
:1010D0000000002700000027000100260000002675
:1010E0000000002600000026000000260001002568
:1010F000000000250000002500000025000000255C
:10110000000000250001002400000024000000244D
:101110000000002400000024000100230000002340
:101120000000002300000023000000230000002333
:101130000000002300010022000000220000002225
:101140000000002200000022000000220001002117
:10115000000000210000002100000021000000210B
:1011600000000021000000210001002000000020FC
:1011700000000020000000200000002000000020EF
:1011800000000020000000200001001F0000001FE0
:101190000000001F0000001F0000001F0000001FD3
:1011A0000000001F0001001E0000001E0000001EC5
:1011B0000000001E00000024F4D43050C38E20C272
:1011C000A24017828B7011127A910D816CD90AA8F6
:1011D00061E108C7586607615143061E4B5D05C1B2
:1011E00045A7041A411104093D98037139310340A0
:1011F00036DB0265339102D4305402802E1D026327
:101200002CEE01752AC501B028A001102781018F9D
:101210002564012B244B01E0223401AC211F018DF8
:10122000200D01801FFC00841EED00971DDF00B81B
:101230001CD200E61BC600201BBC00641AB200B220
:1012400019A8000A19A0006A189900D11791004046
:10125000178B00B516840031167E00B31579003A5D
:10126000157300C7146F0058146A00EE13660088E7
:1012700013630025135E00C7125B006C1257001544
:10128000125400C111510070114F0021114B00D6B2
:101290001049008D1047004610440002104200C063
:1012A0000F4000800F3E00420F3C00060F3B00CB7A
:1012B0000E3800930E37005C0E3500270E3400F315
:1012C0000D3200C10D3100900D3000600D2E003246
:1012D0000D2D00050D2C00D90C2B00AE0C2900851E
:1012E0000C29005C0C2700350C27000E0C2600E8AA
:1012F0000B2400C40B2400A00B23007D0B23005AF9
:101300000B2100390B2100180B2000F80A1F00D90F
:101310000A1E00BB0A1E009D0A1D00800A1D0063F4
:101320000A1C00470A1B002C0A1B00110A1A00F7AE
:10133000091A00DD091900C4091900AB0919009246
:101340000917007B091800630917004C09160036BD
:10135000091600200916000A091500F5081500E015
:10136000081400CC081400B8081400A40814009055
:101370000813007D0812006B08130058081200467D
:10138000081200340811002308110012081100018E
:10139000081100F0071000E0071000D0071000C08F
:1013A000071000B0070F00A107100091070E00837F
:1013B000070F0074070F0065070E0057070E00495E
:1013C000070E003B070D002E070E0020070D00132F
:1013D000070D0006070D00F9060C00ED060D00E0F4
:1013E000060C00D4060C00C8060C00BC060C00B0AD
:1013F000060C00A4060B0099060C008D060B00825B
:10140000060B0077060B006C060B0061060A0057FE
:10141000060B004C060A0042060A0038060A002E97
:10142000060A0024060A001A060A00100609000728
:10143000060A00FD050900F4050900EB050900E2B4
:10144000050900D9050900D0050900C7050900BE36
:10145000050900B5050800AD050800A50509009CB3
:10146000050800940508008C050800840508007C28
:10147000050800740508006C050700650508005D97
:10148000050700560508004E050700470507004000
:1014900005080038050700310507002A0507002365
:1014A0000507001C050600160507000F05070008C4
:1014B00005060002050700FB040600F5040700EE20
:1014C000040600E8040600E2040700DB040600D579
:1014D000040600CF040600C9040600C3040600BDCC
:1014E000040600B7040600B1040500AC040600A61B
:1014F000040600A00405009B040600950405009066
:101500000406008A04050085040500800406007AAC
:1015100004050075040500700405006B04050066F1
:10152000040500610405005C040500570405005231
:101530000405004D04050048040500430405003E71
:101540000404003A04050035040500300404002CAE
:1015500004050027040400230405001E0404001AE7
:1015600004040016040500110404000D040400091D
:101570000405000404040000040400FC030400F853
:10158000030400F4030400F0030400EC030400E887
:10159000030400E4030400E0030400DC030400D8B7
:1015A000030400D4030400D0030400CC030400C8E7
:1015B000030300C50303006563686F3A00656E644A
:1015C00073746F7073206869743A205A00205A3A15
:1015D00000656E6473746F7073206869743A205983
:1015E0000020593A00656E6473746F7073206869E7
:1015F000743A20580020583A00656E6473746F7016
:1016000073206869743A20007C3C3E5E2B3D3F2F7E
:101610005B5D3B2C2A225C006563686F3A00486181
:101620007264636F6465642044656661756C7420E0
:1016300053657474696E6773204C6F6164656400F0
:1016400053746F7265642073657474696E67732078
:1016500072657472696576656400205A00205900CD
:1016600020204D3231312058004D617820706F7349
:101670006974696F6E20286D6D293A00205A002028
:10168000590020204D3231302058004D696E2070B5
:101690006F736974696F6E20286D6D293A0020445C
:1016A000002049002020204D333031205000504987
:1016B000442073657474696E67733A00205A002081
:1016C000590020204D323036205800486F6D65207B
:1016D0006F666673657420286D6D293A0020450099
:1016E000205A0020580020420020540020204D3273
:1016F0003035205300416476616E63656420766105
:10170000726961626C65733A20533D4D696E206663
:101710006565647261746520286D6D2F73292C20B6
:10172000543D4D696E2074726176656C2066656506
:10173000647261746520286D6D2F73292C20423DE1
:101740006D696E696D756D207365676D656E74206A
:1017500074696D6520286D73292C20583D6D617862
:10176000696D756D205859206A65726B20286D6D02
:101770002F73292C20205A3D6D6178696D756D207D
:101780005A206A65726B20286D6D2F73292C2020DA
:10179000453D6D6178696D756D2045206A65726B98
:1017A00020286D6D2F73290020540020204D3230E9
:1017B00034205300416363656C65726174696F6EB8
:1017C0003A20533D616363656C65726174696F6E45
:1017D0002C20543D7265747261637420616363658B
:1017E0006C65726174696F6E00204500205A00209C
:1017F000590020204D3230312058004D6178696DFC
:10180000756D20416363656C65726174696F6E20EC
:10181000286D6D2F7332293A00204500205A002090
:10182000590020204D3230332058004D6178696DC9
:10183000756D2066656564726174657320286D6DD1
:101840002F73293A00204500205A002059002020FB
:101850004D393220580053746570732070657220C2
:10186000756E69743A0053657474696E67732053BA
:10187000746F726564004D383420582059205A2006
:1018800045006563686F3A0043616E6E6F74206552
:101890006E746572207375626469723A20004D320D
:1018A00034004D3233202573006175746F25692E25
:1018B00067004572726F723A006572726F722077BC
:1018C000726974696E6720746F2066696C65004E7A
:1018D0006F74205344207072696E74696E67002FB4
:1018E000005344207072696E74696E672062797467
:1018F0006520002E0044656C6574696F6E2066611A
:10190000696C65642C2046696C653A200046696CF8
:10191000652064656C657465643A002E006F7065BF
:101920006E206661696C65642C2046696C653A209E
:101930000057726974696E6720746F2066696C6500
:101940003A20002E006F70656E206661696C6564D8
:101950002C2046696C653A20002E006F70656E2061
:101960006661696C65642C2046696C653A200046A6
:10197000696C652073656C656374656400205369E8
:101980007A653A200046696C65206F70656E656403
:101990003A20002E006F70656E206661696C656488
:1019A0002C2046696C653A200053442063617264C0
:1019B000206F6B006F70656E526F6F742066616987
:1019C0006C656400766F6C756D652E696E69742048
:1019D0006661696C656400534420696E69742066B1
:1019E00061696C000129022904290829102920298C
:1019F00040298029012C022C0126022604260826D3
:101A00001026202640268026402C802C01230223ED
:101A100004230823102320234023802301200220B5
:101A2000042008201020202040208020102C202C72
:101A3000012F022F042F082F102F202F402F802F2F
:101A40007EFE7EFD7EFB7EF77EEF7EDF7EBF7E7FAD
:101A500000010000841A1200020000961A430003DD
:101A60000000D91A0401030904DD1A18020309044D
:101A7000F71A16030309040F1B0C0001C1020180B1
:101A8000360181361201000202000020C0168304D4
:101A900000010102030109024300020100C03209F2
:101AA00004000001020201000524001001052401C8
:101AB000000104240206052406000107058203082C
:101AC000004009040100020A00000007050302406B
:101AD00000000705840240000004030904180354B1
:101AE00000650065006E0073007900640075006990
:101AF000006E006F000000160355005300420020E6
:101B000000530065007200690061006C0000000C69
:101B100003310032003300340035000000494E46E6
:101B2000494E4954594E414ECDCCCC3D0AD7233C69
:101B300017B7D13877CC2B329595E6241FB14F0AD1
:101B4000000020410000C84200401C4620BCBE4CA2
:101B5000CA1B0E5AAEC59D74B26EB17B74CE3DDA0F
:101B6000AC7B11241FBECFEFD0E2DEBFCDBF13E0B0
:101B7000A0E0B1E0ECE3F0EC01E00BBF02C00790A5
:101B80000D92AA3BB107D9F71BBE11E1AAEBB3E056
:101B900001C01D92A136B107E1F71BE1C0E6DBE110
:101BA00004C02297FE010E94C4DFC835D107C9F7DF
:101BB0000E94ADDA0C9412E00C940000A0E0B0E0BA
:101BC000E4EEFDE00C94E1DFEC015B0161157105D1
:101BD00019F0FB0191838083F9908F2D90E00E9492
:101BE000C8DF892BC9F7FDE2FF1621F4F990EE2436
:101BF000E39405C02BE2F21609F4F990EE248E016D
:101C000001501040C8016DE17BE143E050E072D229
:101C1000892BF9F48E010E5F1F4FC80160E27BE152
:101C200045E050E067D2892B19F48E01095F1F4F00
:101C3000A114B10419F0F50111830083E0FC04C084
:101C400070E090E080E813C070E090E080E86FEF13
:101C500007C1C80165E27BE143E050E04BD2892B2C
:101C600069F4A114B10429F470E090E080EC6FE70E
:101C7000F7C02296F501D183C083F6CF882499243A
:101C800040E050E060E070E0EF2DE053EA30A0F576
:101C9000F2E0EF2A8E2D90E09C0128703070E2FE79
:101CA00006C0232B79F50894811C911C2BC0232B93
:101CB00019F0089481089108DB01CA0112E0880F2D
:101CC000991FAA1FBB1F1A95D1F7480F591F6A1FEA
:101CD0007B1F440F551F661F771F4E0F511D611D3F
:101CE000711D483929E9520729E9620729E172077C
:101CF00048F084E0E82A06C0EE3F31F4E3FC39C046
:101D000098E0E92AF990C0CFE53311F0E53189F583
:101D100029912D3219F4E0E1EE2A05C02B3219F099
:101D200081E090E003C0299182E090E0E22FE0534F
:101D3000EA3018F0C81BD90B1CC020E030E0FCE0F2
:101D400020383F075CF4C901880F991F880F991F3D
:101D5000280F391F220F331F2E0F311DE991E05339
:101D6000EA3068F3E4FE03C0309521953F4F820EC0
:101D7000931ECE2CDD24E1FE07C0A114B10421F096
:101D80002197F501D183C083CB01BA010E942DDCDC
:101D90007B018C01F3E0CF22DD2423E0C216D104C5
:101DA00021F417FB109517F9109557016801C80128
:101DB000B70120E030E040E050E00E948DDB882356
:101DC00009F44AC097FE0DC02CE3E22E2BE1F22E5F
:101DD0009094819491089394C0E2D0E000E010E0E8
:101DE00012C094E5E92E9BE1F92EF6CFF70125917B
:101DF000359145915491C601B5010E946DDE5B019C
:101E00006C018C1A9D0A8C169D0684F7D595C79592
:101E10000F5F1F4F0630110529F08CEF9FEFE80E82
:101E2000F91EF1CFC501D6017C018D018C2D880FE3
:101E30008D2D881F8F3F51F0C601B50120E030E0A5
:101E400040E050E00E948DDB882331F482E290E094
:101E50009093601180935F117E2D9F2D802F612FB5
:101E6000272F392F482F562FB901CA01CDB7DEB71A
:101E7000ECE00C94FDDF2F923F925F926F927F9285
:101E80008F929F92AF92BF92CF92DF92EF92FF928A
:101E90000F931F93CF93DF938C011B01EA01611510
:101EA000710519F0FB0191838083209749F0CE01E1
:101EB0000297839728F020E030E040E050E0F6C041
:101EC000F801A1908F018A2D90E00E94C8DF892B34
:101ED000B9F7FDE2AF1631F4F801A1908F01552456
:101EE000539407C0FBE2AF1619F4F801A1908F01DB
:101EF0005524209719F0C031D105C1F4F0E3AF1695
:101F000079F4F8018081883711F0883549F4F801B7
:101F1000A1800E5F1F4FF2E05F2AC0E1D0E006C053
:101F2000209721F480E3A816E9F427C0C830D10532
:101F300031F1C930D10524F4C230D10531F50CC0DE
:101F4000CA30D10589F0C031D105F9F4C12CD12CAA
:101F5000E12CB8E0FB2E28C0C12CD12CE12CA0E450
:101F6000FA2E22C0CAE0D0E0FCECCF2EFCECDF2E33
:101F7000FCECEF2EFCE0FF2E17C0C8E0D0E0C12C37
:101F8000D12CE12CE0E1FE2E0FC09E01442737FD4D
:101F90004095542F60E070E080E090E80E9485DF7B
:101FA000C901DA016C017D0120E030E040E050E041
:101FB00060E03E01882477FC8094982C70EDB72E69
:101FC000BA0CE9E0EB1570F48A2D81548A3118F4CB
:101FD00099ECB92E06C08A2D81568A3150F589EACE
:101FE000B82EBA0C8B2D90E08C179D0714F56F3F1F
:101FF000E1F0C216D306E406F506B0F0CA01B90155
:10200000A40193010E943FDF9B01AC012B0D311D08
:10201000411D511D2130F0E03F07F0E04F07F0E88F
:102020005F0710F461E001C06FEFF801A1908F012C
:10203000C5CF2114310481F0662331F001501040E6
:10204000F1011183008308C051FE1AC002501040F4
:10205000F1011183008314C067FF12C050FC05C05A
:102060002FEF3FEF4FEF5FE704C020E030E040E0AC
:1020700050E882E290E09093601180935F1116C067
:1020800050FE08C050954095309521953F4F4F4FD9
:102090005F4F0CC057FF0AC082E290E0909360113E
:1020A00080935F112FEF3FEF4FEF5FE7B901CA0158
:1020B000DF91CF911F910F91FF90EF90DF90CF9024
:1020C000BF90AF909F908F907F906F905F903F9068
:1020D0002F900895FB01DC0105900D920020E1F79F
:1020E0000895FC0105900020E9F7809590958E0FEA
:1020F0009F1F0895FB01DC014150504088F08D91F5
:1021000081341CF08B350CF4805E659161341CF0D9
:102110006B350CF4605E861B611171F3990B0895A9
:10212000881BFCCFFB01DC014150504048F005907A
:102130000D920020C9F701C01D9241505040E0F7B8
:102140000895FB0155915523A9F0BF01DC014D9184
:1021500045174111E1F759F4CD010590002049F0F0
:102160004D9140154111C9F3FB014111EFCF81E0C1
:1021700090E001970895FB01DC0104C08D9101906E
:10218000801921F441505040C8F7881B990B0895DD
:10219000FB01DC0102C001900D9241505040D8F784
:1021A0000895FB01DC010D900020E9F711970190E3
:1021B0000D920020E1F70895FC018191861721F02E
:1021C0008823D9F7992708953197CF010895FB0106
:1021D000DC0101900D920020E1F70895FB01DC0184
:1021E0004150504030F08D910190801919F4002039
:1021F000B9F7881B990B0895FB01DC014150504051
:1022000048F001900D920020C9F701C01D92415085
:102210005040E0F70895AEE0B0E0E1E1F1E10C9468
:10222000E9DF0D891E898EE08C831A8309838FEF85
:102230009FE79E838D839E01275E3F4FCE010196CF
:102240006F89788DA9010AD02F813885020F131F5D
:10225000F80110822E96E4E00C9405E0ABE0B0E0CB
:10226000E4E3F1E10C94DBDF3C012B015A01FC01BA
:1022700017821682838181FD03C06FEF7FEFB9C1A2
:102280009AE0892E1E010894211C311CF301238140
:10229000F20123FD859123FF81912F01882309F409
:1022A000A5C1853239F423FD859123FF81912F014A
:1022B000853221F490E0B301B7D1E8CF982FFF2405
:1022C000EE249924FFE1FF15D0F09B3269F09C3297
:1022D00028F4903259F0933291F40EC09D3249F0B7
:1022E000903369F441E024C052E0F52A84E0F82AF2
:1022F00028C098E0F92A25C0E0E1FE2A22C0F7FCB8
:1023000029C0892F80538A3070F4F6FE05C0989C4E
:10231000902C1124980E15C0E89CE02C1124E80E96
:10232000F0E2FF2A0EC09E3229F4F6FC5FC140E4C1
:10233000F42A07C09C3619F450E8F52A02C09836F2
:1023400049F4F20123FD959123FF91912F019923E7
:1023500009F0B8CF892F8554833018F0805283302C
:1023600038F444E050E0A40EB51E5FE359830FC07B
:10237000933631F0933779F0933509F052C01FC08E
:10238000F5018081898342E050E0A40EB51E610111
:1023900001E010E011C0F501C080D180F6FC03C05F
:1023A0006FEF7FEF02C0692D70E042E050E0A40EB5
:1023B000B51EC6012ED18C015FE7F52213C0F501D1
:1023C000C080D180F6FC03C06FEF7FEF02C0692DA3
:1023D00070E042E050E0A40EB51EC6010FD18C01A2
:1023E00050E8F52AF3FE06C018C080E290E0B30181
:1023F0001BD1EA948E2D90E008171907B0F30DC099
:10240000F601F7FC8591F7FE81916F0190E0B30131
:102410000BD1E110EA94015010400115110581F72C
:10242000E2C0943611F0993661F5F7FE08C0F50167
:10243000208131814281538184E090E00AC0F5011E
:10244000808191819C01442737FD4095542F82E083
:1024500090E0A80EB91E9FE6F92257FF09C05095DB
:102460004095309521953F4F4F4F5F4FE0E8FE2A52
:10247000CA01B901A1012AE030E002D1D82ED21858
:102480003FC0953729F41F2D1F7E2AE030E01DC084
:102490001F2D197F9F3661F0903720F4983509F091
:1024A000A5C00FC0903739F0983709F09FC004C01D
:1024B00028E030E00AC0106114FD146020E130E033
:1024C00004C014FD166020E132E017FF08C0F501DA
:1024D000608171818281938144E050E008C0F50100
:1024E00080819181BC0180E090E042E050E0A40E48
:1024F000B51EA101C5D0D82ED2188FE7F82EF12233
:10250000F6FE0BC05EEFF522D91438F4F4FE07C0D6
:10251000F2FC05C08FEEF82202C01D2D01C0192D5E
:10252000F4FE0DC0FE01ED0DF11D8081803319F424
:1025300099EEF92208C01F5FF2FE05C003C08F2D7F
:10254000867809F01F5F0F2DF3FC13C0F0FE0EC05C
:102550001E1510F09D2C0AC09D2C9E0C911A1E2D4C
:1025600005C080E290E0B3015FD01F5F1E15C8F385
:1025700004C01E1510F4E11A01C0EE2404FF0EC0C1
:1025800080E390E0B30150D002FF1BC001FD03C007
:1025900088E790E00EC088E590E00BC0802F867839
:1025A00081F001FF02C08BE201C080E2F7FC8DE206
:1025B00090E0B30139D005C080E390E0B30134D09E
:1025C0009A94D914C8F3DA94F101ED0DF11D8081CC
:1025D00090E0B30129D0DD20B1F705C080E290E0A2
:1025E000B30122D0EA94EE20C9F750CEF301668100
:1025F0007781CB012B96E2E10C94F7DFFC0105908B
:10260000615070400110D8F7809590958E0F9F1FF4
:102610000895FC016150704001900110D8F7809539
:1026200090958E0F9F1F08950F931F93CF93DF9365
:102630008C01EB018B8181FF1BC082FF0DC02E81BD
:102640003F818C819D812817390764F4E881F981E5
:102650000193F983E88306C0E885F985802F099501
:10266000892B31F48E819F8101969F838E8302C0D6
:102670000FEF1FEFC801DF91CF911F910F910895C8
:10268000FA01AA27283051F1203181F1E8946F93A3
:102690006E7F6E5F7F4F8F4F9F4FAF4FB1E03ED049
:1026A000B4E03CD0670F781F891F9A1FA11D680FE7
:1026B000791F8A1F911DA11D6A0F711D811D911D1A
:1026C000A11D20D009F468943F912AE0269F11248F
:1026D0003019305D3193DEF6CF010895462F4770F3
:1026E000405D4193B3E00FD0C9F7F6CF462F4F704E
:1026F000405D4A3318F0495D31FD4052419302D0AC
:10270000A9F7EACFB4E0A695979587957795679551
:10271000BA95C9F700976105710508959B01AC0151
:102720000A2E06945795479537952795BA95C9F778
:10273000620F731F841F951FA01D08958091C0050F
:10274000882399F14091BA035091BB036091BC0377
:102750007091BD038091BE059091BF052EEB33E0D3
:102760000E942375882319F14091C1055091C2053B
:102770006091C3057091C40541155105610571054E
:1027800091F08091BE059091BF052EEB33E00E9441
:102790002375882361F01092C1051092C205109232
:1027A000C3051092C4051092C00581E0089580E031
:1027B0000895DF92EF92FF920F931F937B018C019C
:1027C000D42E8091BA039091BB03A091BC03B09129
:1027D000BD038E159F05A007B107B9F0AFDF8823B1
:1027E000E1F08091BE059091BF05B801A7012EEBE5
:1027F00033E00E94F875882381F0E092BA03F092EA
:10280000BB030093BC031093BD03DD2011F481E0F2
:1028100005C081E08093C00501C080E01F910F9149
:10282000FF90EF90DF9008958F929F92AF92BF92AA
:10283000CF92DF92EF92FF920F931F93CF93DF938C
:102840006C01142F7093BF056093BE05FC01178ABD
:1028500082E090E0A0E0B0E080839183A283B38324
:102860001092C0051092C1051092C2051092C305C6
:102870001092C4058FEF9FEFAFEFBFEF8093BA03C5
:102880009093BB03A093BC03B093BD03442321F4F6
:102890008824992454013FC0453008F01CC160E0F1
:1028A00070E080E090E040E084DF882309F413C109
:1028B000C12FD0E02197FE0174E0EE0FFF1F7A9543
:1028C000E1F7E254FC4FE254FE4F8081EE5BF140B1
:1028D00090E08F779070892B09F0FDC0E653FE4F92
:1028E00080819181A281B38184369105A105B105D2
:1028F00008F4F1C064E0CC0FDD1F6A95E1F7CC5716
:10290000DA4F88809980AA80BB8081149104A10449
:10291000B10409F4E0C0C501B40140E04ADF8823F6
:1029200009F4D9C08091C9039091CA0380509240A4
:1029300009F0D1C02091CE03222309F4CCC08091AC
:10294000CC039091CD03892B09F4C5C08091CB03B2
:10295000882309F4C0C0F601228B8091CB038483C5
:10296000158661E070E007C04F5FF6014587415072
:10297000483008F0B0C0F6014585848190E09B01A5
:10298000042E02C0220F331F0A94E2F78217930726
:1029900059F72091D4033091D5032115310519F051
:1029A00040E050E008C02091E2033091E303409101
:1029B000E4035091E503F60125833683478350876E
:1029C000E090CC03F090CD0300E010E0E80CF91C9F
:1029D0000A1D1B1DE38AF48A058B168B8091CF0399
:1029E0009091D003918F808F6091CE0370E080E052
:1029F00090E00E943FDF6E0D7F1D801F911FF6014A
:102A0000628F738F848F958F2091CF033091D00385
:102A100055E0220F331F5A95E1F721503E4F232FE7
:102A20003327269540E050E0260F371F481F591FD7
:102A300026873787408B518B8091D1039091D203A9
:102A4000009719F0A0E0B0E008C08091DE039091FB
:102A5000DF03A091E003B091E10385017401E21A64
:102A6000F30A040B150BA8019701280F391F4A1F01
:102A70005B1FF601058404C0569547953795279549
:102A80000A94D2F72187328743875487253FFFE096
:102A90003F07F0E04F07F0E05F0720F48CE0F6011D
:102AA000878B19C0255F3F4F4040504018F480E1AC
:102AB000F6010EC08091EA039091EB03A091EC0324
:102AC000B091ED03F601828F938FA48FB58F80E2D2
:102AD000878B81E001C080E0DF91CF911F910F9142
:102AE000FF90EF90DF90CF90BF90AF909F908F902E
:102AF00008956F927F928F929F92AF92BF92CF92E2
:102B0000DF92EF92FF920F931F93CF93DF93EC012D
:102B10005A016B01380149014230510561057105C7
:102B200008F45DC089859A85AB85BC850196A11D99
:102B3000B11D84179507A607B70708F450C08F8901
:102B4000803129F4E52EF62E072F11270CC0803294
:102B500009F045C07A018B0187E016950795F79437
:102B6000E7948A95D1F78B899C89AD89BE89E80E57
:102B7000F91E0A1F1B1FC801B70141E01ADE882396
:102B800071F18F89803149F4F501F070EE0FFF1F6C
:102B9000E254FC4F718260820DC0F501EF77F07056
:102BA000EE0FFF1FEE0FFF1FE254FC4F6082718299
:102BB000828293828A89823080F08D819E81AF816A
:102BC000B885E80EF91E0A1F1B1FE092C105F0929E
:102BD000C2050093C3051093C40581E001C080E0E5
:102BE000DF91CF911F910F91FF90EF90DF90CF90E9
:102BF000BF90AF909F908F907F906F900895CF92ED
:102C0000DF92EF92FF920F931F93CF93DF93EC012C
:102C10007A018B01690189859A85AB85BC8501960E
:102C2000A11DB11D84179507A607B70708F452C068
:102C30008F89803129F45527412F302F2F2D0CC03B
:102C4000803209F047C09A01AB0167E0569547957D
:102C5000379527956A95D1F78B899C89AD89BE896F
:102C6000280F391F4A1F5B1F8091BA039091BB0345
:102C7000A091BC03B091BD03281739074A075B0731
:102C800031F0CA01B90140E094DD882319F18F8940
:102C9000803159F4F701F070EE0FFF1FE254FC4F42
:102CA00080819181A0E0B0E00EC0F701EF77F07075
:102CB000EE0FFF1FEE0FFF1FE254FC4F808191814A
:102CC000A281B381BF70F60180839183A283B38315
:102CD00081E001C080E0DF91CF911F910F91FF90C3
:102CE000EF90DF90CF900895AF92BF92CF92DF9296
:102CF000EF92FF920F931F93DF93CF9300D000D0FA
:102D0000CDB7DEB76C017A018B0182E090E0A0E0E4
:102D1000B0E0F60180839183A283B3835E010894BF
:102D2000A11CB11CC601B801A701950168DF882369
:102D300039F1C601B801A70100E010E020E030E061
:102D4000D8DE8823E9F0E980FA800B811C81F60146
:102D50008789803151F4F8EFEF16FFEFFF06F0E0BE
:102D60000F07F0E01F07F0F209C088EFE8168FEFB9
:102D7000F8068FEF08078FE01807A0F281E001C086
:102D800080E00F900F900F900F90CF91DF911F91E7
:102D90000F91FF90EF90DF90CF90BF90AF9008958C
:102DA0004F925F926F927F928F929F92AF92BF925B
:102DB000CF92DF92EF92FF920F931F93DF93CF9307
:102DC00000D000D0CDB7DEB76C0149835A836B8346
:102DD0007C833901EE24FF2487012E010894411CD5
:102DE000511C812CE2E09E2EA12CB12C49815A81EC
:102DF0006B817C81C601920102DF882339F1D50104
:102E0000C401F601058404C0880F991FAA1FBB1FC7
:102E10000A94D2F7E80EF91E0A1F1B1F29813A8176
:102E20004B815C818789803131F4285F3F4F40407E
:102E30005040E0F205C0285F3F4F4F4F5F40B0F277
:102E4000F301E082F1820283138381E00F900F90FF
:102E50000F900F90CF91DF911F910F91FF90EF9006
:102E6000DF90CF90BF90AF909F908F907F906F90AA
:102E70005F904F9008952F923F924F925F926F9282
:102E80007F928F929F92AF92BF92CF92DF92EF92FA
:102E9000FF920F931F93DF93CF93CDB7DEB72F979A
:102EA0000FB6F894DEBF0FBECDBF1C014A875B870B
:102EB0006C877D873F872E87DC0119968D919D91C8
:102EC0000D90BC91A02D0196A11DB11D8E839F83F5
:102ED000A887B987F9010081118122813381011509
:102EE00011052105310549F0480159010894811C5B
:102EF000911CA11CB11C1D8210C0D1018D909D9010
:102F0000AD90BC901D828A859B85AC85BD8501975F
:102F1000A105B10511F491E09D837501640144247C
:102F2000552432018E010F5F1F4FF101818592857B
:102F3000A385B485481659066A067B0608F08CC03E
:102F40008E819F81A885B9858C159D05AE05BF052D
:102F500050F4A2E0CA2ED12CE12CF12CF2E08F2EFD
:102F6000912CA12CB12CC101B701A601980147DE1B
:102F7000882309F471C089819A81AB81BC81A70142
:102F800096012F5F3F4F4F4F5F4F0097A105B1054F
:102F900019F049015A010DC0281939094A095B097C
:102FA0008A859B85AC85BD85281739074A075B074D
:102FB00059F00894411C511C611C711C0894C11CDF
:102FC000D11CE11CF11CB1CFC101A601B7010FEF6B
:102FD0001FEF2FEF3FE08DDD882391F43DC02601E8
:102FE000370108944108510861087108C101B30113
:102FF000A201970186017DDD882371F173016201D1
:103000008C149D04AE04BF0450F3AE85BF854D9172
:103010005D916D917C91411551056105710531F00E
:10302000C1019501840165DD8823B1F0EE85FF853E
:1030300080829182A282B382FD81FF2359F008949D
:10304000811C911CA11CB11CD1018D929D92AD924D
:10305000BC92139781E001C080E02F960FB6F894E0
:10306000DEBF0FBECDBFCF91DF911F910F91FF90BB
:10307000EF90DF90CF90BF90AF909F908F907F9018
:103080006F905F904F903F902F9008953F924F9296
:103090005F926F927F928F929F92AF92BF92CF92E8
:1030A000DF92EF92FF920F931F93CF93DF93809164
:1030B0003506882309F4F6C08090380290903902D2
:1030C000A0903A02B0903B026091930F7091940FE0
:1030D000882777FD8095982F0E942FDC20E030E034
:1030E00040E050E40E94B4DAA50194010E948DDB17
:1030F00087FDD8C03090070B0F2EF0E04F2EF0E088
:103100005F2EF0E06F2EF0E07F2EF02DCDE4D0E0CA
:1031100058C0232D30E02C9FF0012D9FF00D3C9FD7
:10312000F00D1124EA5CF94F80819181A281B38175
:103130000097A105B10581F484819581A681B781AD
:103140000097A105B10541F480859185A285B385DD
:103150000097A105B10591F12C9F60012D9FD00C26
:103160003C9FD00C112486E396E0C80ED91EF601D0
:1031700064857585868597850E942FDC7B018C018F
:10318000F60160897189828993890E942DDC9B01F7
:10319000AC01C801B7010E9494DBF60122A133A162
:1031A00044A155A10E946DDE7B018C01A301920117
:1031B0000E949BDD181614F4270138013394FFE0B8
:1031C0003F228091060B381609F0A3CFC301B2014C
:1031D00020913C0230913D0240913E0250913F02CD
:1031E0000E946DDE9B01AC01C501B4010E94B4DAFE
:1031F0007B018C01A50194010E948DDB87FD02C03B
:10320000470158011091340200913502F0903602C6
:10321000E0903702C501B401212F302F4F2D5E2DD4
:103220000E949BDD181634F4812F902FAF2DBE2DF8
:103230004C015D0140901C0B50901D0B60901E0BCB
:1032400070901F0BC301B201A50194010E949BDD88
:103250001816C4F4C501B40120E037ED43EA5CE37D
:103260000E946DDE7B018C01C301B20128E431EEC6
:103270004AE75FE30E946DDEA80197010E94B4DA7D
:103280004B015C0180921C0B90921D0BA0921E0BB7
:10329000B0921F0BC501B4010E94FCDB7093940F28
:1032A0006093930FDF91CF911F910F91FF90EF905B
:1032B000DF90CF90BF90AF909F908F907F906F9056
:1032C0005F904F903F900895E091B20D9091070B61
:1032D0008091060B981711F43E2F30C04091070BD8
:1032E000242F30E08DE490E0289FF001299FF00D1D
:1032F000389FF00D1124E258F94F308120E06DE441
:1033000070E016C0842F90E0869FF001879FF00D3B
:10331000969FF00D1124EA5CF94F80859185A28576
:10332000B3850097A105B10509F02F5F4F5F4F707E
:103330008091060B481731F7222309F4479A3E9AE9
:10334000832F90E090939900809398008091900053
:103350008068809390009ACE8091060B9091070B25
:10336000891B8F700895609340027093410280938F
:1033700042029093430208950F931F93CF93DF93DC
:10338000C0E0D0E08E010B5E194FFE01E751FA4F0D
:1033900060817181828193810E942DDCFE01E75260
:1033A000FA4F20813181428153810E946DDE0E945B
:1033B00001DCF80160837183828393832496C0319A
:1033C000D10501F7DF91CF911F910F910895FC0175
:1033D00060817181828193812091E5053091E605BC
:1033E0004091E7055091E8050E946DDE0E943DDEA8
:1033F00060933106709332068093330690933406BF
:1034000081E396E00C9414A8AF92BF92CF92DF9222
:10341000EF92FF920F931F93FC017B016A01590108
:1034200060817181828193812091D9053091DA0583
:103430004091DB055091DC050E946DDE0E943DDE6F
:1034400005E216E060932506709326068093270612
:1034500090932806F7016081718182819381209188
:10346000DD053091DE054091DF055091E0050E94B9
:103470006DDE0E943DDE6093290670932A068093DC
:103480002B0690932C06F6016081718182819381D5
:103490002091E1053091E2054091E3055091E4056A
:1034A0000E946DDE0E943DDE28E0E22EF12CE00E4F
:1034B000F11E60932D0670932E0680932F06909335
:1034C0003006F50160817181828193812091E5054B
:1034D0003091E6054091E7055091E8050E946DDEC8
:1034E0000E943DDE9801245F3F4F60933106709348
:1034F00032068093330690933406C8010C5F1F4F49
:10350000B801A7010E94DAA780E090E0A0E0B0E057
:103510008093080B9093090BA0930A0BB0930B0BAD
:1035200080930C0B90930D0BA0930E0BB0930F0B8D
:103530008093100B9093110BA093120BB093130B6D
:103540008093140B9093150BA093160BB093170B4D
:103550008093180B9093190BA0931A0BB0931B0B2D
:103560001F910F91FF90EF90DF90CF90BF90AF90A1
:1035700008958F929F92AF92BF92CF92DF92EF9277
:10358000FF920F931F93CF93DF93EC016B01009792
:1035900009F45CC08FA9882309F058C0EEA0FFA0F1
:1035A00008A519A5FB01B6A0A7A090A481A4C801F5
:1035B000B7012B2D3A2D492D582D0E948DDB8823E4
:1035C0000CF044C0C801B701A80197010E946DDE4C
:1035D0007B018C016AA97BA98CA99DA9905820E048
:1035E00030E040E050EC0E946DDE2EA53FA548A9DA
:1035F00059A90E946DDE9B01AC01C801B7010E9470
:10360000B4DA0E94DADE7B018C016B2D7A2D892DD4
:10361000982D9701A8010E948DDB882324F4EB2CC0
:10362000FA2C092D182D6B2D7A2D892D982D9701A7
:10363000A8010E948DDB882349F0C701D801F6015B
:1036400086A397A3A0A7B1A781E086ABDF91CF9116
:103650001F910F91FF90EF90DF90CF90BF90AF90B0
:103660009F908F900895EF92FF920F931F93CF93A7
:10367000DF93F090070B00E010E020E030E04DE435
:10368000E42E11C0FE9CE0011124CA5CD94FC9018F
:10369000B801AE016EDF8F2D8F5F803109F480E0BD
:1036A000F82E98018E018091060BF81659F7C90182
:1036B000B80140E050E05DDFDF91CF911F910F91A5
:1036C000FF90EF900895AF92BF92CF92DF92EF926A
:1036D000FF920F931F93CF93DF93EB018A01611544
:1036E000710509F466C04115510509F462C0DAA4F8
:1036F000CBA4BCA4ADA46EA17FA188A599A52D2DB6
:103700003C2D4B2D5A2D0E948DDB882309F451C08E
:103710008FA9882309F043C0F801E6A0F7A000A50F
:1037200011A56D2D7C2D8B2D9A2DA80197010E943E
:103730009BDD1816A4F5C801B701A80197010E94E6
:103740006DDE7B018C016AA97BA98CA99DA990588B
:1037500020E030E040E050EC0E946DDE2EA53FA559
:1037600048A959A90E946DDE9B01AC01C801B701AF
:103770000E94B4DA0E94DADE7B018C016D2D7C2D73
:103780008B2D9A2D9701A8010E948DDB882324F4AC
:10379000ED2CFC2C0B2D1A2DC701D80104C08D2D4A
:1037A0009C2DAB2DBA2D8EA39FA3A8A7B9A781E00E
:1037B0008EABDF91CF911F910F91FF90EF90DF9033
:1037C000CF90BF90AF900895CF92DF92EF92FF928B
:1037D0000F93DF93CF9300D0CDB7DEB78091060B68
:1037E0008FB7F894F090070B8FBF8091060B90E095
:1037F00040968F1991098F7090700497FCF000919A
:10380000060B03500F70CC24DD2440E050E06DE443
:10381000E62E12C0802F002309F480E1082F01500A
:103820000E9DC00111248A5C994F9A838983B60149
:103830004ADFA601C980DA800F1561F70F900F905B
:10384000CF91DF910F91FF90EF90DF90CF9008958F
:103850001092060B1092070B80E1E5E2F6E0DF0123
:103860001D928A95E9F780E090E0A0E0B0E08093B7
:103870000C0B90930D0BA0930E0BB0930F0B80933A
:10388000100B9093110BA093120BB093130B80931A
:10389000140B9093150BA093160BB093170B8093FA
:1038A000180B9093190BA0931A0BB0931B0B8093DA
:1038B000080B9093090BA0930A0BB0930B0B089580
:1038C0002F923F924F925F926F927F928F929F9230
:1038D000AF92BF92CF92DF92EF92FF920F931F931E
:1038E000DF93CF93CDB7DEB766970FB6F894DEBF00
:1038F0000FBECDBF9E8B8D8B6A017B0148015901A4
:10390000DC01D8966D917D918D919C91DB970E9401
:103910002DDC698B7A8B8B8B9C8BA70196010E9487
:103920006DDE0E947ADB0E9401DC6D837E838F83D3
:10393000988769897A898B899C89A50194010E945D
:103940006DDE0E947ADB0E9401DC69837A838B83BF
:103950009C832D813E814F81588528373105410553
:10396000510540F448E750E060E070E04D835E832D
:103970006F83788769817A818B819C816837710533
:103980008105910540F488E790E0A0E0B0E08983EC
:103990009A83AB83BC83AD89BE89AC5BBF4FAD90CE
:1039A000BD90CD90DC901397A454B040BE8BAD8BEE
:1039B000DC966D917D918D919C91DF970E942DDC1D
:1039C0006D877E878F87988BC601B5010E942FDC9B
:1039D0001B012C0120E030E040E050E00E948DDB34
:1039E000882321F4E0E070E060E028C069897A89EA
:1039F0008B899C899B01AC010E946DDE7B018C014F
:103A00006D857E858F8598899B01AC010E946DDE56
:103A10009B01AC01C801B7010E94B3DA7B018C01A4
:103A2000C201B101A20191010E94B4DA9B01AC0173
:103A3000C801B7010E9494DBE62F692F2E2F372F84
:103A4000482F562FB901CA010E947ADB0E94FCDB85
:103A50003B014C01ED89FE89E05CFF4F6081718183
:103A6000828193810E942DDC69877A878B879C876E
:103A700066277727CB016A197B098C099D090E946B
:103A80002FDC5B016C0120E030E040E050E00E9460
:103A90008DDB882321F4E0E070E060E028C06985D8
:103AA0007A858B859C859B01AC010E946DDE7B0134
:103AB0008C0169897A898B899C899B01AC010E9460
:103AC0006DDE9B01AC01C801B7010E94B3DA7B0136
:103AD0008C01C601B501A60195010E94B4DA9B01D3
:103AE000AC01C801B7010E9494DBE62F692F2E2F8D
:103AF000372F482F562FB901CA010E946ADCED8981
:103B0000FE89A088B188C288D38886017501E6182D
:103B1000F708080919090E94FCDBA8019701261B78
:103B2000370B480B590B57FF71C0C201B10120E0A0
:103B300030E040E050E00E948DDB882321F4E0E09B
:103B400070E060E044C0C201B101A20191010E9495
:103B5000B4DA7B018C01C601B5010E942DDC9B010A
:103B6000AC01C801B7010E946DDE7B018C016D853F
:103B70007E858F8598899B01AC010E946DDE9B013B
:103B8000AC01C801B7010E94B3DA7B018C016985E1
:103B90007A858B859C859B01AC010E946DDE9B0123
:103BA000AC01C801B7010E94B4DA7B018C01C201EB
:103BB000B10120E030E040E850E40E946DDE9B015E
:103BC000AC01C801B7010E9494DBE62F692F2E2FAC
:103BD000372F482F562FB901CA010E947ADB0E9465
:103BE000FCDBAC01CB01DA013C014D0197FE03C0C7
:103BF0006624772443016A147B048C049D0410F02E
:103C00003501460120E030E040E050E09FB7F894F5
:103C10006D897E89645B7F4FDB018C91AC54B04031
:103C2000BE8BAD8B882321F5FD01648A758A868A57
:103C3000978A260D371D481D591D58962D933D9383
:103C40004D935C935B972D813E814F815885DC9627
:103C50002D933D934D935C93DF97A05CBF4F2981DB
:103C60003A814B815C812D933D934D935C931397E7
:103C70009FBF66960FB6F894DEBF0FBECDBFCF9143
:103C8000DF911F910F91FF90EF90DF90CF90BF9049
:103C9000AF909F908F907F906F905F904F903F90EC
:103CA0002F9008954F925F927F928F929F92AF9242
:103CB000BF92CF92DF92EF92FF920F931F93CF9319
:103CC000DF937090070BC0E0D0E07DE4472E512CCD
:103CD00045C02097A9F18EA9882361F4849CF00146
:103CE000859CF00D949CF00D1124EA5CF94F86A997
:103CF000882331F1EAA0FBA00CA11DA16EA17FA138
:103D000088A599A5A80197010E9494DB5B016C012D
:103D1000849CF001859CF00D949CF00D1124EA5CCC
:103D2000F94F66A177A180A591A5A80197010E94EE
:103D300094DB8B019C01CE01B601A501C1DD1EAA59
:103D4000739480E1781609F47724849CE001859CC3
:103D5000D00D949CD00D1124CA5CD94F872C992486
:103D600087FC90948091060B90E08816990609F0E4
:103D7000B0CF2097E9F0EAA0FBA00CA11DA16EA195
:103D80007FA188A599A5A80197010E9494DB5B01FA
:103D90006C016DEC7CEC8CE49DE3A80197010E9422
:103DA00094DB8B019C01CE01B601A50189DD1EAA21
:103DB000DF91CF911F910F91FF90EF90DF90CF9007
:103DC000BF90AF909F908F907F905F904F9008959D
:103DD000FBDC49DC67CF2F923F924F925F926F924C
:103DE0007F928F929F92AF92BF92CF92DF92EF928B
:103DF000FF920F931F93DF93CF93CDB7DEB7C958D0
:103E0000D0400FB6F894DEBF0FBECDBF5C014B01B2
:103E10003A012901CA57DF4FE882C658D040C95736
:103E2000DF4FF882C758D040C857DF4F0883C858C3
:103E3000D040C757DF4F1883C958D040E496DFAE53
:103E4000CEAEE4978091060B8F5F803109F480E05D
:103E5000282F332727FD30953DA72CA706C00E94A9
:103E60005AA00E94487C0E941E6F8091070B90E030
:103E70004CA55DA58417950791F3D5016D917D91B2
:103E80008D919C912091D9053091DA054091DB0507
:103E90005091DC050E946DDE0E943DDEE2966CAF23
:103EA0007DAF8EAF9FAFE297F40160817181828117
:103EB00093812091DD053091DE054091DF05509121
:103EC000E0050E946DDE0E943DDEAE966CAF7DAFD8
:103ED0008EAF9FAFAE97D3016D917D918D919C91E7
:103EE0002091E1053091E2054091E3055091E40510
:103EF0000E946DDE0E943DDEAA966CAF7DAF8EAF54
:103F00009FAFAA97F2016081718182819381209194
:103F1000E5053091E6054091E7055091E8050E94DE
:103F20006DDE0E943DDEA6966CAF7DAF8EAF9FAF7B
:103F3000A6978091310690913206A0913306B091F8
:103F40003406A6962CAD3DAD4EAD5FADA6972817B5
:103F500039074A075B0709F404C1E091B10DF0E0AD
:103F6000EE0FFF1FEE0FFF1FEF55F04F60817181C5
:103F7000828193812091400230914102409142021E
:103F8000509143020E948DDB88230CF045C0A69619
:103F90004CAD5DAD6EAD7FADA697409331065093AD
:103FA00032066093330670933406E3EEF0E08491BA
:103FB0008F017E010894E11CF11C0CC0898385E50A
:103FC00091E1B70141E050E00E9426D90F5F1F4FF9
:103FD000F8018491882391F7E7E0F1E084918F0163
:103FE0007E010894E11CF11C0CC0898385E591E1F8
:103FF000B70141E050E00E9426D90F5F1F4FF80142
:104000008491882391F78AE0898385E591E1B7015E
:1040100041E050E00E9426D980913106909132060D
:10402000A0913306B0913406A6962CAD3DAD4EADB1
:104030005FADA697281B390B4A0B5B0BCA01B90170
:1040400057FF07C090958095709561957F4F8F4F72
:104050009F4F0E942FDC5B016C0160917C0270918C
:104060007D0280917E0290917F022091BD0D309162
:10407000BE0D4091BF0D5091C00D0E94B3DA7B017F
:104080008C016091800270918102809182029091F6
:1040900083022091C10D3091C20D4091C30D50910A
:1040A000C40D0E94B3DA9B01AC01C801B7010E94A4
:1040B000B4DA2091E5053091E6054091E70550918D
:1040C000E8050E946DDE9B01AC01C601B5010E94AE
:1040D0009BDD18160CF045C0A6964CAD5DAD6EADDF
:1040E0007FADA69740933106509332066093330616
:1040F00070933406E3EEF0E084918F017E01089422
:10410000E11CF11C0CC0898385E591E1B70141E018
:1041100050E00E9426D90F5F1F4FF8018491882339
:1041200091F7E9EEF0E084918F017E010894E11CA3
:10413000F11C0CC0898385E591E1B70141E050E0B5
:104140000E9426D90F5F1F4FF8018491882391F7B1
:104150008AE0898385E591E1B70141E050E00E9462
:1041600026D98091060B282F30E0A2963FAF2EAFC4
:10417000A2978DE490E0289FF001299FF00D389FD1
:10418000F00D1124EA5CF94FE45BFF4F1082EC5410
:10419000F0404091250650912606609127067091C7
:1041A0002806A0964CAF5DAF6EAF7FAFA097E296AA
:1041B0008CAD9DADAEADBFADE297841B950BA60B4C
:1041C000B70B6C968CAF9DAFAEAFBFAF6C978083D3
:1041D0009183A283B383B7FF0BC0B095A095909550
:1041E00081959F4FAF4FBF4F80839183A283B3834D
:1041F0002091290630912A0640912B0650912C06D9
:1042000068962CAF3DAF4EAF5FAF6897AE966CAD82
:104210007DAD8EAD9FADAE97621B730B840B950B7E
:1042200064966CAF7DAF8EAF9FAF64978DE490E0E6
:10423000A296AEADBFADA297A89FF001A99FF00DC9
:10424000B89FF00D1124EA5CF94F64962CAD3DAD9A
:104250004EAD5FAD6497248335834683578357FF04
:104260000DC0DA01C901B095A095909581959F4F39
:10427000AF4FBF4F84839583A683B78340912D06AC
:1042800050912E0660912F067091300660964CAFCB
:104290005DAF6EAF7FAF6097AA968CAD9DADAEADB2
:1042A000BFADAA97841B950BA60BB70B2C968CAFB2
:1042B0009DAFAEAFBFAF2C978DE490E0A296AEADB0
:1042C000BFADA297A89FF001A99FF00DB89FF00D78
:1042D0001124EA5CF94F2C962CAD3DAD4EAD5FAD8F
:1042E0002C97208731874287538757FF0DC0DA010B
:1042F000C901B095A095909581959F4FAF4FBF4F45
:1043000080879187A287B38720903106309032064C
:104310004090330650903406A6964CAD5DAD6EAD20
:104320007FADA69742195309640975094EA35FA38F
:1043300068A779A760916E0270916F0228967FAF8F
:104340006EAF28976EA17FA188A599A597FF07C09A
:1043500090958095709561957F4F8F4F9F4F2896D0
:10436000AEADBFAD28979D01442737FD4095542F32
:104370000E943FDF24E630E040E050E00E94A7DFEB
:104380008DE490E0A2966EAD7FADA297689FF0019C
:10439000699FF00D789FF00D1124EA5CF94FDF0161
:1043A0001C96248711963C93119712964C93129762
:1043B00013965C936080718082809380A480B58026
:1043C000C680D780E084F18402851385C901DA01B3
:1043D0008E159F05A007B10714F4D801C7018A15EF
:1043E0009B05AC05BD0514F4D601C5019C01AD01CA
:1043F00086159705A805B90514F4A40193018DE469
:1044000090E0A296AEADBFADA297A89FB001A99FC4
:10441000700DB89F700D11246A5C794FFB01208BE1
:10442000318B428B538B263031054105510510F4F9
:104430000C94022BE85BFF4F8091B20D9091B30D6D
:10444000AA2797FDA095BA2F80839183A283B38377
:10445000DB0190961C92E2962CAD3DAD4EAD5FAD6A
:10446000E297A0968CAD9DADAEADBFADA0972817DD
:1044700039074A075B0724F481E0DB0190968C93AF
:10448000AE962CAD3DAD4EAD5FADAE9768966CADC2
:104490007DAD8EAD9FAD6897261737074807590742
:1044A00094F48DE490E0A296AEADBFADA297A89F24
:1044B000F001A99FF00DB89FF00D1124EA5CF94FAF
:1044C00080A1826080A3AA962CAD3DAD4EAD5FADBC
:1044D000AA9760966CAD7DAD8EAD9FAD60972617A7
:1044E00037074807590794F48DE490E0A296AEADE3
:1044F000BFADA297A89FF001A99FF00DB89FF00D46
:104500001124EA5CF94F80A1846080A3A6962CADAB
:104510003DAD4EAD5FADA69722153305440555055B
:1045200094F48DE490E0A2964EAD5FADA297489FC3
:10453000F001499FF00D589FF00D1124EA5CF94FEE
:1045400080A1886080A38DE490E0A2966EAD7FADDF
:10455000A297689FF001699FF00D789FF00D1124DC
:10456000EA5CF94FE496AEADBFADE4978C9181A3C0
:10457000208131814281538126962CAF3DAF4EAFD1
:104580005FAF2697211531054105510509F0779850
:104590008DE490E0A2964EAD5FADA297489FF001EA
:1045A000499FF00D589FF00D1124EA5CF94F64808B
:1045B000758086809780611471048104910409F0EC
:1045C00076988DE490E0A2966EAD7FADA297689F3D
:1045D000F001699FF00D789FF00D1124EA5CF94F0E
:1045E000A084B184C284D384A114B104C104D104D1
:1045F00009F047988DE490E0A296AEADBFADA297CA
:10460000A89FF001A99FF00DB89FF00D1124EA5C5E
:10461000F94F84859585A685B7850097A105B105D5
:1046200061F043988C988D982090F9053090FA05A8
:104630004090FB055090FC0508C02090110630907A
:1046400012064090130650901406CA57DF4F688137
:10465000C658D040C957DF4F7881C758D040C85797
:10466000DF4F8881C858D040C757DF4F9881C9585D
:10467000D040A20191010E948DDB87FD16C0CA5770
:10468000DF4F8881C658D040C957DF4F9881C7583F
:10469000D040C857DF4FA881C858D040C757DF4F18
:1046A000B881C958D0401C012D016C966CAD7DAD10
:1046B0008EAD9FAD6C970E942FDC2091D905309173
:1046C000DA054091DB055091DC050E9494DBED9604
:1046D0006FAFED97EE967FAFEE97EF968FAFEF97B8
:1046E000C158DF4F9883CF57D040AC01CB01DA01DE
:1046F0008A839B83AC83BD8364966CAD7DAD8EADA8
:104700009FAD64970E942FDC2091DD053091DE057E
:104710004091DF055091E0050E9494DBE9966FAF70
:10472000E997EA967FAFEA97EB968FAFEB97EC9617
:104730009FAFEC97AC01CB01DA018E839F83A887F2
:10474000B9872C966CAD7DAD8EAD9FAD2C970E9438
:104750002FDC2091E1053091E2054091E305509175
:10476000E4050E9494DBE5966FAFE597E6967FAF90
:10477000E697E7968FAFE797E8969FAFE897AC018B
:10478000CB01DA018A879B87AC87BD876EA17FA1A9
:1047900088A599A50E942FDC2091E5053091E605BA
:1047A0004091E7055091E8050E9494DB7B018C0164
:1047B0002896EEADFFAD2897BF01882777FD80953D
:1047C000982F0E942FDC9B01AC01C801B7010E9409
:1047D0006DDE20E030E048EC52E40E9494DB9B0167
:1047E000AC016E877F87888B998B26966CAD7DADEB
:1047F0008EAD9FAD269766307105810591051CF53C
:1048000076E06716710481049104ECF486E0A81642
:10481000B104C104D104BCF48DE490E0A296AEAD25
:10482000BFADA297A89FF001A99FF00DB89FF00D12
:104830001124EA5CF94FDA01C901BF7786A797A76F
:10484000A0ABB1AB57C0ED962FADED97EE963FAD57
:10485000EE97EF964FADEF97C158DF4F5881CF5786
:10486000D040B901CA010E9424DF3B014C01E99606
:104870002FADE997EA963FADEA97EB964FADEB97F0
:10488000EC965FADEC97B901CA010E9424DF5B0191
:104890006C01E5962FADE597E6963FADE697E79676
:1048A0004FADE797E8965FADE897B901CA010E945E
:1048B00024DF7B018C01C401B301A60195010E9494
:1048C000B4DAA80197010E94B4DA0E94DADE2DE47E
:1048D00030E0A2964EAD5FADA297429FF001439F9C
:1048E000F00D529FF00D1124EA5CF94F66A777A7EF
:1048F00080AB91AB8DE490E0A2966EAD7FADA297B8
:10490000689FF001699FF00D789FF00D1124EA5C1B
:10491000F94F86A597A5A0A9B1A922968CAF9DAF06
:10492000AEAFBFAF229760E070E080E89FE32296D1
:104930002CAD3DAD4EAD5FAD22970E9494DB9B0147
:10494000AC01C201B1010E946DDE2B013C018091DE
:10495000060B9091070BA82FB0E05096A91BB10948
:10496000AF70B070BBA7AAA7A230B1050CF44EC0BF
:104970005D01CC24B7FCC094DC2CC601B5010E94BB
:104980002FDC20E030E040E051E40E948DDB882302
:10499000ECF560E074E284E799E4A30192010E94DF
:1049A00094DB0E943DDE7B018C016091C505709116
:1049B000C6058091C7059091C805E616F706080759
:1049C000190720F56E197F09800B910B660F771F71
:1049D000881F991FA60195010E9485DFCA01B901B0
:1049E0000E942DDC0E943DDEE60EF71E081F191FF7
:1049F000C801B7010E942DDC9B01AC0160E074E2AC
:104A000084E799E40E9494DB2B013C018DE490E063
:104A1000A296EEADFFADA297E89F8001E99F100D31
:104A2000F89F100D11240A5C194F22966CAD7DADD4
:104A30008EAD9FAD2297A30192010E946DDED80139
:104A400092966D937D938D939C93959750966D91CF
:104A50007D918D919C9153970E942DDCA301920131
:104A60000E946DDE0E947ADB0E9401DCF80160AFDB
:104A700071AF82AF93AFC058DF4F1882C058D0409B
:104A8000CF57DF4F1882C158D04020E8222E9FE335
:104A9000392E88249924E2E0F0E0EC0FFD1FE80DA8
:104AA000F91DC301B20120813181428153810E94ED
:104AB0006DDEE2E1F0E0EC0FFD1FE80DF91D608313
:104AC0007183828393835B016C01E894D7F8F401CE
:104AD000E753FA4FE080F18002811381C601B501EE
:104AE000A80197010E949BDD1816CCF4C801B701FC
:104AF000A60195010E9494DB6B017C01C058DF4F39
:104B00006881C058D040CF57DF4F7881C158D0401E
:104B1000C101A70196010E948DDB88236CF4C05867
:104B2000DF4F8881C058D040CF57DF4F9881C158A0
:104B3000D040D1016C017D0124E030E0820E931E53
:104B400030E18316910471F0D701C601C058DF4FE0
:104B5000C882C058D040CF57DF4F9883C158D0404B
:104B60001D0199CFC701B60120E030E040E85FE3C6
:104B70000E948DDB88230CF04CC08E010E5E1F4F0F
:104B800082E2A82EB12CAC0EBD1ED8016D917D9194
:104B90008D919C91A70196010E946DDEF8016193B1
:104BA0007193819391938F01EA15FB0571F78DE461
:104BB00090E0A2962EAD3FADA297289F8001299F3D
:104BC000100D389F100D11240A5C194FD8019296D0
:104BD0006D917D918D919C919597A70196010E9471
:104BE0006DDEF80162A373A384A395A360AD71ADDC
:104BF00082AD93AD0E942DDCA70196010E946DDE6F
:104C00000E9401DCD801D8966D937D938D939C937F
:104C1000DB978DE490E0A296EEADFFADA297E89F02
:104C20008001E99F100DF89F100D11240A5C194FA7
:104C3000D80150966D917D918D919C9153970E94D2
:104C40002DDCF80126A537A540A951A90E9494DBC7
:104C50001B012C01F80180819181A281B381009711
:104C6000A105B10549F584819581A681B781009799
:104C7000A105B10509F580859185A285B3850097C9
:104C8000A105B105C9F4C201B1012091010630911D
:104C9000020640910306509104060E946DDE0E94B8
:104CA0007ADB0C5B1F4F0E9401DCD8016D937D9372
:104CB0008D939C93139771C1C201B1012091FD05A1
:104CC0003091FE054091FF05509100060E946DDE77
:104CD0000E947ADB0E9401DC2DE430E0A296EEAD6A
:104CE000FFADA297E29F6001E39FD00CF29FD00C32
:104CF000112426E336E0C20ED31EB4E46B2E712CD1
:104D00006C0C7D1CD3016D937D938D939C931397B5
:104D10008090150690901606A0901706B090180681
:104D20000E942DDC7B018C01F60160817181828102
:104D300093810E942FDC9B01AC01C801B7010E9446
:104D40006DDE7B018C01D60150966D917D918D9128
:104D50009C9153970E942DDC9B01AC01C801B701C7
:104D60000E9494DB7B018C01C501B4010E942DDC03
:104D70009B01AC01C801B7010E949BDD18162CF401
:104D8000F30180829182A282B38280901906909072
:104D90001A06A0901B06B0901C068DE490E0A29627
:104DA0002EAD3FADA297289F6001299FD00C389F60
:104DB000D00C112446E356E0C40ED51EA4E46A2E9E
:104DC000712C6C0C7D1CD3016D917D918D919C910A
:104DD0000E942DDC7B018C01F60164817581868146
:104DE00097810E942FDC9B01AC01C801B7010E9492
:104DF0006DDE7B018C01D60150966D917D918D9178
:104E00009C9153970E942DDC9B01AC01C801B70116
:104E10000E9494DB7B018C01C501B4010E942DDC52
:104E20009B01AC01C801B7010E949BDD18162CF450
:104E3000F30180829182A282B382809021069090B9
:104E40002206A0902306B09024068DE490E0A2965E
:104E50002EAD3FADA297289F6001299FD00C389FAF
:104E6000D00C112446E356E0C40ED51EF4E46F2E98
:104E7000712C6C0C7D1CD3016D917D918D919C9159
:104E80000E942DDC7B018C01F60164857585868589
:104E900097850E942FDC9B01AC01C801B7010E94DD
:104EA0006DDE7B018C01D60150966D917D918D91C7
:104EB0009C9153970E942DDC9B01AC01C801B70166
:104EC0000E9494DB7B018C01C501B4010E942DDCA2
:104ED0009B01AC01C801B7010E949BDD18162CF4A0
:104EE000F30180829182A282B38280901D0690900D
:104EF0001E06A0901F06B09020068DE490E0A296BA
:104F00002EAD3FADA297289F6001299FD00C389FFE
:104F1000D00C112446E356E0C40ED51EE4E46E2EF8
:104F2000712C6C0C7D1CD3016D917D918D919C91A8
:104F30000E942DDC7B018C01F601608571858285E4
:104F400093850E942FDC9B01AC01C801B7010E9430
:104F50006DDE7B018C01D60150966D917D918D9116
:104F60009C9153970E942DDC9B01AC01C801B701B5
:104F70000E9494DB7B018C01C501B4010E942DDCF1
:104F80009B01AC01C801B7010E949BDD18162CF4EF
:104F9000F30180829182A282B3828DE490E0A29696
:104FA0002EAD3FADA297289F6001299FD00C389F5E
:104FB000D00C112446E356E0C40ED51EF601EC5B7E
:104FC000FF4F60817181828193810E942DDC7B0182
:104FD0008C01A20191010E9494DBD601D2966D93BF
:104FE0007D938D939C93D597C801B7012DEB37E343
:104FF00046E051E40E946DDE0E94FCDBF601648F06
:10500000758F868F978F609005067090060680904A
:10501000070690900806C401B30120E030E040E0AC
:105020005FE30E946DDE5B016C012A8D3B8D4C8D30
:105030005D8D2AAF3BAF4CAF5DAF409109065091FB
:105040000A0660910B0670910C064EAB5FAB68AF21
:1050500079AFCB01BA0120E030E040E05FE30E948D
:105060006DDE7B018C016AAD7BAD8CAD9DAD9F7714
:10507000A80197010E949BDD181644F4C601B501F2
:10508000A80197010E948DDB882314F48601750125
:105090006E8D7F8D88A199A16AAB7BAB8CAB9DABEC
:1050A00080910D0690910E06A0910F06B09110060A
:1050B0008EA79FA7A8ABB9ABBC01CD0120E030E023
:1050C00040E05FE30E946DDE1B012C016AA97BA911
:1050D0008CA99DA99F77A20191010E949BDD1816C2
:1050E00044F4C801B701A20191010E948DDB88231D
:1050F00014F4170128018DE490E0A296AEADBFAD87
:10510000A297A89FF001A99FF00DB89FF00D112460
:10511000EA5CF94F22A133A144A155A12AA33BA3E4
:105120004CA35DA3C201B1010E948DDB87FD04C0C9
:105130002AA03BA04CA05DA04AA55BA5423051052A
:105140000CF405C15091080BCE57DF4F5883C2585D
:10515000D0406091090BCD57DF4F6883C358D040D2
:1051600070910A0BCC57DF4F7883C458D0408091A0
:105170000B0BCB57DF4F8883C558D040652FCD57D9
:10518000DF4F7881C358D040CC57DF4F8881C45857
:10519000D040CB57DF4F9881C558D04027E137EB3F
:1051A00041ED58E30E949BDD18160CF0D0C06A89CF
:1051B0007B898C899D8920910C0B30910D0B40913E
:1051C0000E0B50910F0B0E94B3DA9B01AC010E94B1
:1051D0006DDE7B018C016E897F89888D998D209190
:1051E000100B3091110B4091120B5091130B0E9438
:1051F000B3DA9B01AC010E946DDE9B01AC01C801DA
:10520000B7010E94B4DA0E94DADE7B018C01A401AE
:1052100093010E949BDD18165CF00F2EF0E06F2EBC
:10522000F0E07F2EF0E88F2EFFE39F2EF02D08C0D8
:10523000C401B301A80197010E9494DB3B014C011A
:105240006AAD7BAD8CAD9DAD2091140B3091150BEB
:105250004091160B5091170B0E94B3DA7B018C0121
:10526000E89417F9C801B7012EA93FA948AD59AD77
:105270000E949BDD181694F46EA97FA988AD99ADA4
:10528000A80197010E9494DB5B016C01C401B3018A
:10529000A60195010E948DDB882314F4640153015B
:1052A0006AA97BA98CA99DA92091180B3091190B93
:1052B00040911A0B50911B0B0E94B3DA7B018C01B9
:1052C000E89417F9C801B7012EA53FA548A959A927
:1052D0000E949BDD181694F46EA57FA588A999A954
:1052E000A80197010E9494DB7B018C01C601B501E6
:1052F000A80197010E948DDB882314F486017501B3
:105300006AA17BA18CA19DA1A80197010E946DDEDD
:105310007B018C01CE57DF4F6881C258D040CD57FA
:10532000DF4F7881C358D040CC57DF4F8881C458B5
:10533000D040CB57DF4F9881C558D040A801970186
:105340000E948DDB87FD19C0D801C70102C0D201C0
:10535000C101CE57DF4F8883C258D040CD57DF4FB1
:105360009883C358D040CC57DF4FA883C458D0404F
:10537000CB57DF4FB883C558D0408DE490E0A2965C
:10538000AEADBFADA297A89F8001A99F100DB89F99
:10539000100D11240A5C194FCE57DF4F8881C25877
:1053A000D040CD57DF4F9881C358D040CC57DF4F06
:1053B000A881C458D040CB57DF4FB881C558D040E2
:1053C000F80182A793A7A4A7B5A762A973A984A986
:1053D00095A9905820E030E040E050EC0E946DDE4E
:1053E000D8019E962D913D914D915C91D1970E944F
:1053F0006DDE2BE037ED43E25BE30E94B4DA0E94FE
:10540000DADEF62EE72ED82EC92ECE57DF4F688172
:10541000C258D040CD57DF4F7881C358D040CC57C9
:10542000DF4F8881C458D040CB57DF4F9881C55893
:10543000D0402F2D3E2D4D2D5C2D0E948DDB87FD04
:1054400014C0CE57DF4FF882C258D040CD57DF4F3F
:10545000E882C358D040CC57DF4FD882C458D040E0
:10546000CB57DF4FC882C558D0408DE490E0A2965C
:10547000EEADFFADA297E89F8001E99F100DF89F68
:10548000100D11240A5C194FCE57DF4F8881C25886
:10549000D040CD57DF4F9881C358D040CC57DF4F15
:1054A000A881C458D040CB57DF4FB881C558D040F1
:1054B000F80186A397A3A0A7B1A762A173A184A1B5
:1054C00095A12F2D3E2D4D2D5C2D0E948DDB1816A4
:1054D0002CF081E0D801D7968C9302C0F80117AA6E
:1054E0008DE490E0A2962EAD3FADA297289FF001EB
:1054F000299FF00D389FF00D1124EA5CF94F81E0EF
:1055000086ABACE0BBE0FE01729680E101900D92AB
:105510008150E1F78DE490E0A2964EAD5FADA29789
:10552000489F6001499FD00C589FD00C112466E31E
:1055300076E0C60ED71ED6019296ED90FD900D91A5
:105540001C919597E092080BF092090B00930A0BBF
:1055500010930B0B96966D917D918D919C919997DF
:10556000A80197010E9494DB4B015C01C201B101CB
:10557000A80197010E9494DB8B019C01C601B50133
:10558000A4010E94601CBCA5B093060BA6962CAD8E
:105590003DAD4EAD5FADA6972093310630933206F8
:1055A0004093330650933406AA964CAD5DAD6EAD74
:1055B0007FADAA9740932D0650932E0660932F0639
:1055C00070933006AE966CAD7DAD8EAD9FADAE974F
:1055D0006093290670932A0680932B0690932C06DD
:1055E000E2968CAD9DADAEADBFADE2978093250642
:1055F00090932606A0932706B09328060E94E81EE3
:105600000E947CA7C757DF4F0FB6F894DEBF0FBECE
:10561000CDBFCF91DF911F910F91FF90EF90DF9061
:10562000CF90BF90AF909F908F907F906F905F9042
:105630004F903F902F90089510922C0B089560E0AA
:10564000309B61E0319B62600FB6F89420914C1161
:1056500030914D1140914E1150914F110FBE8091DC
:10566000430B9091440BA091450BB091460B8217D0
:105670009307A407B50710F4329B64606093410B55
:105680009091410B91708091410B81FD92608091CE
:10569000470B981729F19130B1F0913028F09230F2
:1056A00041F09330E9F40AC0813079F08230C1F4DE
:1056B00012C0882351F0833099F40DC0823029F054
:1056C000813071F408C0833021F48091480B8F5FE2
:1056D00005C0882329F48091480B81508093480BA2
:1056E0009093470B08958091410B90E09695879594
:1056F0009695879581700895FC012081822F90E016
:105700006AE070E00E9472DFCB016AE070E00E9404
:1057100072DF805D8093700B822F90E06AE070E012
:105720000E9472DF805D8093710B1092720B80E794
:105730009BE00895FC01608171818281938120E06A
:1057400030E040E251E40E946DDE0E94FCDB9B01F0
:1057500077FF02C08DE201C08BE28093700B37FFB0
:1057600003C0309521953F4FC90168EE73E00E9458
:1057700072DFCB016AE070E00E9472DF805D80938F
:10578000710BC90164E670E00E9472DFCB016AE030
:1057900070E00E9472DF805D8093720BC9016AE045
:1057A00070E00E9472DFCB016AE070E00E9472DF5D
:1057B000805D8093730B8EE28093740BC9016AE065
:1057C00070E00E9472DF805D8093750B1092760B03
:1057D00080E79BE00895EF92FF920F931F93FC01E7
:1057E000608171818281938120E030E048EC52E455
:1057F0000E946DDE0E94FCDB7B018C0197FD12C0D4
:1058000020E137E240E050E00E94A7DFCA01B90181
:105810002AE030E040E050E00E94A7DF605D609346
:10582000700B03C08DE28093700B17FF08C01095BA
:105830000095F094E094E11CF11C011D111DC801BC
:10584000B70128EE33E040E050E00E94A7DFCA0134
:10585000B9012AE030E040E050E00E94A7DF605D3F
:105860006093710BC801B70124E630E040E050E0DE
:105870000E94A7DFCA01B9012AE030E040E050E011
:105880000E94A7DF605D6093720B8EE28093730BC2
:10589000C801B7012AE030E040E050E00E94A7DFF5
:1058A000CA01B9012AE030E040E050E00E94A7DFE1
:1058B000605D6093740BC801B7012AE030E040E0FE
:1058C00050E00E94A7DF605D6093750B1092760B2D
:1058D00080E79BE01F910F91FF90EF900895FC01EE
:1058E00080819181843691055CF064E670E00E94CD
:1058F00072DFCB016AE070E00E9472DF805D01C060
:1059000080E28093700B808191818A3091055CF0F8
:105910006AE070E00E9472DFCB016AE070E00E94F2
:1059200072DF805D01C080E28093710B8081918184
:105930006AE070E00E9472DF805D8093720B1092CB
:10594000730B80E79BE00895DF93CF9300D0CDB732
:10595000DEB7FC0160817181828193810E94FCDB52
:105960007A836983CE010196BADF0F900F90CF91B1
:10597000DF910895FC01808191818436910534F195
:1059800064E670E00E9472DFCB016AE070E00E9482
:1059900072DF805D8093700B808191816AE070E09E
:1059A0000E9472DFCB016AE070E00E9472DF805DCE
:1059B0008093710B808191816AE070E00E9472DFB8
:1059C000805D8093720B1092730B24C08A30910516
:1059D000C4F06AE070E00E9472DFCB016AE070E020
:1059E0000E9472DF805D8093700B808191816AE0FC
:1059F00070E00E9472DF805D8093710B1092720BD9
:105A000009C06AE070E00E9472DF805D8093700BD5
:105A10001092710B80E79BE00895EF92FF920F9335
:105A20001F93FC01E080F18002811381C801B7015E
:105A300020E030E040E050E00E949BDD18161CF4AE
:105A4000C801B70103C0C801B70190580E94FCDB30
:105A50007B018C0180E1E81687E2F80680E0080708
:105A600080E01807A4F0C801B70120E137E240E068
:105A700050E00E94A7DFCA01B9012AE030E040E00F
:105A800050E00E94A7DF605D6093700B0CC080E265
:105A90008093700B98EEE91693E0F90690E0090701
:105AA00090E01907A4F0C801B70128EE33E040E008
:105AB00050E00E94A7DFCA01B9012AE030E040E0CF
:105AC00050E00E94A7DF605D6093710B08C0809377
:105AD000710B94E6E916F10401051105A4F0C80163
:105AE000B70124E630E040E050E00E94A7DFCA01A1
:105AF000B9012AE030E040E050E00E94A7DF605D9D
:105B00006093720B08C08093720B9AE0E916F1045F
:105B100001051105A4F0C801B7012AE030E040E01A
:105B200050E00E94A7DFCA01B9012AE030E040E05E
:105B300050E00E94A7DF605D6093730B02C080930A
:105B4000730BC801B7012AE030E040E050E00E944A
:105B5000A7DF605D6093740B1092750B80E79BE08C
:105B60001F910F91FF90EF900895EF92FF920F9386
:105B70001F93FC01608171818281938120E030E07C
:105B800040E251E40E946DDE0E94FCDB97FF02C000
:105B90002DE201C02BE22093700B7B018C0197FF5B
:105BA00008C010950095F094E094E11CF11C011DD3
:105BB000111DC801B70120E137E240E050E00E942A
:105BC000A7DFCA01B9012AE030E040E050E00E94BE
:105BD000A7DF605D6093710BC801B70128EE33E069
:105BE00040E050E00E94A7DFCA01B9012AE030E09E
:105BF00040E050E00E94A7DF605D6093720BC80137
:105C0000B70124E630E040E050E00E94A7DFCA017F
:105C1000B9012AE030E040E050E00E94A7DF605D7B
:105C20006093730BC801B7012AE030E040E050E018
:105C30000E94A7DFCA01B9012AE030E040E050E04D
:105C40000E94A7DF605D6093740B8EE28093750BFA
:105C5000C801B7012AE030E040E050E00E94A7DF31
:105C6000605D6093760B1092770B80E79BE01F914D
:105C70000F91FF90EF900895EF92FF920F931F9373
:105C8000FC01608171818281938120E030E048ECE9
:105C900052E40E946DDE0E94FCDB97FF02C02DE201
:105CA00001C02BE22093700B7B018C0197FF08C091
:105CB00010950095F094E094E11CF11C011D111D5C
:105CC000C801B70120E137E240E050E00E94A7DFC1
:105CD000CA01B9012AE030E040E050E00E94A7DFAD
:105CE000605D6093710BC801B70128EE33E040E0BE
:105CF00050E00E94A7DFCA01B9012AE030E040E08D
:105D000050E00E94A7DF605D6093720BC801B7018D
:105D100024E630E040E050E00E94A7DFCA01B9016C
:105D20002AE030E040E050E00E94A7DF605D609331
:105D3000730B8EE28093740BC801B7012AE030E048
:105D400040E050E00E94A7DFCA01B9012AE030E03C
:105D500040E050E00E94A7DF605D6093750BC801D2
:105D6000B7012AE030E040E050E00E94A7DF605D2C
:105D70006093760B1092770B80E79BE01F910F9159
:105D8000FF90EF9008950F931F93CF93DF93382FD9
:105D9000EB01142F022F8DE29BE060E0432F0E9465
:105DA00077D1E0912D0BF0912E0B0190F081E02D39
:105DB0008DE29BE0612F099511E1FE01649166235C
:105DC000B9F01123A9F0E0912D0BF0912E0B019069
:105DD000F081E02D8DE29BE0099521961150EDCFE9
:105DE0000190F081E02D8DE29BE060E20995115079
:105DF000E0912D0BF0912E0B112391F70190F08182
:105E0000E02D8DE29BE0602F0995E0912D0BF09144
:105E10002E0B0190F081E02D8DE29BE060E2099570
:105E2000DF91CF911F910F910895BF92CF92DF9292
:105E3000EF92FF920F931F938091490B90914A0B21
:105E4000A0914B0BB0914C0B81509048A040B040BA
:105E500040F01092490B10924A0B10924B0B10928B
:105E60004C0B6091490B70914A0B80914B0B9091B8
:105E70004C0B25E030E040E050E00E9485DF7901E6
:105E80008A018091420B90E0A0E0B0E0E816F906AC
:105E90000A071B0710F42093420B0091420B10E0FD
:105EA00033E1C32ED12CE12CF12CBB24B39400237D
:105EB00009F049C080915B028823B9F08091490BB9
:105EC00090914A0BA0914B0BB0914C0B0597A105FB
:105ED000B10528F4812F6AE375E043E004C0812F07
:105EE0006AE375E040E223E04EDF8091410B82FFE0
:105EF00043C18091490B90914A0BA0914B0BB091FB
:105F00004C0B0597A105B10508F036C182E08093DE
:105F10005B020FB6F89480914C1190914D11A091B5
:105F20004E11B0914F110FBE8C509E4FAF4FBF4FCF
:105F30008093430B9093440BA093450BB093460B77
:105F40008DE191E70CC1013009F057C080915B02EF
:105F50008823F1F06091490B70914A0B80914B0BB3
:105F600090914C0B25E030E040E050E00E9485DF4E
:105F7000213031054105510529F4812F60E375E099
:105F80004EE304C0812F60E375E040E22EE7FBDEC4
:105F90008091410B82FFF0C06091490B70914A0BD8
:105FA00080914B0B90914C0B25E030E040E050E0AD
:105FB0000E9485DF213031054105510509F0DCC023
:105FC00082E080935B020FB6F89480914C1190911F
:105FD0004D11A0914E11B0914F110FBE8C509E4F9C
:105FE000AF4FBF4F8093430B9093440BA093450B4F
:105FF000B093460B8AE793E3B2C0023009F057C072
:1060000080915B028823F1F06091490B70914A0BFB
:1060100080914B0B90914C0B25E030E040E050E03C
:106020000E9485DF223031054105510529F4812F79
:1060300067E275E04EE304C0812F67E275E040E25D
:106040002EE7A1DE8091410B82FF96C06091490B43
:1060500070914A0B80914B0B90914C0B25E030E0F6
:1060600040E050E00E9485DF2230310541055105B6
:1060700009F082C082E080935B020FB6F8948091B1
:106080004C1190914D11A0914E11B0914F110FBE36
:106090008C509E4FAF4FBF4F8093430B9093440B58
:1060A000A093450BB093460B8DE693E358C00330A5
:1060B00009F062C080915B028823F1F06091490B86
:1060C00070914A0B80914B0B90914C0B25E030E086
:1060D00040E050E00E9485DF233031054105510545
:1060E00029F4812F6CE175E04EE304C0812F6CE14F
:1060F00075E040E22EE747DE8091410B82FF3CC015
:106100006091490B70914A0B80914B0B90914C0B15
:1061100025E030E040E050E00E9485DF233031058B
:106120004105510549F582E080935B020FB6F89472
:1061300080914C1190914D11A0914E11B0914F1141
:106140000FBE8C509E4FAF4FBF4F8093430B909329
:10615000440BA093450BB093460B80E693E39093DA
:106160005A02809359021092490B10924A0B1092D6
:106170004B0B10924C0B38C08091490B90914A0BFD
:10618000A0914B0BB0914C0B4497A105B10540F089
:10619000C092490BD0924A0BE0924B0BF0924C0B01
:1061A0006091490B70914A0B80914B0B90914C0B75
:1061B00025E030E040E050E00E9485DF422F8091F2
:1061C000420B90E0039630E08217930744F443506B
:1061D0004093420BB0925B02042F01501FEF1F5FF0
:1061E000143010F40F5F63CE1F910F91FF90EF906A
:1061F000DF90CF90BF900895DF92EF92FF920F93C0
:106200001F938091490B90914A0BA0914B0BB09139
:106210004C0B81509048A040B04040F01092490B88
:1062200010924A0B10924B0B10924C0B6091490B41
:1062300070914A0B80914B0B90914C0B25E030E014
:1062400040E050E00E9485DF79018A018091420B95
:1062500090E0A0E0B0E0E816F9060A071B0710F48A
:106260002093420BF090420B00E045E0E42EDD2449
:10627000D394FF2009F049C080915B028823B9F0D4
:106280008091490B90914A0BA0914B0BB0914C0B14
:106290000597A105B10528F4802F60E675E043E07D
:1062A00004C0802F60E675E040E223E06CDD809161
:1062B000410B82FFDFC08091490B90914A0BA09166
:1062C0004B0BB0914C0B0597A105B10508F0D2C05E
:1062D00082E080935B020FB6F89480914C1190910C
:1062E0004D11A0914E11B0914F110FBE8C509E4F89
:1062F000AF4FBF4F8093430B9093440BA093450B3C
:10630000B093460B85E19FE27AC181E0F81609F06F
:1063100057C080915B028823F1F06091490B709126
:106320004A0B80914B0B90914C0B25E030E040E004
:1063300050E00E9485DF213031054105510529F4E7
:10634000802F69E575E04EE304C0802F69E575E0B4
:1063500040E22EE718DD8091410B82FF8BC06091F7
:10636000490B70914A0B80914B0B90914C0B25E09F
:1063700030E040E050E00E9485DF213031054105EA
:10638000510509F077C082E080935B020FB6F89464
:1063900080914C1190914D11A0914E11B0914F11DF
:1063A0000FBE8C509E4FAF4FBF4F8093430B9093C7
:1063B000440BA093450BB093460B84EE9DE61FC1A2
:1063C00022E0F21609F056C080915B028823F1F0BA
:1063D0006091490B70914A0B80914B0B90914C0B43
:1063E00025E030E040E050E00E9485DF22303105BA
:1063F0004105510529F4802F62E575E04EE304C0A4
:10640000802F62E575E040E22EE7BDDC8091410B14
:1064100082FF30C06091490B70914A0B80914B0B09
:1064200090914C0B25E030E040E050E00E9485DF89
:106430002230310541055105E9F482E080935B0289
:106440000FB6F89480914C1190914D11A0914E117E
:10645000B0914F110FBE8C509E4FAF4FBF4F8093E6
:10646000430B9093440BA093450BB093460B86E1EE
:106470009DE6C5C060916C0B70916D0B80916E0BA9
:1064800090916F0B20E030E040E251E40E948DDB00
:1064900088230CF0C1C083E0F81609F057C0809142
:1064A0005B028823F1F06091490B70914A0B809157
:1064B0004B0B90914C0B25E030E040E050E00E9407
:1064C00085DF233031054105510529F4802F6BE428
:1064D00075E04EE304C0802F6BE475E040E22EE7E8
:1064E00052DC8091410B82FF99C06091490B709101
:1064F0004A0B80914B0B90914C0B25E030E040E033
:1065000050E00E9485DF233031054105510509F037
:1065100085C082E080935B020FB6F89480914C11A5
:1065200090914D11A0914E11B0914F110FBE8C5012
:106530009E4FAF4FBF4F8093430B9093440BA0935C
:10654000450BB093460B88E49CE659C024E0F21654
:1065500009F064C080915B028823F1F06091490BDF
:1065600070914A0B80914B0B90914C0B25E030E0E1
:1065700040E050E00E9485DF24303105410551059F
:1065800029F4802F62E475E04EE304C0802F62E4BA
:1065900075E040E22EE7F7DB8091410B82FF3EC0C1
:1065A0006091490B70914A0B80914B0B90914C0B71
:1065B00025E030E040E050E00E9485DF24303105E6
:1065C0004105510559F582E080935B020FB6F894BE
:1065D00080914C1190914D11A0914E11B0914F119D
:1065E0000FBE8C509E4FAF4FBF4F8093430B909385
:1065F000440BA093450BB093460B8CEA9BE690931B
:106600005A02809359021092490B10924A0B109231
:106610004B0B10924C0B4EC013E001C015E0609183
:10662000490B70914A0B80914B0B90914C0B25E0DC
:1066300030E040E050E00E9485DF812F90E0A0E054
:10664000B0E0281739074A075B0780F01E9DC0019C
:1066500011240197AA2797FDA095BA2F8093490B83
:1066600090934A0BA0934B0BB0934C0B6091490B4A
:1066700070914A0B80914B0B90914C0B25E030E0D0
:1066800040E050E00E9485DF422F8091420B90E075
:10669000039630E08217930744F443504093420B33
:1066A000D0925B02F42EFA940FEF0F5F043010F4D7
:1066B000F394DFCD1F910F91FF90EF90DF9008953D
:1066C0008DEC9CECACECBDE380936C0B90936D0B6C
:1066D000A0936E0BB0936F0B8FCD80E090E0A0E89D
:1066E000BFE380936C0B90936D0BA0936E0BB093F4
:1066F0006F0B82CD80E090E0A0E2B1E480936C0B60
:1067000090936D0BA0936E0BB0936F0B75CDCF93E1
:10671000DF93EC0104C08DE29BE00E9441D1FE01B9
:10672000219664916623B9F7DF91CF910895CF93B5
:10673000DF93DB010D900020E9F71197A61BB70B43
:10674000EC01E881F9810280F381E02DAD0109952A
:10675000DF91CF910895AF92BF92CF92DF92EF92E7
:10676000FF920F931F93DF93CF93CDB7DEB7289798
:106770000FB6F894DEBF0FBECDBF6091A10F709130
:10678000A20F8091A30F9091A40F20E030E040E091
:106790005FE30E94B4DA0E94FCDB7C836B83609130
:1067A000930F7091940F882777FD8095982F0E9402
:1067B0002FDC20E030E040E05FE30E94B4DA0E948A
:1067C000FCDB7E836D838DE29BE060E040E00E9415
:1067D00077D1E0912D0BF0912E0B0190F081E02DFF
:1067E0008DE29BE062E00995CE01039678D8BC016A
:1067F0008DE29BE09CDFE0912D0BF0912E0B019040
:10680000F081E02D8DE29BE06FE20995CE010596C7
:10681000B1D8BC018DE29BE08ADF84E391E077DFB1
:106820008D819E810A975CF4E0912D0BF0912E0BE7
:106830000190F081E02D8DE29BE060E209958DE210
:106840009BE06AE040E00E9477D16091A50F7091D3
:10685000A60F8091A70F9091A80F20E030E040E0B4
:106860005FE30E94B4DA0E94FCDB7C836B8360915F
:10687000950F7091960F882777FD8095982F0E942D
:106880002FDC20E030E040E05FE30E94B4DA0E94B9
:10689000FCDB7E836D83E0912D0BF0912E0B01903C
:1068A000F081E02D8DE29BE062E00995CE01039638
:1068B00016D8BC018DE29BE03ADFE0912D0BF09100
:1068C0002E0B0190F081E02D8DE29BE06FE20995A7
:1068D000CE0105964FD8BC018DE29BE028DF81E315
:1068E00091E015DF8D819E810A975CF4E0912D0B7C
:1068F000F0912E0B0190F081E02D8DE29BE060E2A3
:1069000009956091AF0F7091B00F8091B10F909188
:10691000B20F20E030E040E05FE30E94B4DA0E9472
:10692000FCDB7C836B836091990F70919A0F8827B1
:1069300077FD8095982F0E942FDC20E030E040E02A
:106940005FE30E94B4DA0E94FCDB7E836D838DE2FC
:106950009BE060E041E00E9477D1E0912D0BF09147
:106960002E0B0190F081E02D8DE29BE060E0099517
:10697000CE0103960E946F2CBC018DE29BE0D7DE16
:10698000E0912D0BF0912E0B0190F081E02D8DE226
:106990009BE06FE20995CE0105960E94BA2CBC01DE
:1069A0008DE29BE0C4DE8EE291E0B1DE8D819E81BE
:1069B0000A975CF4E0912D0BF0912E0B0190F08181
:1069C000E02D8DE29BE060E209958DE29BE06CE0BA
:1069D00041E00E9477D1E0912D0BF0912E0B0190B8
:1069E000F081E02D8DE29BE06AE5099589E79DE065
:1069F0000E94EB2BBC018DE29BE099DE8DE29BE0D7
:106A000060E042E00E9477D1E0912D0BF0912E0BD7
:106A10000190F081E02D8DE29BE066E009958CE627
:106A200092E00E946F2CBC018DE29BE080DEE09141
:106A30002D0BF0912E0B0190F081E02D8DE29BE06B
:106A400065E209958DE29BE067E042E00E9477D124
:106A50008BE291E05CDE80917E0B882391F1809146
:106A6000400D882311F16091580D7091590D80915E
:106A70005A0D90915B0D6115710581059105A9F085
:106A80006D597F4F8F4F9F4F24E630E040E050E03C
:106A90000E9485DF6091600D7091610D8091620DA3
:106AA0009091630D0E9485DF01C020E02F8318863E
:106AB000CE0107960E946F2CBC018DE29BE037DE71
:106AC00003C087E291E023DEE0912D0BF0912E0BC5
:106AD0000190F081E02D8DE29BE065E209958DE269
:106AE0009BE06EE042E00E9477D1E0912D0BF091A7
:106AF0002E0B0190F081E02D8DE29BE067E009957F
:106B0000A090B40DB090B50DC090B60DD090B70D5B
:106B1000A114B104C104D10409F445C00FB6F8941E
:106B200060914C1170914D1180914E1190914F11C7
:106B30000FBE20E63AEE40E050E00E9485DF79018A
:106B40008A01C601B50120E63AEE40E050E00E941D
:106B500085DFE21AF30AC7016CE370E00E945EDF92
:106B60006983CE0101960E947C2BBC018DE29BE0E3
:106B7000DEDDE0912D0BF0912E0B0190F081E02DE8
:106B80008DE29BE06AE30995C7016CE370E00E9427
:106B90005EDF8A83CE0102960E947C2BBC018DE2CF
:106BA0009BE0C5DD03C081E291E0B1DD8DE29BE0B9
:106BB00060E043E00E9477D18DE29BE064E472E004
:106BC000B6DD28960FB6F894DEBF0FBECDBFCF91CD
:106BD000DF911F910F91FF90EF90DF90CF90BF90CA
:106BE000AF9008958091510B882321F081508093BC
:106BF000510B03C081E080935B0280915B0288238C
:106C000021F0A9DD8AE08093510B8091410B82FF36
:106C100028C08EE494E590935A0280935902109212
:106C2000490B10924A0B10924B0B10924C0B82E0C6
:106C300080935B020FB6F89480914C1190914D11A6
:106C4000A0914E11B0914F110FBE8C509E4FAF4F7F
:106C5000BF4F8093430B9093440BA093450BB0938D
:106C6000460B20916C0230916D022436310554F4AC
:106C70008091490B90914A0B280F391F2536310519
:106C80006CF41AC025363105BCF08091490B909107
:106C90004A0B280F391F2436310574F41092490B22
:106CA00010924A0B10924B0B10924C0B84E690E022
:106CB00090936D0280936C0220916C0230916D0272
:106CC0002436310589F48091490B90914A0B8B3021
:106CD00091051CF0865A9F4F0DC02FEF863F9207FB
:106CE000ACF482599F4F06C08091490B90914A0B9A
:106CF000820F931F90936D0280936C021092490B48
:106D000010924A0B10924B0B10924C0B80916C021C
:106D100090916D020A9734F48AE090E090936D02AE
:106D200080936C0280916C0290916D02885E93401A
:106D300034F087EE93E090936D0280936C02089597
:106D4000EF92FF920F931F93CF93DF93582FEB0196
:106D5000142FF22EE32EE22FF32FDF010D900020EF
:106D6000E9F7022F0A1B0E5E8DE29BE060E0452FE3
:106D70000E9477D1E0912D0BF0912E0B0190F081C4
:106D8000E02D8DE29BE0612F0995FE016491662361
:106D900079F0002369F0E0912D0BF0912E0B01901A
:106DA000F081E02D8DE29BE0099521960150EDCF19
:106DB000E0912D0BF0912E0B0190F081E02D8DE2F2
:106DC0009BE06AE309950CC0E0912D0BF0912E0B2E
:106DD0000190F081E02D8DE29BE060E20995015089
:106DE000002391F78DE29BE06F2D7E2DA0DCDF91DB
:106DF000CF911F910F91FF90EF9008952F923F92A6
:106E00004F925F926F927F928F929F92AF92BF92BA
:106E1000CF92DF92EF92FF920F931F93DF93CF9366
:106E2000CDB7DEB7A0970FB6F894DEBF0FBECDBFCB
:106E30008091490B90914A0BA0914B0BB0914C0B58
:106E400081509048A040B04040F01092490B109201
:106E50004A0B10924B0B10924C0B6091490B7091A6
:106E60004A0B80914B0B90914C0B25E030E040E0B9
:106E700050E00E9485DF79018A018091420B90E009
:106E8000A0E0B0E0E816F9060A071B0710F420930B
:106E9000420B0091420B10E0BDE1EB2EF12CEC0E09
:106EA000FD1EA9E1CA2ED12CCC0EDD1EF5E1AF2EC0
:106EB000B12CAC0EBD1EE1E18E2E912C8C0E9D1ED0
:106EC0007DE0672E712C6C0E7D1E69E0462E512CE4
:106ED0004C0E5D1E55E0252E312C2C0E3D1E002340
:106EE00009F05AC080915B028823C1F08091490B60
:106EF00090914A0BA0914B0BB0914C0B0597A105BB
:106F0000B10528F4812F62E573E043E004C0812FCE
:106F100062E573E040E223E00E94C32E8091410BC2
:106F200082FD02C00C94A0448091490B90914A0BC1
:106F3000A0914B0BB0914C0B0597A105B10510F03A
:106F40000C94A04482E080935B020FB6F894809189
:106F50004C1190914D11A0914E11B0914F110FBE57
:106F60008C509E4FAF4FBF4F8093430B9093440B79
:106F7000A093450BB093460B8DEC9EE590935A027F
:106F8000809359021092490B10924A0B10924B0BAE
:106F900010924C0B0C94DF44013009F0A4C0809196
:106FA0005B02882339F16091490B70914A0B809103
:106FB0004B0B90914C0B25E030E040E050E00E94FC
:106FC00085DF213031054105510551F48DEF95E004
:106FD0000E940D2D9C01812F6CE473E04EE309C0EB
:106FE0008DEF95E00E940D2D9C01812F6CE473E0E4
:106FF00040E2A6DE8091410B82FD02C00C94A044C9
:107000006091490B70914A0B80914B0B90914C0B06
:1070100025E030E040E050E00E9485DF213031057E
:107020004105510511F00C94A0440FB6F8948091DD
:107030004C1190914D11A0914E11B0914F110FBE76
:107040008C509E4FAF4FBF4F8093430B9093440B98
:10705000A093450BB093460B8091590290915A0230
:107060009093530B8093520B8091490B90914A0B54
:107070009093550B8093540B82E080935B028CE5D8
:107080009DE490935A028093590286E493E0909392
:10709000570B8093560B8DEF95E09093590B80938F
:1070A000580B85E090E0A0E0B0E080935A0B9093FD
:1070B0005B0BA0935C0BB0935D0B8EED93E0A0E0B7
:1070C000B0E080935E0B90935F0BA093600BB09346
:1070D000610B6091FD057091FE058091FF05909117
:1070E00000060C94F741023009F0A4C080915B02C5
:1070F000882339F16091490B70914A0B80914B0BB9
:1071000090914C0B25E030E040E050E00E9485DF9C
:10711000223031054105510551F485E096E00E9489
:10712000A42C9C01812F6DE373E04EE309C085E040
:1071300096E00E94A42C9C01812F6DE373E040E255
:10714000FFDD8091410B82FD02C00C94A044609150
:10715000490B70914A0B80914B0B90914C0B25E0A1
:1071600030E040E050E00E9485DF223031054105EB
:10717000510511F00C94A0440FB6F89480914C1175
:1071800090914D11A0914E11B0914F110FBE8C50A6
:107190009E4FAF4FBF4F8093430B9093440BA093F0
:1071A000450BB093460B8091590290915A029093EF
:1071B000530B8093520B8091490B90914A0B909303
:1071C000550B8093540B82E080935B0282ED9EE42A
:1071D00090935A028093590284E393E09093570B63
:1071E0008093560B85E096E09093590B8093580B53
:1071F00081E090E0A0E0B0E080935A0B90935B0BAD
:10720000A0935C0BB0935D0B8EED93E0A0E0B0E03B
:1072100080935E0B90935F0BA093600BB093610B18
:107220006091050670910606809107069091080608
:107230000C949544033009F0A4C080915B0288232C
:1072400039F16091490B70914A0B80914B0B9091F1
:107250004C0B25E030E040E050E00E9485DF233019
:1072600031054105510551F489E096E00E943C2E1C
:107270009C01812F6CE273E04EE309C089E096E047
:107280000E943C2E9C01812F6CE273E040E258DDAD
:107290008091410B82FD02C00C94A0446091490B87
:1072A00070914A0B80914B0B90914C0B25E030E094
:1072B00040E050E00E9485DF233031054105510553
:1072C00011F00C94A0440FB6F89480914C11909159
:1072D0004D11A0914E11B0914F110FBE8C509E4F89
:1072E000AF4FBF4F8093430B9093440BA093450B3C
:1072F000B093460B8091590290915A029093530B90
:107300008093520B8091490B90914A0B9093550BAF
:107310008093540B82E080935B0286EE9BE4909313
:107320005A028093590284E293E09093570B809322
:10733000560B89E096E09093590B8093580B8AE0A6
:1073400090E0A0E0B0E080935A0B90935B0BA09389
:107350005C0BB0935D0B88EB92E8A1E0B0E080930A
:107360005E0B90935F0BA093600BB093610B6091E9
:10737000090670910A0680910B0690910C060C94F8
:107380004343043009F0A4C080915B02882339F1A3
:107390006091490B70914A0B80914B0B90914C0B73
:1073A00025E030E040E050E00E9485DF24303105E8
:1073B0004105510551F48DE096E00E94A42C9C01FA
:1073C000812F6CE173E04EE309C08DE096E00E94EE
:1073D000A42C9C01812F6CE173E040E2B1DC809130
:1073E000410B82FD02C00C94A0446091490B709146
:1073F0004A0B80914B0B90914C0B25E030E040E024
:1074000050E00E9485DF243031054105510511F01F
:107410000C94A0440FB6F89480914C1190914D11AA
:10742000A0914E11B0914F110FBE8C509E4FAF4F97
:10743000BF4F8093430B9093440BA093450BB093A5
:10744000460B8091590290915A029093530B80936E
:10745000520B8091490B90914A0B9093550B80935E
:10746000540B82E080935B0282ED9EE490935A027B
:107470008093590284E193E09093570B8093560BCD
:107480008DE096E09093590B8093580B81E090E04B
:10749000A0E0B0E080935A0B90935B0BA0935C0B41
:1074A000B0935D0B8EED93E0A0E0B0E080935E0BB7
:1074B00090935F0BA093600BB093610B60910D06EE
:1074C00070910E0680910F06909110060C949544D1
:1074D000053009F0A4C080915B02882339F16091E6
:1074E000490B70914A0B80914B0B90914C0B25E00E
:1074F00030E040E050E00E9485DF25303105410555
:10750000510551F489EC95E00E94A42C9C01812F37
:107510006DE073E04EE309C089EC95E00E94A42C75
:107520009C01812F6DE073E040E20ADC8091410B09
:1075300082FD02C00C94A0446091490B70914A0BEB
:1075400080914B0B90914C0B25E030E040E050E0F7
:107550000E9485DF253031054105510511F00C945D
:10756000A0440FB6F89480914C1190914D11A091C8
:107570004E11B0914F110FBE8C509E4FAF4FBF4F69
:107580008093430B9093440BA093450BB093460B11
:107590008091590290915A029093530B8093520B11
:1075A0008091490B90914A0B9093550B8093540B0B
:1075B00082E080935B0282ED9EE490935A02809376
:1075C000590286E093E09093570B8093560B89EC19
:1075D00095E09093590B8093580B81E090E0A0E0E8
:1075E000B0E080935A0B90935B0BA0935C0BB0932D
:1075F0005D0B87EE93E0A0E0B0E080935E0B90938C
:107600005F0BA093600BB093610B6091C905709103
:10761000CA058091CB059091CC050C949544063019
:1076200009F0A4C080915B02882339F16091490B75
:1076300070914A0B80914B0B90914C0B25E030E000
:1076400040E050E00E9485DF2630310541055105BC
:1076500051F48DEC95E00E94A42C9C01812F6FEFDA
:1076600072E04EE309C08DEC95E00E94A42C9C01D1
:10767000812F6FEF72E040E263DB8091410B82FD6E
:1076800002C00C94A0446091490B70914A0B809108
:107690004B0B90914C0B25E030E040E050E00E9415
:1076A00085DF263031054105510511F00C94A044C9
:1076B0000FB6F89480914C1190914D11A0914E11FC
:1076C000B0914F110FBE8C509E4FAF4FBF4F809364
:1076D000430B9093440BA093450BB093460B8091C2
:1076E000590290915A029093530B8093520B8091C0
:1076F000490B90914A0B9093550B8093540B82E069
:1077000080935B0282ED9EE490935A02809359022B
:1077100088EF92E09093570B8093560B8DEC95E099
:107720009093590B8093580B81E090E0A0E0B0E07B
:1077300080935A0B90935B0BA0935C0BB0935D0B03
:1077400087EE93E0A0E0B0E080935E0B90935F0B38
:10775000A093600BB093610B6091CD057091CE0545
:107760008091CF059091D0050C949544073009F095
:10777000A4C080915B02882339F16091490B70911C
:107780004A0B80914B0B90914C0B25E030E040E090
:1077900050E00E9485DF273031054105510551F445
:1077A00081ED95E00E94A42C9C01812F61EF72E095
:1077B0004EE309C081ED95E00E94A42C9C01812F2D
:1077C00061EF72E040E2BCDA8091410B82FD02C0C1
:1077D0000C94A0446091490B70914A0B80914B0B23
:1077E00090914C0B25E030E040E050E00E9485DFB6
:1077F000273031054105510511F00C94A0440FB616
:10780000F89480914C1190914D11A0914E11B0912E
:107810004F110FBE8C509E4FAF4FBF4F8093430B05
:107820009093440BA093450BB093460B8091590263
:1078300090915A029093530B8093520B8091490B75
:1078400090914A0B9093550B8093540B82E0809358
:107850005B0282ED9EE490935A02809359028AEE75
:1078600092E09093570B8093560B81ED95E09093A7
:10787000590B8093580B81E090E0A0E0B0E080933A
:107880005A0B90935B0BA0935C0BB0935D0B87EE50
:1078900093E0A0E0B0E080935E0B90935F0BA09329
:1078A000600BB093610B6091D1057091D20580910E
:1078B000D3059091D4050C949544083009F0A2C0EA
:1078C00080915B02882339F16091490B70914A0BDA
:1078D00080914B0B90914C0B25E030E040E050E064
:1078E0000E9485DF283031054105510551F485EDB1
:1078F00095E00E94A42C9C01812F63EE72E04EE380
:1079000009C085ED95E00E94A42C9C01812F63EEB7
:1079100072E040E215DA8091410B82FD02C00C94C6
:10792000A0446091490B70914A0B80914B0B909150
:107930004C0B25E030E040E050E00E9485DF28302D
:1079400031054105510509F0FBC70FB6F894809148
:107950004C1190914D11A0914E11B0914F110FBE4D
:107960008C509E4FAF4FBF4F8093430B9093440B6F
:10797000A093450BB093460B8091590290915A0207
:107980009093530B8093520B8091490B90914A0B2B
:107990009093550B8093540B82E080935B0282EDB1
:1079A0009EE490935A02809359028CED92E090935A
:1079B000570B8093560B85ED95E09093590B809370
:1079C000580B81E090E0A0E0B0E080935A0B9093D8
:1079D0005B0BA0935C0BB0935D0B87EE93E0A0E094
:1079E000B0E080935E0B90935F0BA093600BB0931D
:1079F000610B6091D5057091D6058091D705909166
:107A0000D80593C7093009F09CC080915B02882398
:107A100039F16091490B70914A0B80914B0B909119
:107A20004C0B25E030E040E050E00E9485DF29303B
:107A300031054105510551F489EF95E00E94A42CD0
:107A40009C01812F67ED72E04EE309C089EF95E05C
:107A50000E94A42C9C01812F67ED72E040E270D956
:107A60008091410B82FF6CC76091490B70914A0B6A
:107A700080914B0B90914C0B25E030E040E050E0C2
:107A80000E9485DF293031054105510509F058C7AD
:107A90000FB6F89480914C1190914D11A0914E1118
:107AA000B0914F110FBE8C509E4FAF4FBF4F809380
:107AB000430B9093440BA093450BB093460B8091DE
:107AC000590290915A029093530B8093520B8091DC
:107AD000490B90914A0B9093550B8093540B82E085
:107AE00080935B0282ED9EE490935A028093590248
:107AF00082ED92E09093570B8093560B89EF95E0BF
:107B00009093590B8093580B10925A0B10925B0B69
:107B100010925C0B10925D0B87EE93E0A0E0B0E05A
:107B200080935E0B90935F0BA093600BB093610BFF
:107B30006091F9057091FA058091FB059091FC0523
:107B4000F4C60A3009F09CC080915B02882339F1A9
:107B50006091490B70914A0B80914B0B90914C0BAB
:107B600025E030E040E050E00E9485DF2A3031051A
:107B70004105510551F481E196E00E94A42C9C013D
:107B8000812F68EC72E04EE309C081E196E00E942B
:107B9000A42C9C01812F68EC72E040E2D1D8809146
:107BA000410B82FFCDC66091490B70914A0B8091C9
:107BB0004B0B90914C0B25E030E040E050E00E94F0
:107BC00085DF2A3031054105510509F0B9C60FB6E8
:107BD000F89480914C1190914D11A0914E11B0915B
:107BE0004F110FBE8C509E4FAF4FBF4F8093430B32
:107BF0009093440BA093450BB093460B8091590290
:107C000090915A029093530B8093520B8091490BA1
:107C100090914A0B9093550B8093540B82E0809384
:107C20005B0282ED9EE490935A02809359028EEBA0
:107C300092E09093570B8093560B81E196E09093DE
:107C4000590B8093580B10925A0B10925B0B1092A9
:107C50005C0B10925D0B87EE93E0A0E0B0E08093A8
:107C60005E0B90935F0BA093600BB093610B6091E0
:107C7000110670911206809113069091140655C654
:107C80000B3009F0BCC080915B02882309F442C02C
:107C90006091490B70914A0B80914B0B90914C0B6A
:107CA00025E030E040E050E00E9485DF2B303105D8
:107CB00041055105C1F46091E9057091EA05809193
:107CC000EB059091EC050E942DDC69837A838B8310
:107CD0009C83CE0101960E940D2D9C01812F67EBA4
:107CE00072E04EE316C06091E9057091EA0580915B
:107CF000EB059091EC050E942DDC6D837E838F83D4
:107D00009887C1010E940D2D9C01812F67EB72E0C5
:107D100040E216D88091410B82FF12C66091490B58
:107D200070914A0B80914B0B90914C0B25E030E009
:107D300040E050E00E9485DF2B30310541055105C0
:107D400009F0FEC50FB6F89480914C1190914D1139
:107D5000A0914E11B0914F110FBE8C509E4FAF4F5E
:107D6000BF4F8093430B9093440BA093450BB0936C
:107D7000460B8091590290915A029093530B809335
:107D8000520B8091490B90914A0B9093550B809325
:107D9000540B82E080935B0284E69AE490935A024B
:107DA0008093590280EB92E09093570B8093560B8F
:107DB00089EE95E09093590B8093580B81E090E009
:107DC000A0E0B0E080935A0B90935B0BA0935C0B08
:107DD000B0935D0B8EED93E0A0E0B0E080935E0B7E
:107DE00090935F0BA093600BB093610B6091E905DA
:107DF0007091EA058091EB059091EC053CC20C3046
:107E000009F0BCC080915B02882309F442C06091F4
:107E1000490B70914A0B80914B0B90914C0B25E0D4
:107E200030E040E050E00E9485DF2C303105410514
:107E30005105B9F46091ED057091EE058091EF0563
:107E40009091F0050E942DDC69877A878B879C874B
:107E5000C2010E940D2D9C01812F69EA72E04EE360
:107E600016C06091ED057091EE058091EF0590913F
:107E7000F0050E942DDC6D877E878F87988BC3016C
:107E80000E940D2D9C01812F69EA72E040E20E9460
:107E9000A0368091410B82FF53C56091490B7091D0
:107EA0004A0B80914B0B90914C0B25E030E040E069
:107EB00050E00E9485DF2C3031054105510509F065
:107EC0003FC50FB6F89480914C1190914D11A0913F
:107ED0004E11B0914F110FBE8C509E4FAF4FBF4F00
:107EE0008093430B9093440BA093450BB093460BA8
:107EF0008091590290915A029093530B8093520BA8
:107F00008091490B90914A0B9093550B8093540BA1
:107F100082E080935B0284E69AE490935A02809315
:107F2000590282EA92E09093570B8093560B8DEEA4
:107F300095E09093590B8093580B81E090E0A0E07E
:107F4000B0E080935A0B90935B0BA0935C0BB093C3
:107F50005D0B8EED93E0A0E0B0E080935E0B90931C
:107F60005F0BA093600BB093610B6091ED05709176
:107F7000EE058091EF059091F0057DC10D3009F07F
:107F8000BCC080915B02882309F442C06091490B18
:107F900070914A0B80914B0B90914C0B25E030E097
:107FA00040E050E00E9485DF2D303105410551054C
:107FB000B9F46091F1057091F2058091F30590910B
:107FC000F4050E942DDC698B7A8B8B8B9C8BC40112
:107FD0000E940D2D9C01812F6BE972E04EE316C0CB
:107FE0006091F1057091F2058091F3059091F4058F
:107FF0000E942DDC6D8B7E8B8F8B988FC5010E942C
:108000000D2D9C01812F6BE972E040E20E94A036A9
:108010008091410B82FF94C46091490B70914A0B8F
:1080200080914B0B90914C0B25E030E040E050E00C
:108030000E9485DF2D3031054105510509F080C4CE
:108040000FB6F89480914C1190914D11A0914E1162
:10805000B0914F110FBE8C509E4FAF4FBF4F8093CA
:10806000430B9093440BA093450BB093460B809128
:10807000590290915A029093530B8093520B809126
:10808000490B90914A0B9093550B8093540B82E0CF
:1080900080935B0284E69AE490935A02809359029B
:1080A00084E992E09093570B8093560B81EF95E013
:1080B0009093590B8093580B81E090E0A0E0B0E0E2
:1080C00080935A0B90935B0BA0935C0BB0935D0B6A
:1080D0008EED93E0A0E0B0E080935E0B90935F0B99
:1080E000A093600BB093610B6091F1057091F20564
:1080F0008091F3059091F405BEC00E3009F0D4C014
:1081000080915B02882309F442C06091490B709111
:108110004A0B80914B0B90914C0B25E030E040E0F6
:1081200050E00E9485DF2E30310541055105B9F43C
:108130006091F5057091F6058091F7059091F8052D
:108140000E942DDC698F7A8F8B8F9C8FC6010E94D5
:108150000D2D9C01812F6DE872E04EE316C06091F9
:10816000F5057091F6058091F7059091F8050E944C
:108170002DDC6D8F7E8F8F8F98A3C7010E940D2DF0
:108180009C01812F6DE872E040E20E94A036809150
:10819000410B82FFD5C36091490B70914A0B8091CE
:1081A0004B0B90914C0B25E030E040E050E00E94FA
:1081B00085DF2E3031054105510509F0C1C30FB6E9
:1081C000F89480914C1190914D11A0914E11B09165
:1081D0004F110FBE8C509E4FAF4FBF4F8093430B3C
:1081E0009093440BA093450BB093460B809159029A
:1081F00090915A029093530B8093520B8091490BAC
:1082000090914A0B9093550B8093540B82E080938E
:108210005B0284E69AE490935A028093590286E8BE
:1082200092E09093570B8093560B85EF95E09093D7
:10823000590B8093580B81E090E0A0E0B0E0809370
:108240005A0B90935B0BA0935C0BB0935D0B8EED80
:1082500093E0A0E0B0E080935E0B90935F0BA0935F
:10826000600BB093610B6091F5057091F6058091FC
:10827000F7059091F8050E942DDC2AE037ED43E2E6
:108280005CE30E946DDE0E9401DC6093490B7093F9
:108290004A0B80934B0B90934C0B8CEB99E1909392
:1082A000630B8093620B8BC30F3009F0A5C08091E4
:1082B0005B02882341F16091490B70914A0B8091D8
:1082C0004B0B90914C0B25E030E040E050E00E94D9
:1082D00085DF2F3031054105510551F481E096E0ED
:1082E0000E940D2D9C01812F6CE772E04EE309C0C6
:1082F00081E096E00E940D2D9C01812F6CE772E0D9
:1083000040E20E94A0368091410B82FF19C3609128
:10831000490B70914A0B80914B0B90914C0B25E0CF
:1083200030E040E050E00E9485DF2F30310541050C
:10833000510509F005C30FB6F89480914C11909146
:108340004D11A0914E11B0914F110FBE8C509E4F08
:10835000AF4FBF4F8093430B9093440BA093450BBB
:10836000B093460B8091590290915A029093530B0F
:108370008093520B8091490B90914A0B9093550B2F
:108380008093540B82E080935B028CE59DE4909394
:108390005A028093590282E792E09093570B8093A0
:1083A000560B81E096E09093590B8093580B81E037
:1083B00090E0A0E0B0E080935A0B90935B0BA09309
:1083C0005C0BB0935D0B8EED93E0A0E0B0E080938A
:1083D0005E0B90935F0BA093600BB093610B609169
:1083E00001067091020680910306909104062AE02E
:1083F00037ED43E25CE397C2003109F0A1C0809100
:108400005B02882341F16091490B70914A0B809186
:108410004B0B90914C0B25E030E040E050E00E9487
:1084200085DF203131054105510551F489ED95E095
:108430000E943C2E9C01812F68E672E04EE309C049
:1084400089ED95E00E943C2E9C01812F68E672E048
:1084500040E20E94A0368091410B82FF71C2609180
:10846000490B70914A0B80914B0B90914C0B25E07E
:1084700030E040E050E00E9485DF203131054105C9
:10848000510509F05DC20FB6F89480914C1190919E
:108490004D11A0914E11B0914F110FBE8C509E4FB7
:1084A000AF4FBF4F8093430B9093440BA093450B6A
:1084B000B093460B8091590290915A029093530BBE
:1084C0008093520B8091490B90914A0B9093550BDE
:1084D0008093540B82E080935B0286EE9BE4909342
:1084E0005A02809359028EE592E09093570B809345
:1084F000560B89ED95E09093590B8093580B84EFC0
:1085000091E0A0E0B0E080935A0B90935B0BA093B6
:108510005C0BB0935D0B8CED91E4AFE0B0E0809329
:108520005E0B90935F0BA093600BB093610B609117
:10853000D9057091DA058091DB059091DC05A3C027
:10854000013109F0A5C080915B02882341F160915F
:10855000490B70914A0B80914B0B90914C0B25E08D
:1085600030E040E050E00E9485DF213131054105D7
:10857000510551F48DED95E00E943C2E9C01812F18
:1085800064E572E04EE309C08DED95E00E943C2E5B
:108590009C01812F64E572E040E20E94A036809148
:1085A000410B82FFCDC16091490B70914A0B8091C4
:1085B0004B0B90914C0B25E030E040E050E00E94E6
:1085C00085DF213131054105510509F0B9C10FB6EB
:1085D000F89480914C1190914D11A0914E11B09151
:1085E0004F110FBE8C509E4FAF4FBF4F8093430B28
:1085F0009093440BA093450BB093460B8091590286
:1086000090915A029093530B8093520B8091490B97
:1086100090914A0B9093550B8093540B82E080937A
:108620005B0286EE9BE490935A02809359028AE49F
:1086300092E09093570B8093560B8DED95E09093BD
:10864000590B8093580B84EF91E0A0E0B0E0809349
:108650005A0B90935B0BA0935C0BB0935D0B8CED6E
:1086600091E4AFE0B0E080935E0B90935F0BA0933A
:10867000600BB093610B6091DD057091DE05809118
:10868000DF059091E00520E030E048EC52E44BC17A
:10869000023109F0A1C080915B02882341F1609111
:1086A000490B70914A0B80914B0B90914C0B25E03C
:1086B00030E040E050E00E9485DF22313105410585
:1086C000510551F481EE95E00E94B52D9C01812F5A
:1086D00060E472E04EE309C081EE95E00E94B52DA2
:1086E0009C01812F60E472E040E20E94A0368091FC
:1086F000410B82FF25C16091490B70914A0B80911B
:108700004B0B90914C0B25E030E040E050E00E9494
:1087100085DF223131054105510509F011C10FB640
:10872000F89480914C1190914D11A0914E11B091FF
:108730004F110FBE8C509E4FAF4FBF4F8093430BD6
:108740009093440BA093450BB093460B8091590234
:1087500090915A029093530B8093520B8091490B46
:1087600090914A0B9093550B8093540B82E0809329
:108770005B0281EA9CE490935A028093590286E35B
:1087800092E09093570B8093560B81EE95E0909377
:10879000590B8093580B82E390E0A0E0B0E0809307
:1087A0005A0B90935B0BA0935C0BB0935D0B86E927
:1087B00096E8A1E0B0E080935E0B90935F0BA093EE
:1087C000600BB093610B6091E1057091E2058091BF
:1087D000E3059091E405A3C0033109F0B1C0809195
:1087E0005B02882341F16091490B70914A0B8091A3
:1087F0004B0B90914C0B25E030E040E050E00E94A4
:1088000085DF233131054105510551F485EE95E0B1
:108810000E94B52D9C01812F6CE272E04EE309C0ED
:1088200085EE95E00E94B52D9C01812F6CE272E0EF
:1088300040E20E94A0368091410B82FF81C060918E
:10884000490B70914A0B80914B0B90914C0B25E09A
:1088500030E040E050E00E9485DF233131054105E2
:10886000510509F06DC00FB6F89480914C119091AC
:108870004D11A0914E11B0914F110FBE8C509E4FD3
:10888000AF4FBF4F8093430B9093440BA093450B86
:10889000B093460B8091590290915A029093530BDA
:1088A0008093520B8091490B90914A0B9093550BFA
:1088B0008093540B82E080935B0281EA9CE4909366
:1088C0005A028093590282E292E09093570B809370
:1088D000560B85EE95E09093590B8093580B82E3ED
:1088E00090E0A0E0B0E080935A0B90935B0BA093D4
:1088F0005C0BB0935D0B86E996E8A1E0B0E0809355
:108900005E0B90935F0BA093600BB093610B609133
:10891000E5057091E6058091E7059091E80520E076
:1089200030E040E251E40E946DDE0E9401DC609381
:10893000490B70934A0B80934B0B90934C0B3FC0A9
:108940008091490B90914A0BA0914B0BB0914C0B2D
:1089500084369105A105B10560F083E690E0A0E0C2
:10896000B0E08093490B90934A0BA0934B0BB093CC
:108970004C0B6091490B70914A0B80914B0B90917D
:108980004C0B25E030E040E050E00E9485DF422FB4
:108990008091420B90E0039630E0821793074CF4ED
:1089A00043504093420B81E080935B02042F0150BF
:1089B0001FEF1F5F143018F40F5F0C946F37A096F1
:1089C0000FB6F894DEBF0FBECDBFCF91DF911F91E0
:1089D0000F91FF90EF90DF90CF90BF90AF909F905E
:1089E0008F907F906F905F904F903F902F90089561
:1089F0007F928F929F92AF92BF92CF92DF92EF922F
:108A0000FF920F931F938091490B90914A0BA09175
:108A10004B0BB0914C0B81509048A040B04040F0BF
:108A20001092490B10924A0B10924B0B10924C0B68
:108A30006091490B70914A0B80914B0B90914C0BBC
:108A400025E030E040E050E00E9485DF79018A01B6
:108A50008091420B90E0A0E0B0E0E816F9060A072A
:108A60001B0710F42093420BC090420BDD2417E249
:108A7000812E912CA12CB12C77247394CC2009F059
:108A800056C080915B028823C1F08091490B909180
:108A90004A0BA0914B0BB0914C0B0597A105B1056A
:108AA00028F48D2D69ED75E043E004C08D2D69ED4E
:108AB00075E040E223E00E94C32E8091410B82FFCB
:108AC00087C48091490B90914A0BA0914B0BB091B8
:108AD0004C0B0597A105B10508F07AC482E080939C
:108AE0005B020FB6F89480914C1190914D11A091BA
:108AF0004E11B0914F110FBE8C509E4FAF4FBF4FD4
:108B00008093430B9093440BA093450BB093460B7B
:108B10008EE494E590935A02809359021092490B87
:108B200010924A0B10924B0B10924C0B8BC481E0AD
:108B3000C81609F09BC080915B02882341F16091C7
:108B4000490B70914A0B80914B0B90914C0B25E097
:108B500030E040E050E00E9485DF213031054105E2
:108B6000510551F48CE692E00E946F2C9C018D2DF2
:108B700063ED75E04EE309C08CE692E00E946F2C35
:108B80009C018D2D63ED75E040E20E94A03680913E
:108B9000410B82FF1DC4E090490BF0904A0B0091FD
:108BA0004B0B10914C0BC801B70125E030E040E0C1
:108BB00050E00E9485DF213031054105510509F063
:108BC00007C40FB6F89480914C1190914D11A0916B
:108BD0004E11B0914F110FBE8C509E4FAF4FBF4FF3
:108BE0008093430B9093440BA093450BB093460B9B
:108BF0008091590290915A029093530B8093520B9B
:108C0000F092550BE092540B82E080935B0281E876
:108C10009FE490935A02809359028DEC95E09093D3
:108C2000570B8093560B8CE692E09093590B8093F0
:108C3000580B8AE090E0A0E0B0E080935A0B90934C
:108C40005B0BA0935C0BB0935D0B87EE93E0A0E011
:108C5000B0E080935E0B90935F0BA093600BB0939A
:108C6000610B80916C0290916D02A5C322E0C21647
:108C700009F097C080915B02882341F16091490B14
:108C800070914A0B80914B0B90914C0B25E030E09A
:108C900040E050E00E9485DF22303105410551055A
:108CA00051F483E99FE00E946F2C9C018D2D66ECAE
:108CB00075E04EE309C083E99FE00E946F2C9C01A0
:108CC0008D2D66EC75E040E20E94A0368091410B4C
:108CD00082FF7EC3E090490BF0904A0B00914B0B52
:108CE00010914C0BC801B70125E030E040E050E0A6
:108CF0000E9485DF223031054105510509F068C326
:108D00000FB6F89480914C1190914D11A0914E1195
:108D1000B0914F110FBE8C509E4FAF4FBF4F8093FD
:108D2000430B9093440BA093450BB093460B80915B
:108D3000590290915A029093530B8093520BF092E8
:108D4000550BE092540B82E080935B0281E89FE434
:108D500090935A02809359028FEB95E09093570BB2
:108D60008093560B83E99FE09093590B8093580BA7
:108D700010925A0B10925B0B10925C0B10925D0BD1
:108D800084E091E0A0E0B0E080935E0B90935F0BF5
:108D9000A093600BB093610B8091930F9091940F0F
:108DA0000AC383E0C81609F097C080915B0288234C
:108DB00041F16091490B70914A0B80914B0B90915E
:108DC0004C0B25E030E040E050E00E9485DF23308E
:108DD00031054105510551F485E99FE00E946F2C52
:108DE0009C018D2D67EB75E04EE309C085E99FE09E
:108DF0000E946F2C9C018D2D67EB75E040E20E9474
:108E0000A0368091410B82FFE3C2E090490BF090C5
:108E10004A0B00914B0B10914C0BC801B70125E098
:108E200030E040E050E00E9485DF2330310541050D
:108E3000510509F0CDC20FB6F89480914C11909174
:108E40004D11A0914E11B0914F110FBE8C509E4FFD
:108E5000AF4FBF4F8093430B9093440BA093450BB0
:108E6000B093460B8091590290915A029093530B04
:108E70008093520BF092550BE092540B82E080935A
:108E80005B0281E89FE490935A02809359028FEA33
:108E900095E09093570B8093560B85E99FE0909354
:108EA000590B8093580B10925A0B10925B0B109237
:108EB0005C0B10925D0B84E091E0A0E0B0E0809349
:108EC0005E0B90935F0BA093600BB093610B80914E
:108ED000950F9091960F6FC224E0C21609F097C0CB
:108EE00080915B02882341F16091490B70914A0B9C
:108EF00080914B0B90914C0B25E030E040E050E02E
:108F00000E9485DF243031054105510551F487E980
:108F10009FE00E946F2C9C018D2D67EA75E04EE367
:108F200009C087E99FE00E946F2C9C018D2D67EAA4
:108F300075E040E20E94A0368091410B82FF48C25A
:108F4000E090490BF0904A0B00914B0B10914C0BA9
:108F5000C801B70125E030E040E050E00E9485DF25
:108F6000243031054105510509F032C20FB6F8949D
:108F700080914C1190914D11A0914E11B0914F11D3
:108F80000FBE8C509E4FAF4FBF4F8093430B9093BB
:108F9000440BA093450BB093460B809159029091DE
:108FA0005A029093530B8093520BF092550BE09220
:108FB000540B82E080935B0281E89FE490935A0215
:108FC000809359028FE995E09093570B8093560B4D
:108FD00087E99FE09093590B8093580B10925A0B9E
:108FE00010925B0B10925C0B10925D0B84E091E091
:108FF000A0E0B0E080935E0B90935F0BA093600BBA
:10900000B093610B8091970F9091980FD4C185E038
:10901000C81609F097C080915B02882341F16091E6
:10902000490B70914A0B80914B0B90914C0B25E0B2
:1090300030E040E050E00E9485DF253031054105F9
:10904000510551F489E99FE00E946F2C9C018D2D00
:109050006BE975E04EE309C089E99FE00E946F2C3F
:109060009C018D2D6BE975E040E20E94A036809155
:10907000410B82FFADC1E090490BF0904A0B00918B
:109080004B0B10914C0BC801B70125E030E040E0DC
:1090900050E00E9485DF253031054105510509F07A
:1090A00097C10FB6F89480914C1190914D11A091F9
:1090B0004E11B0914F110FBE8C509E4FAF4FBF4F0E
:1090C0008093430B9093440BA093450BB093460BB6
:1090D0008091590290915A029093530B8093520BB6
:1090E000F092550BE092540B82E080935B0281E892
:1090F0009FE490935A028093590287E995E09093F8
:10910000570B8093560B89E99FE09093590B8093FE
:10911000580B10925A0B10925B0B10925C0B109232
:109120005D0B87E890E0A0E0B0E080935E0B909349
:109130005F0BA093600BB093610B8091990F90919E
:109140009A0F39C126E0C21609F097C080915B02E0
:10915000882341F16091490B70914A0B80914B0B30
:1091600090914C0B25E030E040E050E00E9485DF1C
:10917000263031054105510551F482EB9DE00E94F6
:109180006F2C9C018D2D6DE875E04EE309C082EBDC
:109190009DE00E946F2C9C018D2D6DE875E040E2F2
:1091A0000E94A0368091410B82FF12C1E090490BD2
:1091B000F0904A0B00914B0B10914C0BC801B7017A
:1091C00025E030E040E050E00E9485DF26303105A8
:1091D0004105510509F0FCC00FB6F89480914C117F
:1091E00090914D11A0914E11B0914F110FBE8C5026
:1091F0009E4FAF4FBF4F8093430B9093440BA09370
:10920000450BB093460B8091590290915A0290936E
:10921000530B8093520BF092550BE092540B82E06B
:1092200080935B0281E89FE490935A0280935902F5
:1092300083E895E09093570B8093560B82EB9DE06B
:109240009093590B8093580B10925A0B10925B0B12
:1092500010925C0B10925D0B8FEF90E0A0E0B0E0FD
:1092600080935E0B90935F0BA093600BB093610BA8
:109270008091B20D9091B30D9EC087E0C81609F0A1
:10928000A7C080915B02882341F16091490B7091E6
:109290004A0B80914B0B90914C0B25E030E040E065
:1092A00050E00E9485DF273031054105510551F41A
:1092B0008EE692E00E946F2C9C018D2D6EE775E08A
:1092C0004EE309C08EE692E00E946F2C9C018D2D2A
:1092D0006EE775E040E20E94A0368091410B82FF6C
:1092E00077C0E090490BF0904A0B00914B0B109126
:1092F0004C0BC801B70125E030E040E050E00E948F
:1093000085DF273031054105510509F061C00FB6F1
:10931000F89480914C1190914D11A0914E11B09103
:109320004F110FBE8C509E4FAF4FBF4F8093430BDA
:109330009093440BA093450BB093460B8091590238
:1093400090915A029093530B8093520BF092550BCD
:10935000E092540B82E080935B0281E89FE490935B
:109360005A028093590289E795E09093570B8093B6
:10937000560B8EE692E09093590B8093580B8AE03F
:1093800090E0A0E0B0E080935A0B90935B0BA09329
:109390005C0BB0935D0B87EE93E0A0E0B0E08093B0
:1093A0005E0B90935F0BA093600BB093610B809169
:1093B0006E0290916F02AA2797FDA095BA2F809315
:1093C000490B90934A0BA0934B0BB0934C0B3AC0B4
:1093D0008091490B90914A0BA0914B0BB0914C0B93
:1093E0008897A105B10540F08092490B90924A0BF5
:1093F000A0924B0BB0924C0B6091490B70914A0BB1
:1094000080914B0B90914C0B25E030E040E050E018
:109410000E9485DF422F8091420B90E0039630E05E
:10942000821793074CF443504093420B70925B02B7
:10943000C42ECA94DD24DA94D39423E02D1510F0C1
:10944000C3941CCB1F910F91FF90EF90DF90CF90B2
:10945000BF90AF909F908F907F900895CF92DF92B2
:10946000EF92FF920F931F937C01D62EC72E0DE231
:109470001BE0C80161E041E00E9477D1C7010E9472
:109480008733E0912D0BF0912E0B0190F081E02DB0
:10949000C8016AE30995ED2DFC2DDF010D90002038
:1094A000E9F7EA1BEC5EC8016E2F41E00E9477D11C
:1094B000C8016D2D7C2D0E9497331F910F91FF9055
:1094C000EF90DF90CF9008950F931F93DF93CF938A
:1094D00000D000D0CDB7DEB720915A0B30915B0B96
:1094E00040915C0B50915D0B8091490B90914A0B20
:1094F000A0914B0BB0914C0B82179307A407B507B3
:1095000044F42093490B30934A0B40934B0B5093F8
:109510004C0B20915E0B30915F0B4091600B509192
:10952000610B8091490B90914A0BA0914B0BB0912C
:109530004C0B281739074A075B0744F42093490B63
:1095400030934A0B40934B0B50934C0B80915B0232
:109550008823F9F00091560B1091570B6091490B3D
:1095600070914A0B80914B0B90914C0B0E942DDC1B
:109570002AE037ED43E25CE30E9494DB69837A835F
:109580008B839C83CE0101960E940D2DBC01C801E6
:1095900065DF8091410B82FF50C00091580B109104
:1095A000590B6091490B70914A0B80914B0B909134
:1095B0004C0B0E942DDC2AE037ED43E25CE30E9475
:1095C00094DB0E9401DCF8016083718382839383C2
:1095D00082E080935B020FB6F89480914C119091D9
:1095E0004D11A0914E11B0914F110FBE8C509E4F56
:1095F000AF4FBF4F8093430B9093440BA093450B09
:10960000B093460B8091520B9091530B90935A025A
:10961000809359028091540B9091550BA0E0B0E0DB
:109620008093490B90934A0BA0934B0BB0934C0B38
:10963000E091620BF091630B09950F900F900F90E2
:109640000F90CF91DF911F910F9108950F931F936A
:10965000DF93CF9300D000D0CDB7DEB720915A0B67
:1096600030915B0B40915C0B50915D0B8091490BED
:1096700090914A0BA0914B0BB0914C0B8217930722
:10968000A407B50744F42093490B30934A0B409349
:109690004B0B50934C0B20915E0B30915F0B409124
:1096A000600B5091610B8091490B90914A0BA091F6
:1096B0004B0BB0914C0B281739074A075B0744F452
:1096C0002093490B30934A0B40934B0B50934C0B18
:1096D00080915B028823F9F00091560B1091570B93
:1096E0006091490B70914A0B80914B0B90914C0B00
:1096F0000E942DDC20E030E048EC52E40E9494DB34
:1097000069837A838B839C83CE0101960E943C2ED1
:10971000BC01C801A3DE8091410B82FF4EC00091C5
:10972000580B1091590B6091490B70914A0B809125
:109730004B0B90914C0B0E942DDC20E030E048EC6C
:1097400052E40E9494DBF8016083718382839383E7
:1097500082E080935B020FB6F89480914C11909157
:109760004D11A0914E11B0914F110FBE8C509E4FD4
:10977000AF4FBF4F8093430B9093440BA093450B87
:10978000B093460B8091520B9091530B90935A02D9
:10979000809359028091540B9091550BA0E0B0E05A
:1097A0008093490B90934A0BA0934B0BB0934C0BB7
:1097B000E091620BF091630B09950F900F900F9061
:1097C0000F90CF91DF911F910F9108950F931F93E9
:1097D000DF93CF9300D000D0CDB7DEB720915A0BE6
:1097E00030915B0B40915C0B50915D0B8091490B6C
:1097F00090914A0BA0914B0BB0914C0B82179307A1
:10980000A407B50744F42093490B30934A0B4093C7
:109810004B0B50934C0B20915E0B30915F0B4091A2
:10982000600B5091610B8091490B90914A0BA09174
:109830004B0BB0914C0B281739074A075B0744F4D0
:109840002093490B30934A0B40934B0B50934C0B96
:1098500080915B028823F9F00091560B1091570B11
:109860006091490B70914A0B80914B0B90914C0B7E
:109870000E942DDC20E030E048EC52E40E9494DBB2
:1098800069837A838B839C83CE0101960E943C2E50
:10989000BC01C801E3DD8091410B82FF49C000910A
:1098A000580B1091590B6091490B70914A0B8091A4
:1098B0004B0B90914C0B0E942DDC20E030E048ECEB
:1098C00052E40E9494DBF801608371838283938366
:1098D00082E080935B020FB6F89480914C119091D6
:1098E0004D11A0914E11B0914F110FBE8C509E4F53
:1098F000AF4FBF4F8093430B9093440BA093450B06
:10990000B093460B8091520B9091530B90935A0257
:10991000809359028091540B9091550BA0E0B0E0D8
:109920008093490B90934A0BA0934B0BB0934C0B35
:109930000F900F900F900F90CF91DF911F910F918B
:1099400008950F931F93DF93CF9300D000D0CDB72E
:10995000DEB720915A0B30915B0B40915C0B50911C
:109960005D0B8091490B90914A0BA0914B0BB091EC
:109970004C0B82179307A407B50744F42093490BB7
:1099800030934A0B40934B0B50934C0B20915E0B42
:1099900030915F0B4091600B5091610B8091490BAE
:1099A00090914A0BA0914B0BB0914C0B28173907A3
:1099B0004A075B0744F42093490B30934A0B4093CA
:1099C0004B0B50934C0B80915B028823F9F0009174
:1099D000560B1091570B6091490B70914A0B809177
:1099E0004B0B90914C0B0E942DDC20E030E040E2CC
:1099F00051E40E9494DB69837A838B839C83CE013C
:109A000001960E94B52DBC01C80128DD8091410B53
:109A100082FF49C00091580B1091590B6091490B7E
:109A200070914A0B80914B0B90914C0B0E942DDC56
:109A300020E030E040E251E40E9494DBF8016083D2
:109A400071838283938382E080935B020FB6F894E4
:109A500080914C1190914D11A0914E11B0914F11E8
:109A60000FBE8C509E4FAF4FBF4F8093430B9093D0
:109A7000440BA093450BB093460B8091520B9091F1
:109A8000530B90935A02809359028091540B9091FA
:109A9000550BA0E0B0E08093490B90934A0BA09344
:109AA0004B0BB0934C0B0F900F900F900F90CF91EA
:109AB000DF911F910F9108950F931F93DF93CF9321
:109AC00000D000D0CDB7DEB720915A0B30915B0BA0
:109AD00040915C0B50915D0B8091490B90914A0B2A
:109AE000A0914B0BB0914C0B82179307A407B507BD
:109AF00044F42093490B30934A0B40934B0B509303
:109B00004C0B20915E0B30915F0B4091600B50919C
:109B1000610B8091490B90914A0BA0914B0BB09136
:109B20004C0B281739074A075B0744F42093490B6D
:109B300030934A0B40934B0B50934C0B80915B023C
:109B40008823F9F00091560B1091570B6091490B47
:109B500070914A0B80914B0B90914C0B0E942DDC25
:109B60002AE037ED43E25CE30E9494DB69837A8369
:109B70008B839C83CE0101960E940D2DBC01C801F0
:109B80006DDC8091410B82FF49C00091580B109110
:109B9000590B6091490B70914A0B80914B0B90913E
:109BA0004C0B0E942DDC2AE037ED43E25CE30E947F
:109BB00094DBF801608371838283938382E08093D6
:109BC0005B020FB6F89480914C1190914D11A091C9
:109BD0004E11B0914F110FBE8C509E4FAF4FBF4FE3
:109BE0008093430B9093440BA093450BB093460B8B
:109BF0008091520B9091530B90935A02809359028B
:109C00008091540B9091550BA0E0B0E08093490BEC
:109C100090934A0BA0934B0BB0934C0B0F900F906B
:109C20000F900F90CF91DF911F910F9108950F9397
:109C30001F93DF93CF9300D000D0CDB7DEB7209134
:109C40005A0B30915B0B40915C0B50915D0B8091F6
:109C5000490B90914A0BA0914B0BB0914C0B821782
:109C60009307A407B50744F42093490B30934A0B9C
:109C700040934B0B50934C0B20915E0B30915F0B3C
:109C80004091600B5091610B8091490B90914A0B70
:109C9000A0914B0BB0914C0B281739074A075B0773
:109CA00044F42093490B30934A0B40934B0B509351
:109CB0004C0B80915B028823F9F00091560B1091B8
:109CC000570B6091490B70914A0B80914B0B90910F
:109CD0004C0B0E942DDC20E030E048EC52E40E9466
:109CE00094DB69837A838B839C83CE0101960E94E7
:109CF000EB2BBC01C801B2DB8091410B82FF49C054
:109D00000091580B1091590B6091490B70914A0BBF
:109D100080914B0B90914C0B0E942DDC20E030E0A9
:109D200048EC52E40E9494DBF801608371838283E3
:109D3000938382E080935B020FB6F89480914C117C
:109D400090914D11A0914E11B0914F110FBE8C50BA
:109D50009E4FAF4FBF4F8093430B9093440BA09304
:109D6000450BB093460B8091520B9091530B9093FF
:109D70005A02809359028091540B9091550BA0E0A8
:109D8000B0E08093490B90934A0BA0934B0BB09398
:109D90004C0B0F900F900F900F90CF91DF911F9170
:109DA0000F9108950F931F93DF93CF9300D000D0AE
:109DB000CDB7DEB720915A0B30915B0B40915C0B15
:109DC00050915D0B8091490B90914A0BA0914B0BE8
:109DD000B0914C0B82179307A407B50744F4209366
:109DE000490B30934A0B40934B0B50934C0B2091F3
:109DF0005E0B30915F0B4091600B5091610B809135
:109E0000490B90914A0BA0914B0BB0914C0B28172A
:109E100039074A075B0744F42093490B30934A0BF8
:109E200040934B0B50934C0B80915B028823C9F0FD
:109E30000091560B1091570B6091490B70914A0B92
:109E400080914B0B90914C0B0E942DDC69837A839F
:109E50008B839C83CE0101960E94A42CBC01C80177
:109E6000FDDA8091410B82FF43C00091580B1091A5
:109E7000590B6091490B70914A0B80914B0B90915B
:109E80004C0B0E942DDCF8016083718382839383E5
:109E900082E080935B020FB6F89480914C11909110
:109EA0004D11A0914E11B0914F110FBE8C509E4F8D
:109EB000AF4FBF4F8093430B9093440BA093450B40
:109EC000B093460B8091520B9091530B90935A0292
:109ED000809359028091540B9091550BA0E0B0E013
:109EE0008093490B90934A0BA0934B0BB0934C0B70
:109EF0000F900F900F900F90CF91DF911F910F91C6
:109F000008950F931F93DF93CF9300D0CDB7DEB7A3
:109F100020915A0B30915B0B40915C0B50915D0B83
:109F20008091490B90914A0BA0914B0BB0914C0B37
:109F300082179307A407B50744F42093490B309385
:109F40004A0B40934B0B50934C0B20915E0B30917E
:109F50005F0B4091600B5091610B8091490B909188
:109F60004A0BA0914B0BB0914C0B281739074A07AD
:109F70005B0744F42093490B30934A0B40934B0BFF
:109F800050934C0B80915B02882389F00091560B13
:109F90001091570B8091490B90914A0B9A838983BA
:109FA000CE0101960E946F2CBC01C80157DA809146
:109FB000410B82FF3AC0E091580BF091590B809110
:109FC000490B90914A0B9183808382E080935B02DE
:109FD0000FB6F89480914C1190914D11A0914E11B3
:109FE000B0914F110FBE8C509E4FAF4FBF4F80931B
:109FF000430B9093440BA093450BB093460B809179
:10A00000520B9091530B90935A0280935902809176
:10A01000540B9091550BA0E0B0E08093490B9093C6
:10A020004A0BA0934B0BB0934C0B0F900F90CF911A
:10A03000DF911F910F9108950F931F93DF93CF939B
:10A04000CDB7DEB76E970FB6F894DEBF0FBECDBFAB
:10A0500000D000D000D0EDB7FEB731969E012F5F43
:10A060003F4FADB7BEB712963C932E9311972DEC90
:10A0700031E033832283958384830E940B118E0108
:10A080000B5F1F4FEDB7FEB736960FB6F894FEBFC5
:10A090000FBEEDBF08C0992787FD90950E94D0DFC5
:10A0A000D8018D938D01F80180818823A1F7CE011D
:10A0B00001960E94759989EC91E00E94FE98109299
:10A0C000490B10924A0B10924B0B10924C0B82EFE3
:10A0D00095E390935A02809359026E960FB6F894C6
:10A0E000DEBF0FBECDBFCF91DF911F910F910895BD
:10A0F0008CE79BE00E9475C31092420B08958CE799
:10A100009BE00E940CC91092420B08959F92AF925F
:10A11000BF92CF92DF92EF92FF920F931F93CF9354
:10A12000DF938CE79BE00E94C3CC5C018091490BDC
:10A1300090914A0BA0914B0BB0914C0B81509048E1
:10A14000A040B04040F01092490B10924A0B109280
:10A150004B0B10924C0B6091490B70914A0B809104
:10A160004B0B90914C0B25E030E040E050E00E941A
:10A1700085DF79018A018091420B90E0A0E0B0E098
:10A18000E816F9060A071B0710F42093420BE0902B
:10A19000420BFF2499249394EE2009F04DC0809146
:10A1A0005B028823C1F08091490B90914A0BA091EA
:10A1B0004B0BB0914C0B0597A105B10528F48F2DE1
:10A1C00064EC71E043E004C08F2D64EC71E040E288
:10A1D00023E00E94C32E8091410B82FF2DC080910D
:10A1E000490B90914A0BA0914B0BB0914C0B0597EA
:10A1F000A105B10508F582E080935B020FB6F894E3
:10A2000080914C1190914D11A0914E11B0914F1130
:10A210000FBE8C509E4FAF4FBF4F8093430B909318
:10A22000440BA093450BB093460B8EE494E59093BA
:10A230005A0280935902BAC18EEC9BE060E87BE041
:10A240000E9426B18091800B8F3209F05DC081E0C1
:10A25000E81621F002E0CC24DD2485C280915B0267
:10A260008823F9F06091490B70914A0B80914B0B58
:10A2700090914C0B25E030E040E050E00E9485DFFB
:10A28000213031054105510529F48F2D6BEB71E02B
:10A290004EE304C08F2D6BEB71E040E220E20E94A0
:10A2A000C32E8091410B82FFD5CF6091490B7091F5
:10A2B0004A0B80914B0B90914C0B25E030E040E035
:10A2C00050E00E9485DF213031054105510511F62E
:10A2D00082E080935B020FB6F89480914C119091CC
:10A2E0004D11A0914E11B0914F110FBE8C509E4F49
:10A2F000AF4FBF4F8093430B9093440BA093450BFC
:10A30000B093460BFCDE81C221E0E21609F0A2CF39
:10A3100080915B028823F9F06091490B70914A0BA0
:10A3200080914B0B90914C0B25E030E040E050E0E9
:10A330000E9485DF213031054105510529F48F2D1B
:10A3400067EB71E04EE304C08F2D67EB71E040E2F4
:10A3500020E20E94C32E8091410B82FF7BCF60914F
:10A36000490B70914A0B80914B0B90914C0B25E05F
:10A3700030E040E050E00E9485DF213031054105AA
:10A38000510509F067CF82E080935B020FB6F89425
:10A3900080914C1190914D11A0914E11B0914F119F
:10A3A0000FBE8C509E4FAF4FBF4F8093430B909387
:10A3B000440BA093450BB093460B9ADE26C20E15B4
:10A3C00009F0CDC18CE79BE06C2D0E9421CD8091DE
:10A3D000A80B90915B02882309F4F1C0992309F43A
:10A3E000A9C06091490B70914A0B80914B0B9091E1
:10A3F0004C0B25E030E040E050E00E9485DF802FEC
:10A4000090E0A0E0B0E0281739074A075B0709F0A1
:10A4100049C08DE29BE060E04F2D0E9477D1E09132
:10A420002D0BF0912E0B0190F081E02D8DE29BE041
:10A430006EE30995E0912D0BF0912E0B0190F081C8
:10A44000E02D8DE29BE065E0099580918D0B8823DE
:10A4500019F4C0E8DBE004C010929F0BCDE8DBE00C
:10A4600012E168816623D9F01123C9F0E0912D0B28
:10A47000F0912E0B0190F081E02D8DE29BE009958B
:10A4800021961150EECFE0912D0BF0912E0B019003
:10A49000F081E02D8DE29BE060E2099511501123DF
:10A4A00091F748C08DE29BE060E04F2D0E9477D18C
:10A4B000E0912D0BF0912E0B0190F081E02D8DE2BB
:10A4C0009BE060E20995E0912D0BF0912E0B01903D
:10A4D000F081E02D8DE29BE065E0099580918D0B88
:10A4E000882319F4C0E8DBE004C010929F0BCDE88C
:10A4F000DBE012E168816623D9F01123C9F0E09115
:10A500002D0BF0912E0B0190F081E02D8DE29BE060
:10A51000099521961150EECFE0912D0BF0912E0B65
:10A520000190F081E02D8DE29BE060E209951150F1
:10A53000112391F78091410B82FF11C16091490B6A
:10A5400070914A0B80914B0B90914C0B25E030E0C1
:10A5500040E050E00E9485DF802F90E0A0E0B0E076
:10A56000281739074A075B0709F0F9C082E0809392
:10A570005B020FB6F89480914C1190914D11A0910F
:10A580004E11B0914F110FBE8C509E4FAF4FBF4F29
:10A590008093430B9093440BA093450BB093460BD1
:10A5A0008CE79BE060E87BE00E9400C41092490BBE
:10A5B00010924A0B10924B0B10924C0B26C1992310
:10A5C00009F492C06091490B70914A0B80914B0B3A
:10A5D00090914C0B25E030E040E050E00E9485DF98
:10A5E000802F90E0A0E0B0E0281739074A075B070A
:10A5F000F1F58DE29BE060E04F2D0E9477D1E09174
:10A600002D0BF0912E0B0190F081E02D8DE29BE05F
:10A610006EE3099580918D0B882319F4C0E8DBE087
:10A6200004C01092A00BCDE8DBE013E16881662343
:10A63000D9F01123C9F0E0912D0BF0912E0B019070
:10A64000F081E02D8DE29BE0099521961150EECF2F
:10A65000E0912D0BF0912E0B0190F081E02D8DE219
:10A660009BE060E209951150112391F73DC08DE206
:10A670009BE060E04F2D0E9477D1E0912D0BF0918F
:10A680002E0B0190F081E02D8DE29BE060E20995B8
:10A6900080918D0B882319F4C0E8DBE004C0109290
:10A6A000A00BCDE8DBE013E168816623D9F011232C
:10A6B000C9F0E0912D0BF0912E0B0190F081E02D6F
:10A6C0008DE29BE0099521961150EECFE0912D0B84
:10A6D000F0912E0B0190F081E02D8DE29BE060E285
:10A6E00009951150112391F78091410B82FF37C0DA
:10A6F0006091490B70914A0B80914B0B90914C0BE0
:10A7000025E030E040E050E00E9485DF802F90E0BF
:10A71000A0E0B0E0281739074A075B0701F582E09F
:10A7200080935B020FB6F89480914C1190914D117B
:10A73000A0914E11B0914F110FBE8C509E4FAF4F54
:10A74000BF4F8093430B9093440BA093450BB09362
:10A75000460B80E89BE06DE87BE06EDC56C00F5F47
:10A760000894C11CD11CCA14DB0408F428CE6091E3
:10A77000490B70914A0B80914B0B90914C0B25E04B
:10A7800030E040E050E00E9485DF802F90E0A0E0C4
:10A79000B0E0281739074A075B0788F085E0089F73
:10A7A000C00111240197AA2797FDA095BA2F809385
:10A7B000490B90934A0BA0934B0BB0934C0B6091B9
:10A7C000490B70914A0B80914B0B90914C0B25E0FB
:10A7D00030E040E050E00E9485DF422F8091420B44
:10A7E00090E0039630E0821793074CF44350409377
:10A7F000420B90925B02E42EEA94FF24FA94F394C5
:10A8000083E08F1510F0E394C7CCDF91CF911F91B7
:10A810000F91FF90EF90DF90CF90BF90AF909F90FF
:10A820000895CF93DF9310927E0B8CE79BE00E94FC
:10A83000C7C40E9437A884ED91E00E94FE988091E1
:10A840003506882301F1109235068091B10DC82F8D
:10A85000D0E0CC0FDD1FCD56D04F6881798188279D
:10A8600077FD8095982F0E942FDC2091380230913F
:10A87000390240913A0250913B020E949BDD18162A
:10A8800014F419821882DF91CF9108958CE79BE030
:10A890000C9469C38CE79BE00C9470C3BF92CF9279
:10A8A000DF92EF92FF920F931F938091490B90914B
:10A8B0004A0BA0914B0BB0914C0B81509048A0409B
:10A8C000B04040F01092490B10924A0B10924B0B83
:10A8D00010924C0B6091490B70914A0B80914B0B7D
:10A8E00090914C0B25E030E040E050E00E9485DF85
:10A8F00079018A018091420B90E0A0E0B0E0E81677
:10A90000F9060A071B0710F42093420B0091420B33
:10A9100010E098E1C92ED12CE12CF12CBB24B3948A
:10A92000002309F049C080915B028823C1F0809127
:10A93000490B90914A0BA0914B0BB0914C0B059792
:10A94000A105B10528F4812F6BEA71E043E004C052
:10A95000812F6BEA71E040E223E00E94C32E8091D8
:10A96000410B82FF29C08091490B90914A0BA09125
:10A970004B0BB0914C0B0597A105B105E8F482E0B3
:10A9800080935B020FB6F89480914C1190914D1119
:10A99000A0914E11B0914F110FBE8C509E4FAF4FF2
:10A9A000BF4F8093430B9093440BA093450BB09300
:10A9B000460B82EF95E30AC30E94AC19882329F461
:10A9C00080917E0B882309F4A2C3013009F0B0C046
:10A9D00080915B028823F9F06091490B70914A0BDA
:10A9E00080914B0B90914C0B25E030E040E050E023
:10A9F0000E9485DF213031054105510529F4812F61
:10AA000066EA71E04EE304C0812F66EA71E040E23D
:10AA10002EE70E94C32E8091410B82FFE3C060911C
:10AA2000490B70914A0B80914B0B90914C0B25E098
:10AA300030E040E050E00E9485DF213031054105E3
:10AA4000510509F0CFC082E080935B020FB6F89405
:10AA500080914C1190914D11A0914E11B0914F11D8
:10AA60000FBE8C509E4FAF4FBF4F8093430B9093C0
:10AA7000440BA093450BB093460B88EF94E4A6C219
:10AA800080915B028823F9F06091490B70914A0B29
:10AA900080914B0B90914C0B25E030E040E050E072
:10AAA0000E9485DF213031054105510529F4812FB0
:10AAB0006EE971E04EE304C0812F6EE971E040E27F
:10AAC0002EE70E94C32E8091410B82FF8BC06091C4
:10AAD000490B70914A0B80914B0B90914C0B25E0E8
:10AAE00030E040E050E00E9485DF21303105410533
:10AAF000510509F077C082E080935B020FB6F894AD
:10AB000080914C1190914D11A0914E11B0914F1127
:10AB10000FBE8C509E4FAF4FBF4F8093430B90930F
:10AB2000440BA093450BB093460B8DE191E74EC2C9
:10AB3000023009F057C080915B028823F9F06091E0
:10AB4000490B70914A0B80914B0B90914C0B25E077
:10AB500030E040E050E00E9485DF223031054105C1
:10AB6000510529F4812F66E971E04EE304C0812F7D
:10AB700066E971E040E22EE70E94C32E8091410B0E
:10AB800082FF30C06091490B70914A0B80914B0B52
:10AB900090914C0B25E030E040E050E00E9485DFD2
:10ABA0002230310541055105E9F482E080935B02D2
:10ABB0000FB6F89480914C1190914D11A0914E11C7
:10ABC000B0914F110FBE8C509E4FAF4FBF4F80932F
:10ABD000430B9093440BA093450BB093460B8DEC25
:10ABE0009EE5F4C180917F0B882309F495C1809183
:10ABF000400D882309F413C180917E0B882309F44A
:10AC00005AC0033009F0B1C080915B028823F9F08B
:10AC10006091490B70914A0B80914B0B90914C0BBA
:10AC200025E030E040E050E00E9485DF2330310530
:10AC30004105510529F4812F6AE871E04EE304C013
:10AC4000812F6AE871E040E220E20E94C32E8091E9
:10AC5000410B82FF24C26091490B70914A0B809195
:10AC60004B0B90914C0B25E030E040E050E00E940F
:10AC700085DF233031054105510509F010C282E01E
:10AC800080935B020FB6F89480914C1190914D1116
:10AC9000A0914E11B0914F110FBE8C509E4FAF4FEF
:10ACA000BF4F8093430B9093440BA093450BB093FD
:10ACB000460BF0DD30C2033009F057C080915B02D3
:10ACC0008823F9F06091490B70914A0B80914B0BEE
:10ACD00090914C0B25E030E040E050E00E9485DF91
:10ACE000233031054105510529F4812F6DE771E0CD
:10ACF0004EE304C0812F6DE771E040E220E20E9444
:10AD0000C32E8091410B82FFCAC16091490B7091A3
:10AD10004A0B80914B0B90914C0B25E030E040E0CA
:10AD200050E00E9485DF233031054105510509F0CF
:10AD3000B6C182E080935B020FB6F89480914C110B
:10AD400090914D11A0914E11B0914F110FBE8C50AA
:10AD50009E4FAF4FBF4F8093430B9093440BA093F4
:10AD6000450BB093460B92DDD6C1043009F097C174
:10AD700080915B028823F9F06091490B70914A0B36
:10AD800080914B0B90914C0B25E030E040E050E07F
:10AD90000E9485DF243031054105510529F4812FBA
:10ADA00062E771E04EE304C0812F62E771E040E2A8
:10ADB00020E20E94C32E8091410B82FF70C16091FE
:10ADC000490B70914A0B80914B0B90914C0B25E0F5
:10ADD00030E040E050E00E9485DF2430310541053D
:10ADE000510509F05CC182E080935B020FB6F894D4
:10ADF00080914C1190914D11A0914E11B0914F1135
:10AE00000FBE8C509E4FAF4FBF4F8093430B90931C
:10AE1000440BA093450BB093460B03DD7CC103307C
:10AE200001F580915B02882309F49CC06091490B75
:10AE300070914A0B80914B0B90914C0B25E030E0C8
:10AE400040E050E00E9485DF233031054105510587
:10AE500021F4812F64E671E07CC0812F64E671E00B
:10AE60007DC0043009F01BC180915B028823F9F09A
:10AE70006091490B70914A0B80914B0B90914C0B58
:10AE800025E030E040E050E00E9485DF24303105CD
:10AE90004105510529F4812F65E571E04EE304C0B9
:10AEA000812F65E571E040E220E20E94C32E80918F
:10AEB000410B82FFF4C06091490B70914A0B809165
:10AEC0004B0B90914C0B25E030E040E050E00E94AD
:10AED00085DF243031054105510509F0E0C082E0ED
:10AEE00080935B020FB6F89480914C1190914D11B4
:10AEF000A0914E11B0914F110FBE8C509E4FAF4F8D
:10AF0000BF4F8093430B9093440BA093450BB0939A
:10AF1000460B81E591E0C0C0033009F064C0809128
:10AF20005B028823F9F06091490B70914A0B809184
:10AF30004B0B90914C0B25E030E040E050E00E943C
:10AF400085DF233031054105510529F4812F69E45E
:10AF500071E04EE304C0812F69E471E040E22EE726
:10AF60000E94C32E8091410B82FF99C06091490BD2
:10AF700070914A0B80914B0B90914C0B25E030E087
:10AF800040E050E00E9485DF233031054105510546
:10AF900009F085C082E080935B020FB6F89480913F
:10AFA0004C1190914D11A0914E11B0914F110FBEC7
:10AFB0008C509E4FAF4FBF4F8093430B9093440BE9
:10AFC000A093450BB093460B86E890E590935A0208
:10AFD000809359021092490B10924A0B10924B0B1E
:10AFE00010924C0B98C0043009F059C080915B025C
:10AFF0008823F9F06091490B70914A0B80914B0BBB
:10B0000090914C0B25E030E040E050E00E9485DF5D
:10B01000243031054105510529F4812F6BE371E09E
:10B020004EE304C0812F6BE371E040E220E20E9416
:10B03000C32E8091410B82FF32C06091490B709109
:10B040004A0B80914B0B90914C0B25E030E040E097
:10B0500050E00E9485DF2430310541055105F9F4A7
:10B0600082E080935B020FB6F89480914C1190912E
:10B070004D11A0914E11B0914F110FBE8C509E4FAB
:10B08000AF4FBF4F8093430B9093440BA093450B5E
:10B09000B093460B87E391E00E94FE983CC08091FC
:10B0A000490B90914A0BA0914B0BB0914C0B4997D7
:10B0B000A105B10540F0C092490BD0924A0BE09235
:10B0C0004B0BF0924C0B6091490B70914A0B8091A5
:10B0D0004B0B90914C0B25E030E040E050E00E949B
:10B0E00085DF422F8091420B90E0039630E082177B
:10B0F000930744F443504093420BB0925B02042FF9
:10B1000001501FEF1F5F143030F40F5F09CC013086
:10B1100009F00ECDB5CC1F910F91FF90EF90DF900D
:10B12000CF90BF9008957F928F929F92AF92BF92DF
:10B13000CF92DF92EF92FF920F931F938091490B72
:10B1400090914A0BA0914B0BB0914C0B81509048C1
:10B15000A040B04040F01092490B10924A0B109260
:10B160004B0B10924C0B6091490B70914A0B8091E4
:10B170004B0B90914C0B25E030E040E050E00E94FA
:10B1800085DF79018A018091420B90E0A0E0B0E078
:10B19000E816F9060A071B0710F42093420BC0902B
:10B1A000420BDD2428E1822E912CA12CB12C772496
:10B1B0007394CC2009F056C080915B028823C1F0C3
:10B1C0008091490B90914A0BA0914B0BB0914C0B85
:10B1D0000597A105B10528F48D2D6AE774E043E0D9
:10B1E00004C08D2D6AE774E040E223E00E94C32E84
:10B1F0008091410B82FF6EC28091490B90914A0B66
:10B20000A0914B0BB0914C0B0597A105B10508F02F
:10B2100061C282E080935B020FB6F89480914C117A
:10B2200090914D11A0914E11B0914F110FBE8C50C5
:10B230009E4FAF4FBF4F8093430B9093440BA0930F
:10B24000450BB093460B87EC91E690935A0280939E
:10B2500059021092490B10924A0B10924B0B10920C
:10B260004C0B72C281E0C81609F097C080915B0256
:10B27000882341F16091490B70914A0B80914B0BEF
:10B2800090914C0B25E030E040E050E00E9485DFDB
:10B29000213031054105510551F48AE29BE00E94BD
:10B2A0006F2C9C018D2D60E774E04EE309C08AE2AB
:10B2B0009BE00E946F2C9C018D2D60E774E040E2C2
:10B2C0000E94A0368091410B82FF04C2E090490B9E
:10B2D000F0904A0B00914B0B10914C0BC801B70139
:10B2E00025E030E040E050E00E9485DF213031056C
:10B2F0004105510509F0EEC10FB6F89480914C114B
:10B3000090914D11A0914E11B0914F110FBE8C50E4
:10B310009E4FAF4FBF4F8093430B9093440BA0932E
:10B32000450BB093460B8091590290915A0290932D
:10B33000530B8093520BF092550BE092540B82E02A
:10B3400080935B0281E89FE490935A0280935902B4
:10B3500086E694E09093570B8093560B8AE29BE02D
:10B360009093590B8093580B10925A0B10925B0BD1
:10B3700010925C0B10925D0B8FEF90E0A0E0B0E0BC
:10B3800080935E0B90935F0BA093600BB093610B67
:10B3900080912A0B90912B0B35C122E0C21609F047
:10B3A00097C080915B02882341F16091490B7091B5
:10B3B0004A0B80914B0B90914C0B25E030E040E024
:10B3C00050E00E9485DF223031054105510551F4DE
:10B3D00086E29BE00E946F2C9C018D2D6FE574E04E
:10B3E0004EE309C086E29BE00E946F2C9C018D2DEC
:10B3F0006FE574E040E20E94A0368091410B82FF2D
:10B4000069C1E090490BF0904A0B00914B0B1091F1
:10B410004C0BC801B70125E030E040E050E00E944D
:10B4200085DF223031054105510509F053C10FB6C2
:10B43000F89480914C1190914D11A0914E11B091C2
:10B440004F110FBE8C509E4FAF4FBF4F8093430B99
:10B450009093440BA093450BB093460B80915902F7
:10B4600090915A029093530B8093520BF092550B8C
:10B47000E092540B82E080935B0281E89FE490931A
:10B480005A028093590288E594E09093570B809379
:10B49000560B86E29BE09093590B8093580B1092C9
:10B4A0005A0B10925B0B10925C0B10925D0B84E0B8
:10B4B00091E0A0E0B0E080935E0B90935F0BA093CF
:10B4C000600BB093610B8091260B9091270B9AC073
:10B4D00083E0C81609F0A3C080915B02882341F184
:10B4E0006091490B70914A0B80914B0B90914C0BE2
:10B4F00025E030E040E050E00E9485DF2330310558
:10B500004105510551F488E29BE00E946F2C9C019B
:10B510008D2D64E574E04EE309C088E29BE00E9453
:10B520006F2C9C018D2D64E574E040E20E94A036F2
:10B530008091410B82FFCEC0E090490BF0904A0B06
:10B5400000914B0B10914C0BC801B70125E030E086
:10B5500040E050E00E9485DF233031054105510570
:10B5600009F0B8C00FB6F89480914C1190914D112C
:10B57000A0914E11B0914F110FBE8C509E4FAF4F06
:10B58000BF4F8093430B9093440BA093450BB09314
:10B59000460B8091590290915A029093530B8093DD
:10B5A000520BF092550BE092540B82E080935B02B9
:10B5B00081E89FE490935A028093590280E594E0D9
:10B5C0009093570B8093560B88E29BE09093590B16
:10B5D0008093580B10925A0B10925B0B10925C0BDD
:10B5E00010925D0B87E890E0A0E0B0E080935E0BE6
:10B5F00090935F0BA093600BB093610B8091280B2D
:10B600009091290BAA2797FDA095BA2F8093490BFB
:10B6100090934A0BA0934B0BB0934C0B95C024E036
:10B62000C21609F057C080915B028823F9F060913F
:10B63000490B70914A0B80914B0B90914C0B25E07C
:10B6400030E040E050E00E9485DF243031054105C4
:10B65000510529F48D2D63E474E04EE304C08D2D73
:10B6600063E474E040E220E20E94C32E8091410B2B
:10B6700082FF30C06091490B70914A0B80914B0B57
:10B6800090914C0B25E030E040E050E00E9485DFD7
:10B690002430310541055105E9F482E080935B02D5
:10B6A0000FB6F89480914C1190914D11A0914E11CC
:10B6B000B0914F110FBE8C509E4FAF4FBF4F809334
:10B6C000430B9093440BA093450BB093460B0E9401
:10B6D00006B93AC08091490B90914A0BA0914B0B4F
:10B6E000B0914C0B4997A105B10540F08092490BF0
:10B6F00090924A0BA0924B0BB0924C0B6091490B6D
:10B7000070914A0B80914B0B90914C0B25E030E0EF
:10B7100040E050E00E9485DF422F8091420B90E094
:10B72000039630E0821793074CF443504093420B4A
:10B7300070925B02C42ECA94DD24DA94D39483E021
:10B740008D1510F0C39435CD1F910F91FF90EF90A0
:10B75000DF90CF90BF90AF909F908F907F90089593
:10B760007F928F929F92AF92BF92CF92DF92EF9291
:10B77000FF920F931F938091490B90914A0BA091D8
:10B780004B0BB0914C0B81509048A040B04040F022
:10B790001092490B10924A0B10924B0B10924C0BCB
:10B7A0006091490B70914A0B80914B0B90914C0B1F
:10B7B00025E030E040E050E00E9485DF79018A0119
:10B7C0008091420B90E0A0E0B0E0E816F9060A078D
:10B7D0001B0710F42093420BC090420BDD2438E18C
:10B7E000832E912CA12CB12C77247394CC2009F0BA
:10B7F00056C080915B028823C1F08091490B9091E3
:10B800004A0BA0914B0BB0914C0B0597A105B105CC
:10B8100028F48D2D6DEB74E043E004C08D2D6DEBAD
:10B8200074E040E223E00E94C32E8091410B82FF2E
:10B830006EC28091490B90914A0BA0914B0BB09135
:10B840004C0B0597A105B10508F061C282E0809319
:10B850005B020FB6F89480914C1190914D11A0911C
:10B860004E11B0914F110FBE8C509E4FAF4FBF4F36
:10B870008093430B9093440BA093450BB093460BDE
:10B8800087EC91E690935A02809359021092490BEB
:10B8900010924A0B10924B0B10924C0B72C281E02B
:10B8A000C81609F097C080915B02882341F160912E
:10B8B000490B70914A0B80914B0B90914C0B25E0FA
:10B8C00030E040E050E00E9485DF21303105410545
:10B8D000510551F484E29BE00E946F2C9C018D2D58
:10B8E00063EB74E04EE309C084E29BE00E946F2C9E
:10B8F0009C018D2D63EB74E040E20E94A0368091A4
:10B90000410B82FF04C2E090490BF0904A0B00917A
:10B910004B0B10914C0BC801B70125E030E040E023
:10B9200050E00E9485DF213031054105510509F0C5
:10B93000EEC10FB6F89480914C1190914D11A091E9
:10B940004E11B0914F110FBE8C509E4FAF4FBF4F55
:10B950008093430B9093440BA093450BB093460BFD
:10B960008091590290915A029093530B8093520BFD
:10B97000F092550BE092540B82E080935B0281E8D9
:10B980009FE490935A028093590289EA94E090933D
:10B99000570B8093560B84E29BE09093590B809356
:10B9A000580B10925A0B10925B0B10925C0B10927A
:10B9B0005D0B8FEF90E0A0E0B0E080935E0B909382
:10B9C0005F0BA093600BB093610B8091240B90915F
:10B9D000250B35C122E0C21609F097C080915B02A9
:10B9E000882341F16091490B70914A0B80914B0B78
:10B9F00090914C0B25E030E040E050E00E9485DF64
:10BA0000223031054105510551F480E29BE00E944E
:10BA10006F2C9C018D2D62EA74E04EE309C080E238
:10BA20009BE00E946F2C9C018D2D62EA74E040E245
:10BA30000E94A0368091410B82FF69C1E090490BC2
:10BA4000F0904A0B00914B0B10914C0BC801B701C1
:10BA500025E030E040E050E00E9485DF22303105F3
:10BA60004105510509F053C10FB6F89480914C116E
:10BA700090914D11A0914E11B0914F110FBE8C506D
:10BA80009E4FAF4FBF4F8093430B9093440BA093B7
:10BA9000450BB093460B8091590290915A029093B6
:10BAA000530B8093520BF092550BE092540B82E0B3
:10BAB00080935B0281E89FE490935A02809359023D
:10BAC0008BE994E09093570B8093560B80E29BE0B8
:10BAD0009093590B8093580B10925A0B10925B0B5A
:10BAE00010925C0B10925D0B84E091E0A0E0B0E05E
:10BAF00080935E0B90935F0BA093600BB093610BF0
:10BB00008091200B9091210B9AC083E0C81609F018
:10BB1000A3C080915B02882341F16091490B709131
:10BB20004A0B80914B0B90914C0B25E030E040E0AC
:10BB300050E00E9485DF233031054105510551F465
:10BB400082E29BE00E946F2C9C018D2D67E974E0DE
:10BB50004EE309C082E29BE00E946F2C9C018D2D78
:10BB600067E974E040E20E94A0368091410B82FFB9
:10BB7000CEC0E090490BF0904A0B00914B0B109116
:10BB80004C0BC801B70125E030E040E050E00E94D6
:10BB900085DF233031054105510509F0B8C00FB6E6
:10BBA000F89480914C1190914D11A0914E11B0914B
:10BBB0004F110FBE8C509E4FAF4FBF4F8093430B22
:10BBC0009093440BA093450BB093460B8091590280
:10BBD00090915A029093530B8093520BF092550B15
:10BBE000E092540B82E080935B0281E89FE49093A3
:10BBF0005A028093590283E994E09093570B809303
:10BC0000560B82E29BE09093590B8093580B109255
:10BC10005A0B10925B0B10925C0B10925D0B87E835
:10BC200090E0A0E0B0E080935E0B90935F0BA09358
:10BC3000600BB093610B8091220B9091230BAA278C
:10BC400097FDA095BA2F8093490B90934A0BA09330
:10BC50004B0BB0934C0B95C024E0C21609F057C0B3
:10BC600080915B028823F9F06091490B70914A0B37
:10BC700080914B0B90914C0B25E030E040E050E080
:10BC80000E9485DF243031054105510529F48D2DB1
:10BC900066E874E04EE304C08D2D66E874E040E28F
:10BCA00020E20E94C32E8091410B82FF30C0609140
:10BCB000490B70914A0B80914B0B90914C0B25E0F6
:10BCC00030E040E050E00E9485DF2430310541053E
:10BCD0005105E9F482E080935B020FB6F8948091FD
:10BCE0004C1190914D11A0914E11B0914F110FBE7A
:10BCF0008C509E4FAF4FBF4F8093430B9093440B9C
:10BD0000A093450BB093460B0E9406B93AC08091B0
:10BD1000490B90914A0BA0914B0BB0914C0B49975A
:10BD2000A105B10540F08092490B90924A0BA09278
:10BD30004B0BB0924C0B6091490B70914A0B809168
:10BD40004B0B90914C0B25E030E040E050E00E941E
:10BD500085DF422F8091420B90E0039630E08217FE
:10BD600093074CF443504093420B70925B02C42EF5
:10BD7000CA94DD24DA94D39483E08D1510F0C39433
:10BD800035CD1F910F91FF90EF90DF90CF90BF9036
:10BD9000AF909F908F907F900895BF92CF92DF9247
:10BDA000EF92FF920F931F938091490B90914A0B52
:10BDB000A0914B0BB0914C0B81509048A040B040EB
:10BDC00040F01092490B10924A0B10924B0B1092BC
:10BDD0004C0B6091490B70914A0B80914B0B9091E9
:10BDE0004C0B25E030E040E050E00E9485DF790117
:10BDF0008A018091420B90E0A0E0B0E0E816F906DD
:10BE00000A071B0710F42093420B0091420B10E02D
:10BE10004DE1C42ED12CE12CF12CBB24B394002392
:10BE200009F04AC080915B028823C1F08091490BE0
:10BE300090914A0BA0914B0BB0914C0B0597A1052B
:10BE4000B10528F4812F6DE172E043E004C0812F39
:10BE50006DE172E040E223E00E94C32E8091410B2D
:10BE600082FFFCC18091490B90914A0BA0914B0B32
:10BE7000B0914C0B0597A105B10508F0EFC182E028
:10BE800080935B020FB6F89480914C1190914D1104
:10BE9000A0914E11B0914F110FBE8C509E4FAF4FDD
:10BEA000BF4F8093430B9093440BA093450BB093EB
:10BEB000460B8EE494E55AC0013009F064C08091CD
:10BEC0005B028823F9F06091490B70914A0B8091D5
:10BED0004B0B90914C0B25E030E040E050E00E948D
:10BEE00085DF213031054105510529F4812F61E1BC
:10BEF00072E04EE304C0812F61E172E040E22EE780
:10BF00000E94C32E8091410B82FFA8C16091490B12
:10BF100070914A0B80914B0B90914C0B25E030E0D7
:10BF200040E050E00E9485DF213031054105510598
:10BF300009F094C182E080935B020FB6F89480917F
:10BF40004C1190914D11A0914E11B0914F110FBE17
:10BF50008C509E4FAF4FBF4F8093430B9093440B39
:10BF6000A093450BB093460B87EC91E690935A0251
:10BF7000809359021092490B10924A0B10924B0B6E
:10BF800010924C0BA3C1023009F058C080915B02A3
:10BF90008823F9F06091490B70914A0B80914B0B0B
:10BFA00090914C0B25E030E040E050E00E9485DFAE
:10BFB000223031054105510529F4812F6AE072E0F4
:10BFC0004EE304C0812F6AE072E040E22EE70E9457
:10BFD000C32E8091410B82FF41C16091490B70914A
:10BFE0004A0B80914B0B90914C0B25E030E040E0E8
:10BFF00050E00E9485DF223031054105510509F0EE
:10C000002DC182E080935B020FB6F89480914C11B1
:10C0100090914D11A0914E11B0914F110FBE8C50C7
:10C020009E4FAF4FBF4F8093430B9093440BA09311
:10C03000450BB093460B8EEF96E398CF033009F093
:10C0400058C080915B028823F9F06091490B709190
:10C050004A0B80914B0B90914C0B25E030E040E077
:10C0600050E00E9485DF233031054105510529F458
:10C07000812F6DEF71E04EE304C0812F6DEF71E011
:10C0800040E220E20E94C32E8091410B82FFE6C075
:10C090006091490B70914A0B80914B0B90914C0B26
:10C0A00025E030E040E050E00E9485DF233031059C
:10C0B0004105510509F0D2C082E080935B020FB6C2
:10C0C000F89480914C1190914D11A0914E11B09126
:10C0D0004F110FBE8C509E4FAF4FBF4F8093430BFD
:10C0E0009093440BA093450BB093460B0E9406B966
:10C0F000EDC0043009F058C080915B028823F9F04C
:10C100006091490B70914A0B80914B0B90914C0BB5
:10C1100025E030E040E050E00E9485DF243031052A
:10C120004105510529F4812F61EF71E04EE304C010
:10C13000812F61EF71E040E220E20E94C32E8091E6
:10C14000410B82FF8BC06091490B70914A0B80912B
:10C150004B0B90914C0B25E030E040E050E00E940A
:10C1600085DF243031054105510509F077C082E0B3
:10C1700080935B020FB6F89480914C1190914D1111
:10C18000A0914E11B0914F110FBE8C509E4FAF4FEA
:10C19000BF4F8093430B9093440BA093450BB093F8
:10C1A000460B0E942DC192C0053009F057C0809106
:10C1B0005B028823F9F06091490B70914A0B8091E2
:10C1C0004B0B90914C0B25E030E040E050E00E949A
:10C1D00085DF253031054105510529F4812F60EEB9
:10C1E00071E04EE304C0812F60EE71E040E220E296
:10C1F0000E94C32E8091410B82FF30C06091490B99
:10C2000070914A0B80914B0B90914C0B25E030E0E4
:10C2100040E050E00E9485DF2530310541055105A1
:10C22000E9F482E080935B020FB6F89480914C11A0
:10C2300090914D11A0914E11B0914F110FBE8C50A5
:10C240009E4FAF4FBF4F8093430B9093440BA093EF
:10C25000450BB093460B0E94A0BB38C08091490BA0
:10C2600090914A0BA0914B0BB0914C0B4E97A105AE
:10C27000B10540F0C092490BD0924A0BE0924B0BB3
:10C28000F0924C0B6091490B70914A0B80914B0BD3
:10C2900090914C0B25E030E040E050E00E9485DFBB
:10C2A000422F8091420B90E0039630E08217930773
:10C2B00044F443504093420BB0925B02042F015070
:10C2C0001FEF1F5F143010F40F5FA9CD1F910F9166
:10C2D000FF90EF90DF90CF90BF900895DF92EF92A4
:10C2E000FF920F931F93CF93DF93182FEB01D42E60
:10C2F0007901C9010E94711001E1081B8DE29BE0E8
:10C3000060E0412F0E9477D1E0912D0BF0912E0B30
:10C310000190F081E02D8DE29BE06D2D0995FE01ED
:10C320006491662379F0002369F0E0912D0BF09180
:10C330002E0B0190F081E02D8DE29BE00995219676
:10C340000150EDCFE0912D0BF0912E0B0190F0817B
:10C35000E02D8DE29BE06AE309950CC0E0912D0B86
:10C36000F0912E0B0190F081E02D8DE29BE060E2D8
:10C3700009950150002391F7C7010E948733DF918F
:10C38000CF911F910F91FF90EF90DF900895EF9262
:10C39000FF920F931F936091950270919602809186
:10C3A0009702909198020E94F69A6093640B7093A2
:10C3B000650B8093660B9093670B60919902709167
:10C3C0009A0280919B0290919C020E94029B609332
:10C3D000680B7093690B80936A0B90936B0B809141
:10C3E000490B90914A0BA0914B0BB0914C0B815093
:10C3F0009048A040B04040F01092490B10924A0B78
:10C4000010924B0B10924C0B6091490B70914A0BA0
:10C4100080914B0B90914C0B25E030E040E050E0D8
:10C420000E9485DF79018A018091420B90E0A0E0B3
:10C43000B0E0E816F9060A071B0710F42093420B38
:10C440000091420B10E0002309F04EC080915B0286
:10C450008823C1F08091490B90914A0BA0914B0B1E
:10C46000B0914C0B0597A105B10528F4812F6BE322
:10C4700074E043E004C0812F6BE374E040E223E00A
:10C480000E94C32E8091410B82FD02C00C94686B08
:10C490008091490B90914A0BA0914B0BB0914C0BA2
:10C4A0000597A105B10510F00C94686B82E08093AC
:10C4B0005B020FB6F89480914C1190914D11A091B0
:10C4C0004E11B0914F110FBE8C509E4FAF4FBF4FCA
:10C4D0008093430B9093440BA093450BB093460B72
:10C4E0008DEC9EE50C945B6B013009F09CC0809153
:10C4F0005B02882341F16091490B70914A0B809156
:10C500004B0B90914C0B25E030E040E050E00E9456
:10C5100085DF213031054105510551F483E99FE064
:10C520000E946F2C9C01812F64E374E04EE309C0EC
:10C5300083E99FE00E946F2C9C01812F64E374E0EB
:10C5400040E20E94A0368091410B82FD02C00C9413
:10C55000686B6091490B70914A0B80914B0B9091E5
:10C560004C0B25E030E040E050E00E9485DF2130B8
:10C5700031054105510511F00C94686B0FB6F89424
:10C5800080914C1190914D11A0914E11B0914F118D
:10C590000FBE8C509E4FAF4FBF4F8093430B909375
:10C5A000440BA093450BB093460B80915902909198
:10C5B0005A029093530B8093520B8091490B9091A8
:10C5C0004A0B9093550B8093540B82E080935B024F
:10C5D00081E89FE490935A02809359028DE294E09F
:10C5E0009093570B8093560B83E99FE09093590BE0
:10C5F0008093580B10925A0B10925B0B10925C0BAD
:10C6000010925D0B84E091E0A0E0B0E080935E0BBF
:10C6100090935F0BA093600BB093610B8091930F8D
:10C620009091940F9EC0023009F0A8C080915B02E7
:10C63000882341F16091490B70914A0B80914B0B1B
:10C6400090914C0B25E030E040E050E00E9485DF07
:10C65000223031054105510551F485E99FE00E94E2
:10C660006F2C9C01812F65E274E04EE309C085E9DF
:10C670009FE00E946F2C9C01812F65E274E040E2F4
:10C680000E94A0368091410B82FD02C00C94686B21
:10C690006091490B70914A0B80914B0B90914C0B20
:10C6A00025E030E040E050E00E9485DF2230310597
:10C6B0004105510511F00C94686B0FB6F894809108
:10C6C0004C1190914D11A0914E11B0914F110FBE90
:10C6D0008C509E4FAF4FBF4F8093430B9093440BB2
:10C6E000A093450BB093460B8091590290915A024A
:10C6F0009093530B8093520B8091490B90914A0B6E
:10C700009093550B8093540B82E080935B0281E8F9
:10C710009FE490935A02809359028DE194E09093A4
:10C72000570B8093560B85E99FE09093590B8093AC
:10C73000580B10925A0B10925B0B10925C0B1092DC
:10C740005D0B84E091E0A0E0B0E080935E0B9093FD
:10C750005F0BA093600BB093610B8091950F90914C
:10C76000960FAA2797FDA095BA2F8093490B909317
:10C770004A0BA0934B0BB0934C0BE9C7033009F065
:10C7800099C080915B02882341F16091490B7091BF
:10C790004A0B80914B0B90914C0B25E030E040E030
:10C7A00050E00E9485DF233031054105510551F4E9
:10C7B00087E99FE00E946F2C9C01812F65E174E066
:10C7C0004EE309C087E99FE00E946F2C9C01812FF6
:10C7D00065E174E040E20E94A0368091410B82FF47
:10C7E00077C76091490B70914A0B80914B0B9091E8
:10C7F0004C0B25E030E040E050E00E9485DF233024
:10C8000031054105510509F063C70FB6F8948091D1
:10C810004C1190914D11A0914E11B0914F110FBE3E
:10C820008C509E4FAF4FBF4F8093430B9093440B60
:10C83000A093450BB093460B8091590290915A02F8
:10C840009093530B8093520B8091490B90914A0B1C
:10C850009093550B8093540B82E080935B0281E8A8
:10C860009FE490935A02809359028DE094E0909354
:10C87000570B8093560B87E99FE09093590B809359
:10C88000580B10925A0B10925B0B10925C0B10928B
:10C890005D0B84E091E0A0E0B0E080935E0B9093AC
:10C8A0005F0BA093600BB093610B8091970F9091F9
:10C8B000980F57CF043009F099C080915B0288230C
:10C8C00041F16091490B70914A0B80914B0B909113
:10C8D0004C0B25E030E040E050E00E9485DF243042
:10C8E00031054105510551F489E99FE00E946F2C03
:10C8F0009C01812F69E074E04EE309C089E99FE063
:10C900000E946F2C9C01812F69E074E040E20E943C
:10C91000A0368091410B82FFDBC66091490B70917C
:10C920004A0B80914B0B90914C0B25E030E040E09E
:10C9300050E00E9485DF243031054105510509F0A2
:10C94000C7C60FB6F89480914C1190914D11A091EB
:10C950004E11B0914F110FBE8C509E4FAF4FBF4F35
:10C960008093430B9093440BA093450BB093460BDD
:10C970008091590290915A029093530B8093520BDD
:10C980008091490B90914A0B9093550B8093540BD7
:10C9900082E080935B0281E89FE490935A02809347
:10C9A000590285E094E09093570B8093560B89E9E8
:10C9B0009FE09093590B8093580B10925A0B109252
:10C9C0005B0B10925C0B10925D0B87E890E0A0E08F
:10C9D000B0E080935E0B90935F0BA093600BB093DD
:10C9E000610B8091990F90919A0FBBCE053009F0A1
:10C9F00099C080915B02882341F16091490B70914D
:10CA00004A0B80914B0B90914C0B25E030E040E0BD
:10CA100050E00E9485DF253031054105510551F474
:10CA200082EB9DE00E946F2C9C01812F6BEF73E0E5
:10CA30004EE309C082EB9DE00E946F2C9C01812F88
:10CA40006BEF73E040E20E94A0368091410B82FFC1
:10CA50003FC66091490B70914A0B80914B0B9091AE
:10CA60004C0B25E030E040E050E00E9485DF2530AF
:10CA700031054105510509F02BC60FB6F894809198
:10CA80004C1190914D11A0914E11B0914F110FBECC
:10CA90008C509E4FAF4FBF4F8093430B9093440BEE
:10CAA000A093450BB093460B8091590290915A0286
:10CAB0009093530B8093520B8091490B90914A0BAA
:10CAC0009093550B8093540B82E080935B0281E836
:10CAD0009FE490935A028093590281EF93E09093E0
:10CAE000570B8093560B82EB9DE09093590B8093EC
:10CAF000580B10925A0B10925B0B10925C0B109219
:10CB00005D0B8FEF90E0A0E0B0E080935E0B909320
:10CB10005F0BA093600BB093610B8091B20D90916D
:10CB2000B30D1FCE063009F06AC080915B028823E6
:10CB300069F16091490B70914A0B80914B0B909178
:10CB40004C0B25E030E040E050E00E9485DF809112
:10CB50003506263031054105510561F4882319F465
:10CB600020EE33E002C024EE33E0812F68EE73E064
:10CB70004EE30BC0882319F428ED33E002C02CEDFE
:10CB800033E0812F68EE73E040E2A8DB8091410B37
:10CB900082FF9EC56091490B70914A0B80914B0BAF
:10CBA00090914C0B25E030E040E050E00E9485DFA2
:10CBB000263031054105510509F08AC582E0809390
:10CBC0005B020FB6F89480914C1190914D11A09199
:10CBD0004E11B0914F110FBE8C509E4FAF4FBF4FB3
:10CBE0008093430B9093440BA093450BB093460B5B
:10CBF0008091350691E0892780933506A8C50730D6
:10CC000009F09DC080915B02882341F16091490B3E
:10CC100070914A0B80914B0B90914C0B25E030E0CA
:10CC200040E050E00E9485DF273031054105510585
:10CC300051F488E392E00E94A42C9C01812F61EDC5
:10CC400073E04EE309C088E392E00E94A42C9C01AB
:10CC5000812F61ED73E040E20E94A0368091410B8C
:10CC600082FF36C56091490B70914A0B80914B0B46
:10CC700090914C0B25E030E040E050E00E9485DFD1
:10CC8000273031054105510509F022C50FB6F8944A
:10CC900080914C1190914D11A0914E11B0914F1176
:10CCA0000FBE8C509E4FAF4FBF4F8093430B90935E
:10CCB000440BA093450BB093460B80915902909181
:10CCC0005A029093530B8093520B8091490B909191
:10CCD0004A0B9093550B8093540B82E080935B0238
:10CCE00082ED9EE490935A02809359028AEC93E07D
:10CCF0009093570B8093560B88E392E09093590BD7
:10CD00008093580B10925A0B10925B0B10925C0B95
:10CD100010925D0B84E091E0A0E0B0E080935E0BA8
:10CD200090935F0BA093600BB093610B60913802FE
:10CD30007091390280913A0290913B02FDC3083014
:10CD400009F09DC080915B02882341F16091490BFD
:10CD500070914A0B80914B0B90914C0B25E030E089
:10CD600040E050E00E9485DF283031054105510543
:10CD700051F484E392E00E94A42C9C01812F63EC87
:10CD800073E04EE309C084E392E00E94A42C9C016E
:10CD9000812F63EC73E040E20E94A0368091410B4A
:10CDA00082FF96C46091490B70914A0B80914B0BA6
:10CDB00090914C0B25E030E040E050E00E9485DF90
:10CDC000283031054105510509F082C40FB6F894A9
:10CDD00080914C1190914D11A0914E11B0914F1135
:10CDE0000FBE8C509E4FAF4FBF4F8093430B90931D
:10CDF000440BA093450BB093460B80915902909140
:10CE00005A029093530B8093520B8091490B90914F
:10CE10004A0B9093550B8093540B82E080935B02F6
:10CE200082ED9EE490935A02809359028CEB93E03A
:10CE30009093570B8093560B84E392E09093590B99
:10CE40008093580B10925A0B10925B0B10925C0B54
:10CE500010925D0B84E091E0A0E0B0E080935E0B67
:10CE600090935F0BA093600BB093610B60913402C1
:10CE70007091350280913602909137025DC309307E
:10CE800009F09DC080915B02882341F16091490BBC
:10CE900070914A0B80914B0B90914C0B25E030E048
:10CEA00040E050E00E9485DF293031054105510501
:10CEB00051F48CE392E00E94EB2B9C01812F64EBF8
:10CEC00073E04EE309C08CE392E00E94EB2B9C01DF
:10CED000812F64EB73E040E20E94A0368091410B09
:10CEE00082FFF6C36091490B70914A0B80914B0B06
:10CEF00090914C0B25E030E040E050E00E9485DF4F
:10CF0000293031054105510509F0E2C30FB6F89407
:10CF100080914C1190914D11A0914E11B0914F11F3
:10CF20000FBE8C509E4FAF4FBF4F8093430B9093DB
:10CF3000440BA093450BB093460B809159029091FE
:10CF40005A029093530B8093520B8091490B90910E
:10CF50004A0B9093550B8093540B82E080935B02B5
:10CF600087E19EE490935A02809359028CEA93E001
:10CF70009093570B8093560B8CE392E09093590B50
:10CF80008093580B10925A0B10925B0B10925C0B13
:10CF900010925D0B84E690E0A0E0B0E080935E0B21
:10CFA00090935F0BA093600BB093610B60913C0278
:10CFB00070913D0280913E0290913F02A3C00A30E1
:10CFC00009F0A7C080915B02882341F16091490B71
:10CFD00070914A0B80914B0B90914C0B25E030E007
:10CFE00040E050E00E9485DF2A30310541055105BF
:10CFF00051F481E992E00E943C2E9C01812F66EA67
:10D0000073E04EE309C081E992E00E943C2E9C014E
:10D01000812F66EA73E040E20E94A0368091410BC6
:10D0200082FF56C36091490B70914A0B80914B0B64
:10D0300090914C0B25E030E040E050E00E9485DF0D
:10D040002A3031054105510509F042C30FB6F89465
:10D0500080914C1190914D11A0914E11B0914F11B2
:10D060000FBE8C509E4FAF4FBF4F8093430B90939A
:10D07000440BA093450BB093460B809159029091BD
:10D080005A029093530B8093520B8091490B9091CD
:10D090004A0B9093550B8093540B82E080935B0274
:10D0A00086EE9BE490935A028093590280EA93E0C3
:10D0B0009093570B8093560B81E992E09093590B14
:10D0C0008093580B84E690E0A0E0B0E080935A0B88
:10D0D00090935B0BA0935C0BB0935D0B88E59EE394
:10D0E000AFE0B0E080935E0B90935F0BA093600B7A
:10D0F000B093610B609191027091920280919302C2
:10D100009091940220E030E048EC52E40E946DDE01
:10D1100013C20B3009F0B3C080915B02882341F148
:10D120006091490B70914A0B80914B0B90914C0B85
:10D1300025E030E040E050E00E9485DF2B303105F3
:10D140004105510551F484E69BE00E943C2E9C0170
:10D15000812F6AE973E04EE309C084E69BE00E94F8
:10D160003C2E9C01812F6AE973E040E20E94A036C8
:10D170008091410B82FFACC26091490B70914A0BC8
:10D1800080914B0B90914C0B25E030E040E050E05B
:10D190000E9485DF2B3031054105510509F098C209
:10D1A0000FB6F89480914C1190914D11A0914E11B1
:10D1B000B0914F110FBE8C509E4FAF4FBF4F809319
:10D1C000430B9093440BA093450BB093460B809177
:10D1D000590290915A029093530B8093520B809175
:10D1E000490B90914A0B9093550B8093540B82E01E
:10D1F00080935B0286E29BE490935A0280935902EB
:10D2000084E993E09093570B8093560B84E69BE060
:10D210009093590B8093580B81E090E0A0E0B0E030
:10D2200080935A0B90935B0BA0935C0BB0935D0BB8
:10D2300088E59EE3AFE0B0E080935E0B90935F0BD8
:10D24000A093600BB093610B6091640B7091650BC0
:10D250008091660B9091670B20E030E048EC52E43F
:10D260000E946DDE0E9401DC6093490B70934A0BB3
:10D2700080934B0B90934C0B89ED9EE6B5C00C3020
:10D2800009F0B7C080915B02882341F16091490B9E
:10D2900070914A0B80914B0B90914C0B25E030E044
:10D2A00040E050E00E9485DF2C30310541055105FA
:10D2B00051F488E69BE00E943C2E9C01812F6EE891
:10D2C00073E04EE309C088E69BE00E943C2E9C017F
:10D2D000812F6EE873E040E20E94A0368091410BFE
:10D2E00082FFF6C16091490B70914A0B80914B0B04
:10D2F00090914C0B25E030E040E050E00E9485DF4B
:10D300002C3031054105510509F0E2C10FB6F89402
:10D3100080914C1190914D11A0914E11B0914F11EF
:10D320000FBE8C509E4FAF4FBF4F8093430B9093D7
:10D33000440BA093450BB093460B809159029091FA
:10D340005A029093530B8093520B8091490B90910A
:10D350004A0B9093550B8093540B82E080935B02B1
:10D3600086E29BE490935A028093590288E893E006
:10D370009093570B8093560B88E69BE09093590B44
:10D380008093580B84E690E0A0E0B0E080935A0BC5
:10D3900090935B0BA0935C0BB0935D0B88E59EE3D1
:10D3A000AFE0B0E080935E0B90935F0BA093600BB7
:10D3B000B093610B6091680B7091690B80916A0B5F
:10D3C00090916B0B20E030E048EC52E40E946DDE5F
:10D3D0000E9401DC6093490B70934A0B80934B0BC6
:10D3E00090934C0B85EC9EE69093630B8093620BBD
:10D3F000AEC10D3009F0ABC080915B02882341F1D2
:10D400006091490B70914A0B80914B0B90914C0BA2
:10D4100025E030E040E050E00E9485DF2D3031050E
:10D420004105510551F48DE992E00E94A42C9C0124
:10D43000812F62E873E04EE309C08DE992E00E941B
:10D44000A42C9C01812F62E873E040E20E94A03688
:10D450008091410B82FF3CC16091490B70914A0B56
:10D4600080914B0B90914C0B25E030E040E050E078
:10D470000E9485DF2D3031054105510509F028C195
:10D480000FB6F89480914C1190914D11A0914E11CE
:10D49000B0914F110FBE8C509E4FAF4FBF4F809336
:10D4A000430B9093440BA093450BB093460B809194
:10D4B000590290915A029093530B8093520B809192
:10D4C000490B90914A0B9093550B8093540B82E03B
:10D4D00080935B0282ED9EE490935A0280935902FE
:10D4E0008CE793E09093570B8093560B8DE992E075
:10D4F0009093590B8093580B81E090E0A0E0B0E04E
:10D5000080935A0B90935B0BA0935C0BB0935D0BD5
:10D5100086E097E2A0E0B0E080935E0B90935F0B13
:10D52000A093600BB093610B60919D0270919E027D
:10D5300080919F029091A0020E9401DC6093490BB0
:10D5400070934A0B80934B0B90934C0B00C10E30A1
:10D5500009F058C080915B028823F9F06091490B73
:10D5600070914A0B80914B0B90914C0B25E030E071
:10D5700040E050E00E9485DF2E3031054105510525
:10D5800029F4812F6BE673E04EE304C0812F6BE634
:10D5900073E040E22EE70E94C32E8091410B82FF90
:10D5A00097C06091490B70914A0B80914B0B909101
:10D5B0004C0B25E030E040E050E00E9485DF2E304B
:10D5C00031054105510509F083C082E080935B027B
:10D5D0000FB6F89480914C1190914D11A0914E117D
:10D5E000B0914F110FBE8C509E4FAF4FBF4F8093E5
:10D5F000430B9093440BA093450BB093460B80EBE9
:10D600009BE559C00F3009F063C080915B0288230D
:10D61000F9F06091490B70914A0B80914B0B9091FE
:10D620004C0B25E030E040E050E00E9485DF2F30D9
:10D6300031054105510529F4812F6AE573E04EE378
:10D6400004C0812F6AE573E040E22EE70E94C32EFA
:10D650008091410B82FF3CC06091490B70914A0B55
:10D6600080914B0B90914C0B25E030E040E050E076
:10D670000E9485DF2F3031054105510549F582E0D3
:10D6800080935B020FB6F89480914C1190914D11EC
:10D69000A0914E11B0914F110FBE8C509E4FAF4FC5
:10D6A000BF4F8093430B9093440BA093450BB093D3
:10D6B000460B83E998E590935A02809359021092A1
:10D6C000490B10924A0B10924B0B10924C0B3FC01F
:10D6D0008091490B90914A0BA0914B0BB0914C0B50
:10D6E00080359105A105B10560F08FE490E0A0E0E0
:10D6F000B0E08093490B90934A0BA0934B0BB093EF
:10D700004C0B6091490B70914A0B80914B0B90919F
:10D710004C0B25E030E040E050E00E9485DF422FD6
:10D720008091420B90E0039630E0821793074CF40F
:10D7300043504093420B81E080935B02042F0150E1
:10D740001FEF1F5F143018F40F5F0C9423621F91BA
:10D750000F91FF90EF900895CF92DF92EF92FF929A
:10D760000F931F932091490B30914A0B40914B0B23
:10D7700050914C0B211531054105510509F448C064
:10D78000B901882777FD8095982F0E942FDC209182
:10D790006C0B30916D0B40916E0B50916F0B0E9492
:10D7A0006DDE9B01AC0160917D0D70917E0D8091CD
:10D7B0007F0D9091800D0E94B4DA60937D0D70937F
:10D7C0007E0D80937F0D9093800D1092490B1092E7
:10D7D0004A0B10924B0B10924C0B81E79DE065E7D2
:10D7E0007DE049E75DE02DE73DE00F2EF0E0EF2E14
:10D7F000F0E0FF2EF0EA0F2FF1E41F2FF02DE1EB08
:10D80000CE2EEDE0DE2E0E94EB1E81E080935B02C7
:10D8100080915B02882349F08DE79DE00E949A2B5E
:10D82000BC018AE695E00E942E4A8091410B82FF5E
:10D8300028C082E080935B020FB6F89480914C116F
:10D8400090914D11A0914E11B0914F110FBE8C507F
:10D850009E4FAF4FBF4F8093430B9093440BA093C9
:10D86000450BB093460B8CEF90E390935A02809354
:10D8700059021092490B10924A0B10924B0B1092C6
:10D880004C0B1F910F91FF90EF90DF90CF90089578
:10D89000CF92DF92EF92FF920F931F932091490B4B
:10D8A00030914A0B40914B0B50914C0B2115310597
:10D8B0004105510509F47AC0B901882777FD8095A3
:10D8C000982F0E942FDC20916C0B30916D0B4091B2
:10D8D0006E0B50916F0B0E946DDE2091790D30918F
:10D8E0007A0D40917B0D50917C0D0E94B4DA6093CB
:10D8F000790D70937A0D80937B0D90937C0DE09061
:10D90000950DF090960D0091970D1091980DA8012E
:10D9100097010E948DDB882344F4E092790DF09208
:10D920007A0D00937B0D10937C0DE0907802F090BF
:10D93000790200917A0210917B026091790D7091C9
:10D940007A0D80917B0D90917C0DA80197010E942A
:10D950009BDD181644F4E092790DF0927A0D009355
:10D960007B0D10937C0D1092490B10924A0B109274
:10D970004B0B10924C0B81E79DE065E77DE049E79A
:10D980005DE02DE73DE00F2EF0E0EF2EF0E0FF2E02
:10D99000F0E70F2FF2E41F2FF02DF1EBCF2EFDE07B
:10D9A000DF2E0E94EB1E81E080935B0280915B0280
:10D9B000882349F089E79DE00E949A2BBC0183E708
:10D9C00095E00E942E4A8091410B82FF28C082E0A0
:10D9D00080935B020FB6F89480914C1190914D1199
:10D9E000A0914E11B0914F110FBE8C509E4FAF4F72
:10D9F000BF4F8093430B9093440BA093450BB09380
:10DA0000460B8CEF90E390935A0280935902109248
:10DA1000490B10924A0B10924B0B10924C0B1F911A
:10DA20000F91FF90EF90DF90CF900895CF92DF920B
:10DA3000EF92FF920F931F932091490B30914A0B65
:10DA400040914B0B50914C0B21153105410551056F
:10DA500009F47AC0B901882777FD8095982F0E9434
:10DA60002FDC20916C0B30916D0B40916E0B50911F
:10DA70006F0B0E946DDE2091750D3091760D4091F7
:10DA8000770D5091780D0E94B4DA6093750D709304
:10DA9000760D8093770D9093780DE090910DF09036
:10DAA000920D0091930D1091940DA80197010E9481
:10DAB0008DDB882344F4E092750DF092760D00938F
:10DAC000770D1093780DE0907402F090750200913C
:10DAD0007602109177026091750D7091760D8091AC
:10DAE000770D9091780DA80197010E949BDD181683
:10DAF00044F4E092750DF092760D0093770D10933B
:10DB0000780D1092490B10924A0B10924B0B109209
:10DB10004C0B81E79DE065E77DE049E75DE02DE79F
:10DB20003DE00F2EF0E0EF2EF0E0FF2EF6E10F2F9C
:10DB3000F4E41F2FF02DA1EBCA2EADE0DA2E0E94E7
:10DB4000EB1E81E080935B0280915B02882349F0A9
:10DB500085E79DE00E949A2BBC0185E795E00E9435
:10DB60002E4A8091410B82FF28C082E080935B02A5
:10DB70000FB6F89480914C1190914D11A0914E11D7
:10DB8000B0914F110FBE8C509E4FAF4FBF4F80933F
:10DB9000430B9093440BA093450BB093460B8CEF33
:10DBA00090E390935A02809359021092490B10927D
:10DBB0004A0B10924B0B10924C0B1F910F91FF9040
:10DBC000EF90DF90CF900895CF92DF92EF92FF9287
:10DBD0000F931F932091490B30914A0B40914B0BAF
:10DBE00050914C0B211531054105510509F47AC0BE
:10DBF000B901882777FD8095982F0E942FDC20910E
:10DC00006C0B30916D0B40916E0B50916F0B0E941D
:10DC10006DDE2091710D3091720D4091730D509118
:10DC2000740D0E94B4DA6093710D7093720D80933D
:10DC3000730D9093740DE0908D0DF0908E0D00910A
:10DC40008F0D1091900DA80197010E948DDB882304
:10DC500044F4E092710DF092720D0093730D1093E5
:10DC6000740DE0907002F0907102009172021091B8
:10DC700073026091710D7091720D8091730D90918E
:10DC8000740DA80197010E949BDD181644F4E092E0
:10DC9000710DF092720D0093730D1093740D10922C
:10DCA000490B10924A0B10924B0B10924C0B81E7D0
:10DCB0009DE065E77DE049E75DE02DE73DE00F2E63
:10DCC000F0E0EF2EF0E0FF2EF6E10F2FF4E41F2F2F
:10DCD000F02DB1EBCB2EBDE0DB2E0E94EB1E81E0E0
:10DCE00080935B0280915B02882349F081E79DE08D
:10DCF0000E949A2BBC0187E795E00E942E4A8091F2
:10DD0000410B82FF28C082E080935B020FB6F8943B
:10DD100080914C1190914D11A0914E11B0914F11E5
:10DD20000FBE8C509E4FAF4FBF4F8093430B9093CD
:10DD3000440BA093450BB093460B8CEF90E390936C
:10DD40005A02809359021092490B10924A0B10927A
:10DD50004B0B10924C0B1F910F91FF90EF90DF90A7
:10DD6000CF900895CF92EF920F938DE29BE069E000
:10DD700048E027E006E055E0E52E34E0C32E0E949F
:10DD800054D20F91EF90CF9008956091680B7091ED
:10DD9000690B80916A0B90916B0B0E94FC9A6093C7
:10DDA000990270939A0280939B0290939C020C9428
:10DDB000EC996091640B7091650B8091660B90916A
:10DDC000670B0E94F09A609395027093960280937D
:10DDD0009702909398020C94EC99BC0180912C0BC3
:10DDE000882349F484E492E044E150E00E949210D8
:10DDF00082E080935B020895F0DF81E080932C0B3A
:10DE00001092490B10924A0B10924B0B10924C0B34
:10DE100082EF95E390935A02809359020895BC01D2
:10DE200080912C0B882349F484E492E044E150E093
:10DE30000E94FC1082E080935B0208950E941F2BD9
:10DE40000FB6F89420914C1130914D1140914E1124
:10DE500050914F110FBE80914D0B90914E0BA091A0
:10DE60004F0BB091500B82179307A407B50708F02A
:10DE7000AFC02091480B2223A9F181E080935B027F
:10DE8000332727FD3095432F532F8091490B9091D5
:10DE90004A0BA0914B0BB0914C0B820F931FA41F08
:10DEA000B51F8093490B90934A0BA0934B0BB093F3
:10DEB0004C0B1092480B0FB6F89480914C11909136
:10DEC0004D11A0914E11B0914F110FBE8856954C37
:10DED000AF4FBF4F8093780B9093790BA0937A0B41
:10DEE000B0937B0B8091410B82FF17C00FB6F89463
:10DEF00080914C1190914D11A0914E11B0914F1104
:10DF00000FBE8856954CAF4FBF4F8093780B9093C0
:10DF1000790BA0937A0BB0937B0BE0915902F091AF
:10DF20005A0209950FB6F89420914C1130914D1179
:10DF300040914E1150914F110FBE8091780B9091EE
:10DF4000790BA0917A0BB0917B0B82179307A407F2
:10DF5000B507C0F48091590290915A02825F9543AF
:10DF600089F01092490B10924A0B10924B0B1092B1
:10DF70004C0B82EF95E390935A028093590282E012
:10DF800080935B0280915B02823021F48DE29BE002
:10DF90000E94A5D180915B02882319F08150809363
:10DFA0005B020FB6F89480914C1190914D11A091A5
:10DFB0004E11B0914F110FBE8C599F4FAF4FBF4FB5
:10DFC00080934D0B90934E0BA0934F0BB093500B3F
:10DFD0000895DF93CF93CDB7DEB7C054D0400FB6CE
:10DFE000F894DEBF0FBECDBFDE011196E4EFF2E084
:10DFF00088E001900D928150E1F7DE011996ECEE78
:10E00000F2E088E001900D928150E1F7DE01519637
:10E01000E4EEF2E088E001900D928150E1F7DE013C
:10E020005996ECEDF2E088E001900D928150E1F715
:10E03000DE019196E4EDF2E088E001900D928150CE
:10E04000E1F7DE019996ECECF2E088E001900D92A8
:10E050008150E1F7DE01D196E4ECF2E088E0019036
:10E060000D928150E1F7DE01D996ECEBF2E088E009
:10E0700001900D928150E1F78DE29BE064E144E074
:10E0800020E00E94ACD18DE29BE060E0AE014F5FEA
:10E090005F4F0E9448D18DE29BE061E0AE01475F97
:10E0A0005F4F0E9448D18DE29BE062E0AE014F5E7F
:10E0B0005F4F0E9448D18DE29BE063E0AE01475E76
:10E0C0005F4F0E9448D18DE29BE064E0AE014F5D5E
:10E0D0005F4F0E9448D18DE29BE065E0AE01475D55
:10E0E0005F4F0E9448D18DE29BE066E0AE014F5C3D
:10E0F0005F4F0E9448D18DE29BE067E0AE01475C34
:10E100005F4F0E9448D18DE29BE00E94A5D1C05C88
:10E11000DF4F0FB6F894DEBF0FBECDBFCF91DF91BA
:10E12000089557DF38983998409A419A3A98429A18
:10E130000E941F2B1092480B08956091260B70913E
:10E14000270B882777FD8095982F0E942FDC0E944F
:10E15000FCDB7093940F6093930F7093960F609312
:10E16000950F7093980F6093970F6091280B7091A3
:10E17000290B882777FD8095982F0E942FDC0E941D
:10E18000FCDB70939A0F6093990F80912A0B90910A
:10E190002B0B9093B30D8093B20D1092490B1092FC
:10E1A0004A0B10924B0B10924C0B82EF95E390931D
:10E1B0005A02809359020C94D29A6091200B70916C
:10E1C000210B882777FD8095982F0E942FDC0E94D5
:10E1D000FCDB7093940F6093930F7093960F609392
:10E1E000950F7093980F6093970F6091220B709129
:10E1F000230B882777FD8095982F0E942FDC0E94A3
:10E20000FCDB70939A0F6093990F8091240B90918F
:10E21000250B9093B30D8093B20D1092490B109281
:10E220004A0B10924B0B10924C0B82EF95E390939C
:10E230005A02809359020C94D29ABF92CF92DF92E5
:10E24000EF92FF920F931F938091490B90914A0B8D
:10E25000A0914B0BB0914C0B81509048A040B04026
:10E2600040F01092490B10924A0B10924B0B1092F7
:10E270004C0B6091490B70914A0B80914B0B909124
:10E280004C0B25E030E040E050E00E9485DF790152
:10E290008A018091420B90E0A0E0B0E0E816F90618
:10E2A0000A071B0710F42093420B0091420B10E069
:10E2B00062E2C62ED12CE12CF12CBB24B3940023B6
:10E2C00009F04AC080915B028823C1F08091490B1C
:10E2D00090914A0BA0914B0BB0914C0B0597A10567
:10E2E000B10528F4812F67E175E043E004C0812F78
:10E2F00067E175E040E223E00E94C32E8091410B6C
:10E3000082FF73C28091490B90914A0BA0914B0BF5
:10E31000B0914C0B0597A105B10508F066C282E0EB
:10E3200080935B020FB6F89480914C1190914D113F
:10E33000A0914E11B0914F110FBE8C509E4FAF4F18
:10E34000BF4F8093430B9093440BA093450BB09326
:10E35000460B8EE494E53CC2013009F058C0809130
:10E360005B028823F9F06091490B70914A0B809110
:10E370004B0B90914C0B25E030E040E050E00E94C8
:10E3800085DF213031054105510529F4812F66E0F3
:10E3900075E04EE304C0812F66E075E040E220E2C4
:10E3A0000E94C32E8091410B82FF1FC26091490BD6
:10E3B00070914A0B80914B0B90914C0B25E030E013
:10E3C00040E050E00E9485DF2130310541055105D4
:10E3D00009F00BC282E080935B020FB6F894809143
:10E3E0004C1190914D11A0914E11B0914F110FBE53
:10E3F0008C509E4FAF4FBF4F8093430B9093440B75
:10E40000A093450BB093460B82E095E05AC00230D2
:10E4100009F05AC080915B028823F9F06091490BA2
:10E4200070914A0B80914B0B90914C0B25E030E0A2
:10E4300040E050E00E9485DF223031054105510562
:10E4400029F4812F68EF74E04EE304C0812F68EF58
:10E4500074E040E220E20E94C32E8091410B82FFD3
:10E46000C4C16091490B70914A0B80914B0B909104
:10E470004C0B25E030E040E050E00E9485DF223088
:10E4800031054105510509F0B0C182E080935B027E
:10E490000FB6F89480914C1190914D11A0914E11AE
:10E4A000B0914F110FBE8C509E4FAF4FBF4F809316
:10E4B000430B9093440BA093450BB093460B84EF12
:10E4C00094E00E94FE98C9C1033009F057C08091C2
:10E4D0005B028823F9F06091490B70914A0B80919F
:10E4E0004B0B90914C0B25E030E040E050E00E9457
:10E4F00085DF233031054105510529F4812F68EE70
:10E5000074E04EE304C0812F68EE74E040E220E244
:10E510000E94C32E8091410B82FF67C16091490B1D
:10E5200070914A0B80914B0B90914C0B25E030E0A1
:10E5300040E050E00E9485DF233031054105510560
:10E5400009F053C182E080935B020FB6F89480918A
:10E550004C1190914D11A0914E11B0914F110FBEE1
:10E560008C509E4FAF4FBF4F8093430B9093440B03
:10E57000A093450BB093460B20DE6FC1043009F029
:10E5800057C080915B028823F9F06091490B70912C
:10E590004A0B80914B0B90914C0B25E030E040E012
:10E5A00050E00E9485DF243031054105510529F4F2
:10E5B000812F6CED74E04EE304C0812F6CED74E0AC
:10E5C00040E220E20E94C32E8091410B82FF0DC1E8
:10E5D0006091490B70914A0B80914B0B90914C0BC1
:10E5E00025E030E040E050E00E9485DF2430310536
:10E5F0004105510509F0F9C082E080935B020FB636
:10E60000F89480914C1190914D11A0914E11B091C0
:10E610004F110FBE8C509E4FAF4FBF4F8093430B97
:10E620009093440BA093450BB093460B86DD15C128
:10E63000053009F074C080915B028823F9F0609185
:10E64000490B70914A0B80914B0B90914C0B25E03C
:10E6500030E040E050E00E9485DF25303105410583
:10E66000510529F4812F63ED74E04EE304C0812F3E
:10E6700063ED74E040E220E20E94C32E8091410BE2
:10E6800082FFB3C06091490B70914A0B80914B0B94
:10E6900090914C0B25E030E040E050E00E9485DF97
:10E6A000253031054105510509F09FC082E0809376
:10E6B0005B020FB6F89480914C1190914D11A0918E
:10E6C0004E11B0914F110FBE8C509E4FAF4FBF4FA8
:10E6D0008093430B9093440BA093450BB093460B50
:10E6E0001092940F1092930F1092960F1092950F14
:10E6F0001092980F1092970F10929A0F1092990FF4
:10E700001092490B10924A0B10924B0B10924C0B2B
:10E7100082EF95E390935A02809359029EC006308F
:10E7200009F063C080915B028823F9F06091490B86
:10E7300070914A0B80914B0B90914C0B25E030E08F
:10E7400040E050E00E9485DF26303105410551054B
:10E7500029F4812F69EC74E04EE304C0812F69EC49
:10E7600074E040E22EE70E94C32E8091410B82FFAD
:10E770003CC06091490B70914A0B80914B0B90917A
:10E780004C0B25E030E040E050E00E9485DF263071
:10E7900031054105510549F582E080935B020FB6D2
:10E7A000F89480914C1190914D11A0914E11B0911F
:10E7B0004F110FBE8C509E4FAF4FBF4F8093430BF6
:10E7C0009093440BA093450BB093460B85E19FE2D9
:10E7D00090935A02809359021092490B10924A0B5F
:10E7E00010924B0B10924C0B38C08091490B9091BA
:10E7F0004A0BA0914B0BB0914C0B8397A105B1052F
:10E8000040F0C092490BD0924A0BE0924B0BF09231
:10E810004C0B6091490B70914A0B80914B0B90917E
:10E820004C0B25E030E040E050E00E9485DF422FB5
:10E830008091420B90E0039630E08217930744F4F6
:10E8400043504093420BB0925B02042F01501FEFE4
:10E850001F5F143010F40F5F32CD1F910F91FF90A6
:10E86000EF90DF90CF90BF900895FC014281242F5C
:10E8700030E0C9019595879580658CBD40FF02C049
:10E8800080E004C080E0463009F081E08DBD8081E9
:10E89000E82FF0E00C94A5D2DF92EF92FF920F9355
:10E8A0001F93CF93DF93EC01D62E79018A01DDDF30
:10E8B0000FB6F89480914C1190914D11A0914E118A
:10E8C000B0914F110FBE9C014FEF10C00FB6F894DE
:10E8D00080914C1190914D11A0914E11B0914F111A
:10E8E0000FBE821B930B8C52914038F44EBD0DB479
:10E8F00007FEFDCF8EB58F3F49F78D2D80648EBD0D
:10E900000DB407FEFDCF28E130E0D801C701022E8B
:10E9100004C0B695A795979587950A94D2F78EBDB2
:10E920000DB407FEFDCF285030408FEF283F380749
:10E9300061F7DD2011F485E906C058E0D51611F421
:10E9400087E801C08FEF8EBD0DB407FEFDCF8CE0D0
:10E95000D81631F48FEF8EBD0DB407FEFDCF8EB506
:10E960009FEF2FEF2EBD0DB407FEFDCF8EB587FFB5
:10E9700004C0992311F09150F5CF8B83DF91CF9193
:10E980001F910F91FF90EF90DF900895BF92CF926B
:10E99000DF92EF92FF920F931F938C01B62E6901C5
:10E9A0007A0167E320E030E040E050E075DFC80125
:10E9B0006B2DA701960170DF1F910F91FF90EF90D3
:10E9C000DF90CF90BF900895FC018081E82FF0E0A8
:10E9D0000C949FD2DC016EBDFA0120E030E00DB452
:10E9E00007FEFDCF80818EBD0DB407FEFDCF818176
:10E9F0008EBD2E5F3F4F329682E02030380779F788
:10EA00000DB407FEFDCF8FEF8EBD0DB407FEFDCF19
:10EA10008FEF8EBD0DB407FEFDCF8FEF8EBD0DB411
:10EA200007FEFDCF8EB513968C9313978F718530AB
:10EA300011F481E0089583E111968C931197CD0133
:10EA4000C3DF80E00895CF92DF92EF92FF920F93A1
:10EA50001F93CF93DF93EC017A018B0169018C81C5
:10EA6000833039F059E0EE0CFF1C001F111F5A953E
:10EA7000D1F7CE0168E1A80197010EDF882311F0DC
:10EA800086E036C0CE016EEFA601A4DF882389F1AF
:10EA90000FB6F89480914C1190914D11A0914E11A8
:10EAA000B0914F110FBE9C014FEF10C00FB6F894FC
:10EAB00080914C1190914D11A0914E11B0914F1138
:10EAC0000FBE821B930B8855924040F44EBD0DB48F
:10EAD00007FEFDCF1EB51F3F49F717C087E108C0ED
:10EAE0001EBD0DB407FEFDCF8EB58823C1F086E1B3
:10EAF0008983CE0169DF80E0DF91CF911F910F9173
:10EB0000FF90EF90DF90CF900895CE016DE020E070
:10EB100030E040E050E0C0DE882349F7E1CFCE018D
:10EB200053DF81E0E9CFCF93DF93EC010FB6F89488
:10EB300080914C1190914D11A0914E11B0914F11B7
:10EB40000FBEFC013FEF13C00FB6F89480914C113B
:10EB500090914D11A0914E11B0914F110FBE8E1B8F
:10EB60009F0B8D52914018F02B8381E10BC03EBD6D
:10EB70000DB407FEFDCF2EB52F3F31F32B832E3F73
:10EB800031F08FE08983CE011FDF80E02EC0DA01F3
:10EB90001197452BD9F08FEF8EBD20E030E09FEF2D
:10EBA0000BC00DB407FEFDCF8EB5FB01E20FF31FC6
:10EBB00080839EBD2F5F3F4F2A173B0790F30DB414
:10EBC00007FEFDCF8EB5A60FB71F8C938FEF8EBDBE
:10EBD0000DB407FEFDCF8EB58FEF8EBD0DB407FED1
:10EBE000FDCF8EB5CE01F0DE81E0DF91CF910895AB
:10EBF000CF92DF92EF92FF920F931F93CF93DF9309
:10EC0000EC017A018B0169018C81833039F0A9E034
:10EC1000EE0CFF1C001F111FAA95D1F7CE0161E178
:10EC2000A801970139DE882331F084E08983CE0181
:10EC3000CBDE80E005C0CE01B60140E052E073DFDC
:10EC4000DF91CF911F910F91FF90EF90DF90CF90C8
:10EC50000895BF92CF92DF92EF92FF920F931F938E
:10EC6000CF93DF93EC01B62E842F1C821982488348
:10EC70000FB6F89420914C1130914D1140914E11E6
:10EC800050914F110FBE69010E948BD2CE019CDEC4
:10EC900023982B98229A219A209A289A85E08A8391
:10ECA00082E58CBD1DBC80E09FEF9EBD0DB407FECC
:10ECB000FDCF8F5F8A30C9F712C00FB6F8948091EC
:10ECC0004C1190914D11A0914E11B0914F110FBE6A
:10ECD0008C199D09815D974010F081E05BC0CE01E9
:10ECE00060E020E030E040E050E0D6DD182F8B837C
:10ECF000813019F7CE0168E02AEA31E040E050E0C7
:10ED0000CBDD82FF02C01C8311C080E02FEF2EBD3F
:10ED10000DB407FEFDCF9EB58F5F8430C1F79B8396
:10ED20009A3A11F082E036C082E08C838C81823086
:10ED300021F0EE24FF24870118C0E12CF12C012DD5
:10ED400000E4102F12C00FB6F89480914C119091EE
:10ED50004D11A0914E11B0914F110FBE8C199D090C
:10ED6000815D974010F08AE015C0CE0169E2A801EC
:10ED700097010CDE8B83882331F78C81823019F563
:10ED8000CE016AE320E030E040E050E085DD8823FA
:10ED900029F088E08983CE0117DE20C08FEF8EBD79
:10EDA0000DB407FEFDCF8EB5807C803C11F483E06E
:10EDB0008C8380E09FEF9EBD0DB407FEFDCF2EB586
:10EDC0008F5F8330C1F7CE01FFDD86E08B1518F42D
:10EDD00088E1898303C0BA8281E001C080E0DF91CD
:10EDE000CF911F910F91FF90EF90DF90CF90BF9048
:10EDF00008952F923F924F925F926F927F928F92DF
:10EE00009F92AF92BF92CF92DF92EF92FF920F93B9
:10EE10001F93DF93CF93CDB7DEB7CD55D0400FB65C
:10EE2000F894DEBF0FBECDBF2F969FAF8EAF2F974A
:10EE300061967FAF6EAF61972A0162962FAF62979E
:10EE400063960FAF63976496EFAE64976896ACAE27
:10EE5000BDAECEAEDFAE6897E22EFF24EE0CFF1CF7
:10EE6000EE0CFF1C9A012E0D3F1D2D963FAF2EAFCD
:10EE70002D97D9016D907D908D909C90FC01EE0DA9
:10EE8000FF1DC401B30120813181428153810E9461
:10EE9000B4DA69AF7AAF8BAF9CAF10E0000F111FEF
:10EEA000000F111FF201E00FF11F2B96FFAFEEAF25
:10EEB0002B97A080B180C280D3802F96EEADFFAD9E
:10EEC0002F97E00FF11FC601B501208131814281EA
:10EED00053810E94B4DA6DAB7EAB8FAB98AF649672
:10EEE0002FAD6497E22FF0E0EE0FFF1FEE0FFF1F34
:10EEF0002F96AEADBFAD2F97AE0FBF1F4D915D9159
:10EF00006D917C9129964CAF5DAF6EAF7FAF299725
:10EF100061966EAD7FAD6197E60FF71F60817181DD
:10EF20008281938129962CAD3DAD4EAD5FAD299781
:10EF30000E94B3DA69AB7AAB8BAB9CAB6196AEAD9A
:10EF4000BFAD61971C968D919D910D90BC91A02DA8
:10EF500025968CAF9DAFAEAFBFAF25972F96AEADC8
:10EF6000BFAD2F971C962D913D914D915C911F97B0
:10EF700021962CAF3DAF4EAF5FAF2197A401930117
:10EF800050582DA73EA74FA758ABB601A501705802
:10EF900049A75AA76BA77CA761966EAD7FAD619715
:10EFA000E60EF71ED7016D917D918D919C9129AD53
:10EFB0003AAD4BAD5CAD0E94B3DA3B014C016196BA
:10EFC000EEADFFAD61970E0F1F1FD8016D917D91C2
:10EFD0008D919C912DA93EA94FA958AD0E94B3DAFD
:10EFE0005B016C016DA57EA58FA598A9A601950171
:10EFF0000E946DDE7B018C0169A57AA58BA59CA57D
:10F00000A40193010E946DDE9B01AC01C801B70110
:10F010000E94B3DA1B012C016DA57EA58FA598A9CE
:10F02000A40193010E946DDE7B018C0169A57AA584
:10F030008BA59CA5A60195010E946DDE9B01AC01EC
:10F04000C801B7010E94B4DA9B01AC01C201B10151
:10F050000E9427DB5B016C0120E030E040E050E0E3
:10F060000E948DDB882354F4C601B5012BED3FE0EF
:10F0700049EC50E40E94B4DA5B016C01E7968FAD75
:10F08000E797882351F0C601B5012BED3FE049EC2D
:10F0900050E40E94B3DA5B016C01C601B501E6964B
:10F0A0002CAD3DAD4EAD5FADE6970E946DDE29A95A
:10F0B0003AA94BA95CA95F770E94A8DD7B018C016E
:10F0C0002FE632E143E85AE30E948DDB87FDF5C16C
:10F0D000C801B7010E946ADC0E9401DC78A76FA317
:10F0E000672B21F4E1E0F0E0F8A7EFA32FA138A50A
:10F0F000B90180E090E00E942DDC7B018C01C6010B
:10F10000B501A80197010E9494DB6BA37CA38DA39A
:10F110009EA369A97AA98BA99CA9A80197010E941D
:10F1200094DB6F8F78A389A39AA325966CAD7DADF0
:10F130008EAD9FAD259721962CAD3DAD4EAD5FAD0B
:10F1400021970E94B3DAA80197010E9494DB6B8F8C
:10F150007C8F8D8F9E8F6BA17CA18DA19EA120E0C5
:10F1600030E040E05FEB0E946DDE2BA13CA14DA1A1
:10F170005EA10E946DDE20E030E040E85FE30E9487
:10F18000B4DA6F8B788F898F9A8F64963FAD6497CE
:10F19000E32FF0E0EE0FFF1FEE0FFF1F9E012F5F2A
:10F1A0003F4FE20FF31F29964CAD5DAD6EAD7FADC5
:10F1B000299740835183628373832F96AEADBFAD91
:10F1C0002F971C964D915D916D917C911F974D8766
:10F1D0005E876F87788B41E050E05A8B498B6624BD
:10F1E00062967FAD6297672F70E0660F771F660F9C
:10F1F000771FC901860F971F6A969FAF8EAF6A97D8
:10F200006396BFAD6397AB2FB0E0AA0FBB1FAA0FE9
:10F21000BB1F21E030E02C0F3D1F2A0F3B1F6C96D7
:10F220003FAF2EAF6C976E96FFAFEEAF6E9719C1E2
:10F2300038E136150CF446C06DA57EA58FA598A9BA
:10F240002BA13CA14DA15EA10E946DDE7B018C0132
:10F2500069A57AA58BA59CA52F89388D498D5A8DD6
:10F260000E946DDE9B01AC01C801B7010E94B4DAB7
:10F270007B018C016DA57EA58FA598A92F89388D5E
:10F28000498D5A8D0E946DDE5B016C0169A57AA5DE
:10F290008BA59CA52BA13CA14DA15EA10E946DDE7A
:10F2A0009B01AC01C601B5010E94B3DA6DA77EA730
:10F2B0008FA798AB6394C701D80189A79AA7ABA77A
:10F2C000BCA765C049895A89BA0180E090E00E94D4
:10F2D0002DDC2BA13CA14DA15EA10E946DDE7B0126
:10F2E0008C01C8010E9491DB6B8B7C8B8D8B9E8B7C
:10F2F000B701C8010E94D0DE3B014C012D96AEAD96
:10F30000BFAD2D97ED90FD900D911C9117FB1095C1
:10F3100017F910952B96EEADFFAD2B97208031801D
:10F3200042805380C801B7012B893C894D895E8991
:10F330000E946DDE5B016C01C201B101A401930169
:10F340000E946DDE9B01AC01C601B5010E94B4DADA
:10F350006DA77EA78FA798ABC801B701A401930141
:10F360000E946DDE7B018C01C201B1012B893C89B9
:10F370004D895E890E946DDE9B01AC01C801B70119
:10F380000E94B3DA69A77AA78BA79CA7662469AD08
:10F390007AAD8BAD9CAD2DA53EA54FA558A90E9479
:10F3A000B4DA6A96AEADBFAD6A976D937D938D93D7
:10F3B0009C9313976DA97EA98FA998AD29A53AA50D
:10F3C0004BA55CA50E94B4DA6C96EEADFFAD6C97D0
:10F3D00060837183828393836E96AEADBFAD6E976B
:10F3E0006D917D918D919C912F8D38A149A15AA14C
:10F3F0000E94B4DA6E96EEADFFAD6E9760837183B6
:10F40000828393836D857E858F8598892B8D3C8D36
:10F410004D8D5E8D0E94B4DA6D877E878F87988BC5
:10F42000CE010196AED0CE010196BE016B5F7F4F3B
:10F43000AE01475F5F4F9E01235F3F4F6896ECAC84
:10F44000FDAC0EAD1FAD6897F7E7CF2ED12CCC0EDB
:10F45000DD1E0E94EB1E29893A892F5F3F4F3A8BB0
:10F46000298B49895A896FA178A54617570708F44F
:10F47000DFCE61964EAD5FAD6197485F5F4F61969D
:10F480002EAD3FAD6197245F3F4F61968EAD9FAD2E
:10F490006197DC0114966196BFAFAEAF6197BD0175
:10F4A0006896ECACFDAC0EAD1FAD6897E7E7CE2ECD
:10F4B000D12CCC0EDD1E0E94EB1EC35ADF4F0FB6BF
:10F4C000F894DEBF0FBECDBFCF91DF911F910F919A
:10F4D000FF90EF90DF90CF90BF90AF909F908F9074
:10F4E0007F906F905F904F903F902F900895DF93A3
:10F4F000CF930F92CDB7DEB7FC016983A081B181B4
:10F5000012962D913C911397BE016F5F7F4F41E0A2
:10F5100050E0F90109950F90CF91DF910895CF93B5
:10F52000DF930FB6F89480914C1190914D11A091FA
:10F530004E11B0914F110FBE8093D20D9093D30D09
:10F54000A093D40DB093D50DE091FB0DF091FC0D7F
:10F55000E350F24F8081882389F4E3E9F6E0649177
:10F56000EF0106C085E591E1C2DF2196FE016491BD
:10F570006623C1F785E591E16AE0B9DFDF91CF91BC
:10F580000895EF92FF920F931F93CF93DF93EC01B7
:10F59000E0908D0DF0908E0D00918F0D1091900DDB
:10F5A000688179818A819B81A80197010E948DDB06
:10F5B000882324F4E882F9820A831B83E090910D6A
:10F5C000F090920D0091930D1091940D6C817D81BE
:10F5D0008E819F81A80197010E948DDB882324F4EE
:10F5E000EC82FD820E831F83E090950DF090960DC6
:10F5F0000091970D1091980D688579858A859B8576
:10F60000A80197010E948DDB882324F4E886F986FF
:10F610000A871B87E0907002F090710200917202DD
:10F6200010917302688179818A819B81A801970179
:10F630000E949BDD181624F4E882F9820A831B835A
:10F64000E0907402F09075020091760210917702BA
:10F650006C817D818E819F81A80197010E949BDD35
:10F66000181624F4EC82FD820E831F83E09078024A
:10F67000F090790200917A0210917B026885798579
:10F680008A859B85A80197010E949BDD181624F4AA
:10F69000E886F9860A871B87DF91CF911F910F912A
:10F6A000FF90EF9008958091BC0D08950F931F93E4
:10F6B000CF93DF938130910549F46F5F7F4F09F05D
:10F6C00046C08CE79BE00E94C7CD41C0892B09F062
:10F6D0003EC06F5F7F4FD9F585E893E090933B0D77
:10F6E00080933A0D8091400D882321F08DE39DE0B9
:10F6F0000E9416B1C7EFDCE005E813E005C06E9785
:10F700008BE0CB3CD80751F0198308838E81882386
:10F71000B1F3CE0103960E9416B1F1CF85E893E0D4
:10F72000998388838E81882321F0CE0103960E94DD
:10F7300016B185E893E09093AC0B8093AB0B80916E
:10F74000B10B882321F08EEA9BE00E9416B1DF9175
:10F75000CF911F910F91089580E090E06FEF7FEFC0
:10F76000A5CF81E090E06FEF7FEFA0CFEF92FF9207
:10F770000F931F93CF93DF93EC017A018B01FC0170
:10F78000649106C085E591E1B2DE2196FE016491A7
:10F790006623C1F785E591E1B801A7012AE000E001
:10F7A0000E9456D7DF91CF911F910F91FF90EF905C
:10F7B0000895CF93DF930E94D39A8091BC0D882344
:10F7C00009F035C081E08093BC0D8091CA0D909105
:10F7D000CB0DA091CC0DB091CD0D8093CE0D90931B
:10F7E000CF0DA093D00DB093D10DE4EEF5E0649170
:10F7F000EF0106C085E591E17ADE2196FE01649174
:10F800006623C1F7E5EFF5E06491EF0106C085E5F9
:10F8100091E16DDE2196FE0164916623C1F785E5D5
:10F8200091E16AE064DE8BEE95E00E94ED6EDF917F
:10F83000CF910895CF93DF93F8940E94D39A779A4B
:10F84000769A479A439A8C9A8D9AE4EEF5E0649101
:10F85000EF0106C085E591E14ADE2196FE01649143
:10F860006623C1F7E4E7F6E06491EF0106C085E5A1
:10F8700091E13DDE2196FE0164916623C1F785E5A5
:10F8800091E16AE034DE8BE696E00E94FC6EFFCFE9
:10F89000EF92FF920F931F930FB6F89480914C1143
:10F8A00090914D11A0914E11B0914F110FBEE0906B
:10F8B000D60DF090D70D0091D80D1091D90D209153
:10F8C000D20D3091D30D4091D40D5091D50D821BA6
:10F8D000930BA40BB50BE816F9060A071B0730F4C7
:10F8E000E114F1040105110509F0A4DFE09088029C
:10F8F000F090890200918A0210918B02E114F104C8
:10F900000105110541F10FB6F89480914C119091C9
:10F910004D11A0914E11B0914F110FBE2091D20DFB
:10F920003091D30D4091D40D5091D50D821B930B86
:10F93000A40BB50BE816F9060A071B0760F49091B3
:10F94000060B8091070B981731F4779A769A479AAD
:10F95000439A8C9A8D9A0E9464191F910F91FF907F
:10F96000EF9008956F927F928F929F92AF92BF9285
:10F97000CF92DF92EF92FF920F931F93F82E609138
:10F98000DA0D7091DB0D8091DC0D9091DD0D2091F1
:10F99000DE0D3091DF0D4091E00D5091E10D0E94A0
:10F9A000A8DD3B014C0100D000D000D00DB71EB740
:10F9B0000F5F1F4F60916C0270916D02882777FD79
:10F9C0008095982F0E942FDC20918C0230918D021F
:10F9D00040918E0250918F020E946DDE20E030E057
:10F9E00040E752E40E9494DB20E030E048EC52E42F
:10F9F0000E9494DB5B016C01F8016082718282825B
:10FA00009382F4828091B10D858381E79DE066EE5B
:10FA10007DE04AED5DE020E001E032E0E32EE9D94F
:10FA20008091E60D9091E70DA091E80DB091E90D60
:10FA30008093710D9093720DA093730DB093740D1C
:10FA40008091EA0D9091EB0DA091EC0DB091ED0D30
:10FA50008093750D9093760DA093770DB093780DEC
:10FA60008091EE0D9091EF0DA091F00DB091F10D00
:10FA70008093790D90937A0DA0937B0DB0937C0DBC
:10FA80008091F20D9091F30DA091F40DB091F50DD0
:10FA900080937D0D90937E0DA0937F0DB093800D8C
:10FAA0000FB6F89480914C1190914D11A0914E1188
:10FAB000B0914F110FBE8093D20D9093D30DA093B0
:10FAC000D40DB093D50D8DB79EB706960FB6F894AA
:10FAD0009EBF0FBE8DBF1F910F91FF90EF90DF90E3
:10FAE000CF90BF90AF909F908F907F906F90089530
:10FAF000CF92DF92EF92FF920F931F9386EE9DE0DD
:10FB000040DD0FB6F89480914C1190914D11A09169
:10FB10004E11B0914F110FBE8093D20D9093D30D23
:10FB2000A093D40DB093D50D6091710D7091720DAD
:10FB30008091730D9091740D2091E60D3091E70D39
:10FB40004091E80D5091E90D0E948DDB882309F06A
:10FB50007AC06091750D7091760D8091770D9091BE
:10FB6000780D2091EA0D3091EB0D4091EC0D509104
:10FB7000ED0D0E948DDB882309F065C060918C0239
:10FB800070918D0280918E0290918F0220E030E082
:10FB900040E752E40E9494DB7B018C0186EE9DE0FD
:10FBA0006AEE7DE04EEE5DE022EF3DE0E1EBCE2E31
:10FBB000EDE0DE2E0E94EB1E8091E60D9091E70DA8
:10FBC000A091E80DB091E90D8093710D9093720DA5
:10FBD000A093730DB093740D8091EA0D9091EB0D8D
:10FBE000A091EC0DB091ED0D8093750D9093760D75
:10FBF000A093770DB093780D8091EE0D9091EF0D5D
:10FC0000A091F00DB091F10D8093790D90937A0D44
:10FC1000A0937B0DB0937C0D8091F20D9091F30D2C
:10FC2000A091F40DB091F50D80937D0D90937E0D14
:10FC3000A0937F0DB093800D1F910F91FF90EF90D7
:10FC4000DF90CF90089560916C0270916D028827CB
:10FC500077FD8095982F0E942FDC20918C023091A7
:10FC60008D0240918E0250918F020E946DDE20E045
:10FC700030E040E752E40E9494DB20E030E048ECC2
:10FC800052E488CFCF93DF9385E591E10E940ED9AE
:10FC9000E6E9F6E06491EF0106C085E591E127DC35
:10FCA0002196FE0164916623C1F74091CA0D5091DF
:10FCB000CB0D6091CC0D7091CD0D4F5F5F4F6F4FAD
:10FCC0007F4F85E591E10E94E1D785E591E16AE00A
:10FCD0000EDC25DCDF91CF9108952F923F924F9259
:10FCE0005F926F927F928F929F92AF92BF92CF92CC
:10FCF000DF92EF92FF920F931F93DF93CF93CDB7D5
:10FD0000DEB766970FB6F894DEBF0FBECDBF8C018D
:10FD10008330910508F0CCC11C01220C331C220C4D
:10FD2000331C91012F58324F3E872D8780E090E0A1
:10FD3000A0E0B0E0F90180839183A283B38381E7DF
:10FD40009DE065E77DE049E75DE02DE73DE00E944D
:10FD5000041A9E012F5F3F4F3E8B2D8BD901ECE0A3
:10FD60001D92EA95E9F760917C0270917D02809185
:10FD70007E0290917F022091BD0D3091BE0D409189
:10FD8000BF0D5091C00D0E94B3DA69837A838B83D3
:10FD90009C83609180027091810280918202909197
:10FDA00083022091C10D3091C20D4091C30D50913D
:10FDB000C40D0E94B3DA6D837E838F839887609130
:10FDC0008402709185028091860290918702209131
:10FDD000C50D3091C60D4091C70D5091C80D0E94C0
:10FDE000B3DA69877A878B879C87025A174FF801A5
:10FDF000E49091012A51324F388B2F8781E090E0B7
:10FE00008C0F9D1F820D931D9A8B898BDC016D9148
:10FE10007D918D919C9120E030E040EC5FE30E9469
:10FE20006DDE5B016C01FF24E7FCF0940F2D1F2DAC
:10FE3000C801B7010E942FDC2B013C01C601B501AE
:10FE4000A30192010E946DDEEF85F88960837183C2
:10FE5000828393839101245A3D4F3C8B2B8BD90194
:10FE60006D917D918D919C9160938C0270938D0228
:10FE700080938E0290938F0220E030E040E752E4BE
:10FE80000E9494DB7B018C0186EE9DE06AEE7DE0B2
:10FE90004EEE5DE022EF3DE0A1EBCA2EADE0DA2EA2
:10FEA0000E94EB1E0E945AA880E090E0A0E0B0E023
:10FEB000ED85FE8580839183A283B38381E79DE0F6
:10FEC00065E77DE049E75DE02DE73DE00E94041A2B
:10FED000F101EE5AF74F85909590A590B490C50129
:10FEE000B4019058A30192010E946DDEAF85B889DC
:10FEF0006D937D938D939C93139760918C02709179
:10FF00008D0280918E0290918F0220E030E040E7D8
:10FF100052E40E9494DB7B018C0186EE9DE06AEE48
:10FF20007DE04EEE5DE022EF3DE00E94EB1E0E9480
:10FF30005AA8C501B401A50194010E94B4DAA30135
:10FF400092010E946DDEEF85F88960837183828360
:10FF50009383AB89BC896D917D918D919C9120E0BB
:10FF600030E040E05FE30E946DDE60938C027093AE
:10FF70008D0280938E0290938F0220E030E040E764
:10FF800052E40E9494DB7B018C0186EE9DE06AEED8
:10FF90007DE04EEE5DE022EF3DE00E94EB1E0E9410
:10FFA0005AA8ED89FE892CE011922A95E9F78091F3
:10FFB000BD0D9091BE0DA091BF0DB091C00D898374
:10FFC0009A83AB83BC838091C10D9091C20DA091A7
:10FFD000C30DB091C40D8D839E83AF83B88780918C
:10FFE000C50D9091C60DA091C70DB091C80D898720
:10FFF0009A87AB87BC87F101EF57F24FA080B180A1
:020000021000EC
:10000000C280D380C601B501A989BA892D913D91DD
:100010004D915C910E94B4DA7B018C01CB01D80137
:10002000ED85FE8580839183A283B383FDE88F2EC7
:10003000FDE09F2E820C931CF101E354F24F60818E
:10004000718182819381A60195010E94B4DAD40165
:100050006D937D938D939C931397F101E458FD4F1D
:100060006081718182819381A60195010E94B4DA39
:10007000E0E7F2E02E0E3F1ED1016D937D938D934C
:100080009C931397C701D801EF85F88980839183EA
:10009000A283B38380E090E0A0E0B0E080938C0284
:1000A00090938D02A0938E02B0938F020E9472A74C
:1000B00066960FB6F894DEBF0FBECDBFCF91DF912D
:1000C0001F910F91FF90EF90DF90CF90BF90AF9076
:1000D0009F908F907F906F905F904F903F902F9068
:1000E00008954091FB0D5091FC0D20E630E0B901E0
:1000F000469F9001479F300D569F300D1124682F69
:10010000772767FD7095C901895F914F0E94DC10C8
:100110009C019093060E8093050E80E0232B09F03E
:1001200081E00895EF92FF920F931F93CF93DF9397
:10013000EC017A018B01FC01649106C085E591E137
:10014000D6D92196FE0164916623C1F785E591E138
:10015000B801A70122E00E94F2D7DF91CF911F9151
:100160000F91FF90EF9008958091050E9091060EEB
:10017000019660E070E04AE050E00C943B0F809103
:10018000050E9091060E019660E070E00C94DE0D75
:100190000F931F93CF93DF938C018091B10D8093C8
:1001A000C90D84E59EDF882309F44CC0E8DF0E9476
:1001B00001DC6093C90D633008F444C0EEEDF5E056
:1001C0006491EF0106C085E591E191D92196FE0188
:1001D00064916623C1F70936110599F00A361105B5
:1001E00024F408361105E9F407C00D36110571F045
:1001F0000A3D1105B1F40FC085E591E160E071E0C1
:100200000EC085E591E167E171E009C085E591E106
:100210006EE271E004C085E591E165E471E00E9461
:1002200097334091C90D50E060E070E085E591E1C1
:100230002AE000E00E9456D785E591E16AE057D9AF
:1002400081E001C080E0DF91CF911F910F9108956F
:10025000AF92BF92CF92DF92EF92FF920F931F93D4
:10026000CF93DF9311E7E12E1DE0F12EC6EEDDE026
:1002700000E010E0F801E450FD4F808132DF882378
:1002800031F17DDF5B016C01F801E559F24F8081AE
:10029000882311F061E002C06091F60D70E08827BC
:1002A00077FD8095982F0E942FDCF7012081318106
:1002B000428153810E946DDE9B01AC01C601B501F4
:1002C0000E94B4DA688379838A839B8309C0F7012B
:1002D00080819181A281B38188839983AA83BB8322
:1002E0000F5F1F4F84E090E0E80EF91E2496043063
:1002F000110509F0BFCF86E4F4DE8823D9F03FDF93
:100300007B018C016093F70D7093F80D8093F90DCC
:100310009093FA0D20E030E040E050E00E949BDD39
:10032000181644F4E0928C02F0928D0200938E0233
:1003300010938F02DF91CF911F910F91FF90EF905B
:10034000DF90CF90BF90AF90089582DF89E4C9DE3F
:10035000882351F014DF6093DA0D7093DB0D8093E6
:10036000DC0D9093DD0D0CC080E090E0A0E0B0E0EB
:100370008093DA0D9093DB0DA093DC0DB093DD0D2F
:100380008AE4AFDE882351F0FADE6093DE0D7093CD
:10039000DF0D8093E00D9093E10D089580E090E0F3
:1003A000A0E0B0E08093DE0D9093DF0DA093E00D10
:1003B000B093E10D08952F923F924F925F926F920A
:1003C0007F928F929F92AF92BF92CF92DF92EF92E5
:1003D000FF920F931F93DF93CF93CDB7DEB76E9746
:1003E0000FB6F894DEBF0FBECDBF87E47ADE882358
:1003F00009F433C2C4DE0E94FCDB6430710509F4E9
:100400003CC06530710554F46230710531F16330E0
:10041000710554F57723CCF40C947E926A357105FE
:1004200009F4CAC16B35710534F46C31710511F0F2
:100430000C947E927EC06B35710509F4C1C16C3598
:10044000710511F00C947E92C0C18091BC0D88237F
:1004500021F4FEDE4DDB0C94B5928091BC0D882317
:1004600019F473DF81E006C08091BC0D882329F464
:100470006CDF80E077DA0C94B59289E498E00E9412
:10048000ED6E80E52EDE882321F4EE24FF24870123
:1004900005C075DE0E9401DC7B018C0183E521DE55
:1004A000882359F06CDE20E030E04AE754E40E94F3
:1004B0006DDE0E9401DC7B018C010E945AA80FB600
:1004C000F894A0904C11B0904D11C0904E11D09066
:1004D0004F110FBEAE0CBF1CC01ED11E0FB6F8943C
:1004E00080914C1190914D11A0914E11B0914F11EE
:1004F0000FBE8093D20D9093D30DA093D40DB093E3
:10050000D50D05C00E945AA0C3D90E941E6F0FB618
:10051000F89480914C1190914D11A0914E11B09191
:100520004F110FBE8A159B05AC05BD0558F30C9401
:100530007E9280918C0290918D02A0918E02B0915A
:100540008F028093010E9093020EA093030EB0933E
:10055000040E80916C0290916D029093700D8093C7
:100560006F0D84E690E090936D0280936C020FB65D
:10057000F89480914C1190914D11A0914E11B09131
:100580004F110FBE8093D20D9093D30DA093D40D35
:10059000B093D50D81E00E9479A78091710D909163
:1005A000720DA091730DB091740D8093E60D909330
:1005B000E70DA093E80DB093E90D8091750D909132
:1005C000760DA091770DB091780D8093EA0D909300
:1005D000EB0DA093EC0DB093ED0D8091790D909102
:1005E0007A0DA0917B0DB0917C0D8093EE0D9093D0
:1005F000EF0DA093F00DB093F10D80917D0D9091D2
:100600007E0DA0917F0DB091800D8093F20D90939F
:10061000F30DA093F40DB093F50D80E090E0A0E011
:10062000B0E080938C0290938D02A0938E02B093E1
:100630008F0288E556DD882351F489E552DD882351
:1006400031F48AE54EDD882311F481E001C080E0B9
:1006500080939002882321F488E543DD882319F0F4
:1006600080E090E03ADB80919002882321F489E5D4
:1006700038DD882319F081E090E02FDB8091900233
:10068000882321F48AE52DDD882319F082E090E0AB
:1006900024DB88E526DD8823C9F066DD6115710558
:1006A0008105910599F06BDD2091810D3091820DCE
:1006B0004091830D5091840D0E94B4DA6093710DC6
:1006C0007093720D8093730D9093740D89E509DD1D
:1006D0008823C9F049DD611571058105910599F0FF
:1006E0004EDD2091850D3091860D4091870D509102
:1006F000880D0E94B4DA6093750D7093760D809327
:10070000770D9093780D8AE5ECDC8823C9F02CDD19
:10071000611571058105910599F031DD2091890DF3
:1007200030918A0D40918B0D50918C0D0E94B4DA5E
:100730006093790D70937A0D80937B0D90937C0D6F
:1007400081E79DE065E77DE049E75DE02DE73DE07D
:100750000E94041A80E00E9479A78091010E909176
:10076000020EA091030EB091040E80938C02909320
:100770008D02A0938E02B0938F0280916F0D9091A5
:10078000700D90936D0280936C020FB6F894809177
:100790004C1190914D11A0914E11B0914F110FBE7F
:1007A0008093D20D9093D30DA093D40DB093D50D1B
:1007B0000E9472A70C947E921092F60D0C947E9279
:1007C00081E08093F60D0C947E9285E48ADC882388
:1007D00011F40E945AA851E7E52E5DE0F52E41E89C
:1007E000C42E4DE0D42E00E010E0F801E450FD4F9F
:1007F000808177DC882321F1033059F4C0DCF701D4
:1008000060837183828393838DE79DE00E94E71963
:1008100017C0B5DCF60120813181428153810E94ED
:10082000B4DAF701608371838283938381E79DE06B
:1008300065E77DE049E75DE02DE73DE00E94041AB1
:100840000F5F1F4F44E050E0E40EF51EC40ED51EAE
:100850000430110551F60C947E928DE442DC88231D
:1008600011F40C9444918BDC0E94FCDB623771051F
:1008700011F40C94278D633771050CF084C06C3132
:10088000710509F442C26D317105C4F56531710518
:1008900009F4D5C166317105BCF46131710509F403
:1008A00099C16231710534F46230710510F00C9415
:1008B0007E921CC16231710509F4BBC764317105B8
:1008C00011F00C947E9292C16831710509F4DBC17C
:1008D0006931710554F46631710509F4B6C16731A7
:1008E000710511F00C947E92B6C16A31710509F45C
:1008F000E9C16B3171050CF002C2DEC165357105CD
:1009000009F4E4C766357105FCF46A32710509F42F
:1009100069C36B32710554F46E31710509F431C24B
:100920006F31710511F00C947E92ABC26335710585
:1009300009F47BC7643571050CF07BC7623571051E
:1009400011F00C947E926EC76936710509F4BEC32E
:100950006A36710554F46C35710509F4CDC76836F3
:10096000710511F00C947E9285C36B36710509F404
:1009700054C76B3671050CF421C76D36710511F043
:100980000C947E9272C4633D710511F40C94F28F45
:10099000643D71050CF050C06E3B710509F445C60D
:1009A0006F3B710524F56737710511F40C94088EBF
:1009B0006837710564F46337710511F40C94018D87
:1009C0006537710511F00C947E920C94118D693786
:1009D000710511F40C94048E6937710514F40C94AC
:1009E000028E6C38710511F00C947E9260C36C3CE1
:1009F000710511F40C94AA8E6D3C710564F4693C88
:100A0000710511F40C946A8E6B3C710511F00C9415
:100A10007E920C948C8E6E3C710511F40C94288F90
:100A20006E3C710514F40C94CA8E623D710511F090
:100A30000C947E920C94D48F51E06039750711F4B8
:100A40000C941E9181E0613978073CF56D3D71058C
:100A500011F40C941F906E3D710564F46A3D7105AC
:100A600011F40C94468F6C3D710511F00C947E923C
:100A70000C94109091E06E32790711F40C94CF90A1
:100A8000E1E06F327E0711F40C94DE906D527140FC
:100A900011F00C947E920C942E9021E0663F720728
:100AA00011F40C94279141E0673F74076CF451E016
:100AB000643F750711F40C942191655F714011F04A
:100AC0000C947E920C94249193E0603A790709F497
:100AD0009DC1E3E0673E7E0711F40C942D91675FA2
:100AE000714011F00C947E920C942A9188E398E066
:100AF0000E94ED6E80E5F5DA882321F4EE24FF24D0
:100B0000870105C03CDB0E9401DC7B018C0183E591
:100B1000E8DA882359F033DB20E030E04AE754E498
:100B20000E946DDE0E9401DC7B018C010E945AA8AC
:100B30000FB6F89480914C1190914D11A0914E11E7
:100B4000B0914F110FBE8093D20D9093D30DA0930F
:100B5000D40DB093D50DE114F1040105110581F117
:100B60000FB6F894A0904C11B0904D11C0904E115A
:100B7000D0904F110FBEAE0CBF1CC01ED11E0FB6C1
:100B8000F89480914C1190914D11A0914E11B0911B
:100B90004F110FBE8A159B05AC05BD05A8F40E9438
:100BA000732B882389F40E945AA00E94487C0E94DB
:100BB0001E6FE5CF0E945AA00E94487C0E941E6FC3
:100BC0000E94732B8823B1F389E298E00E94ED6EB6
:100BD0000C947E9280E298E00E94ED6E7798769871
:100BE000479843988C988D980C947E92E0E1F8E0B9
:100BF00064918F0108C085E591E10E94777A0F5FCB
:100C00001F4FF80164916623B1F785E591E16AE031
:100C10000E94777A8CE79BE00E947CCDE2E0F8E0CE
:100C200064918F0108C085E591E10E94777A0F5F9A
:100C30001F4FF80164916623B1F70C9479928CE709
:100C40009BE00E940CC90C947E928CE79BE00E9472
:100C500065C30C947E928091050E9091060E0496C9
:100C60006AE270E00E94DC10FC01009711F03197FD
:100C700010826091050E7091060E6C5F7F4F8CE7BD
:100C80009BE041E07AC08CE79BE00E9469C30FB60D
:100C9000F89480914C1190914D11A0914E11B0910A
:100CA0004F110FBE8093B40D9093B50DA093B60D68
:100CB000B093B70D0C947E928CE79BE00E9470C3BA
:100CC0000C947E9280917F0B882311F40C947E9279
:100CD00083E507DA882311F40C947E9245DAAB01A0
:100CE000BC014093600D5093610D8093620D709331
:100CF000630D8DE39DE00E94FDAF0C947E928CE726
:100D00009BE00E9455C50C947E928091050E9091B7
:100D1000060E04966AE270E00E94DC108C010097D7
:100D200019F12091FB0D3091FC0D80E690E0AC01B3
:100D3000249FC001259F900D349F900D1124895F41
:100D4000914F6EE470E00E94DC1060E270E00E945F
:100D5000DC109C012F5F3F4F3093060E2093050E51
:100D600001501040F80110826091050E7091060E3E
:100D70006C5F7F4F8CE79BE040E00E940BC70C94B8
:100D80007E9280917F0B882311F40C947E928CE7E5
:100D90009BE00E94C7C48091050E9091060E0496B8
:100DA0006AE270E00E94DC108C01009719F120913A
:100DB000FB0D3091FC0D80E690E0AC01249FC0015A
:100DC000259F900D349F900D1124895F914F6EE403
:100DD00070E00E94DC1060E270E00E94DC109C0178
:100DE0002F5F3F4F3093060E2093050E01501040A9
:100DF000F80110826091050E7091060E6C5F7F4FB6
:100E00008CE79BE00E94B8C50C947E928091050E01
:100E10009091060E05966AE270E00E94DC108C014B
:100E2000009719F12091FB0D3091FC0D80E690E0C8
:100E3000AC01249FC001259F900D349F900D11247B
:100E4000895F914F6EE470E00E94DC1060E270E018
:100E50000E94DC109C012F5F3F4F3093060E2093C1
:100E6000050E01501040F80110826091050E70913E
:100E7000060E6B5F7F4F8CE79BE00E9406C90C94C7
:100E80007E920FB6F89460914C1170914D11809143
:100E90004E1190914F110FBE6093B80D7093B90D24
:100EA0008093BA0D9093BB0D2091B40D3091B50D88
:100EB0004091B60D5091B70D621B730B840B950BCF
:100EC00028EE33E040E050E00E9485DFF22EE32E72
:100ED000D42EC52E4DB75EB7485050400FB6F8948B
:100EE0005EBF0FBE4DBF0DB71EB70F5F1F4FCE01C8
:100EF0000196EDB7FEB79283818383EF97E0F80107
:100F0000938382836F2D7E2D8D2D9C2D2CE330E0DD
:100F100040E050E00E9485DFF801358324836F2D87
:100F20007E2D8D2D9C2D2CE330E040E050E00E9482
:100F300085DFF801778366830E940B11EEEDF5E003
:100F400064918F014DB75EB7485F5F4F0FB6F8945D
:100F50005EBF0FBE4DBF08C085E591E10E94777A64
:100F60000F5F1F4FF80164916623B1F785E591E1AA
:100F70008E010F5F1F4FB8010E94973385E591E105
:100F80006AE00E94777AC8010E940F6F809135064F
:100F9000882311F40C947E92109235068091B10D45
:100FA000082F10E0000F111F0D56104FF80160813F
:100FB0007181882777FD8095982F0E942FDC2091E2
:100FC00038023091390240913A0250913B020E941E
:100FD0009BDD181614F00C947E92F8011182108299
:100FE0000C947E9283E57DD8882311F40C947E9234
:100FF000C6D80E94FCDB7B018C016B0180E571D8B7
:10100000882361F0F7FC0AC0FFEFEF16F10409F046
:101010002CF4B5D80E94FCDB7B0103C0EE24EA94DB
:10102000FE2CE0E0F3E0808191818E159F0511F4A4
:101030000C947E92329623E0E039F207A1F740E16A
:10104000E416F10429F4D092B30DC092B20D04C09D
:10105000F7FE02C00C947E928E2D0E948BD2EE2D54
:10106000F0E00C2C0E949CD28E2DB6010E9446D43A
:101070000C947E9288E690E08BD8882311F00C9433
:101080007E9283E52ED8882371F079D82091C90DFE
:10109000022F10E0000F111F0D56104F0E94FCDBB5
:1010A000F801718360830E94D29A0C947E9283E54A
:1010B00018D8882311F40C947E9261D80E94FCDB2E
:1010C00070939A0F6093990F0C947E9289E690E04A
:1010D0005FD8882311F00C947E92EDEEF7E06491D6
:1010E0008F0108C085E591E10E94777A0F5F1F4F5D
:1010F000F80164916623B1F7E091C90DF0E0EE0FBD
:10110000FF1FEE0FFF1FEF55F04F408151816281AD
:10111000738185E591E121E00E94F2D7EAEEF7E0E4
:1011200064918F0108C085E591E10E94777A0F5F95
:101130001F4FF80164916623B1F7E091C90DF0E00B
:10114000EE0FFF1FED56F04F60817181882777FD0C
:101150008095982F0E942FDCAB01BC0185E591E1C1
:1011600021E00E94F2D7E6EEF7E064918F0108C01B
:1011700085E591E10E94777A0F5F1F4FF801649136
:101180006623B1F74091AF0F5091B00F6091B10F4E
:101190007091B20F85E591E121E00E94F2D7E3EE74
:1011A000F7E064918F0108C085E591E10E94777AAC
:1011B0000F5F1F4FF80164916623B1F76091990F9B
:1011C00070919A0F882777FD8095982F0E942FDCC9
:1011D000AB01BC0185E591E121E00E94F2D7EFED82
:1011E000F7E064918F0108C085E591E10E94777A6C
:1011F0000F5F1F4FF80164916623B1F78091C90D0D
:1012000090E00E94179AAC01662757FD6095762FF3
:1012100085E591E10E94E1D7EAEDF7E064918F0165
:1012200008C085E591E10E94777A0F5F1F4FF801B2
:1012300064916623B1F78FEF9FEF0E94179AAC017C
:10124000662757FD6095762F85E591E10E94E1D7ED
:1012500085E591E16CE571E00E94973385E591E1C8
:101260006AE00E94777A0C94B5928DE690E00E9435
:10127000C880882311F00C947E928FEC97E00E9436
:10128000ED6E1092350683E50E947180882379F017
:101290000E94BF802091C90D022F10E0000F111F86
:1012A0000D56104F0E94FCDBF8017183608383E5CB
:1012B0000E947180882351F00E94BF8060933802A1
:1012C0007093390280933A0290933B0282E40E9429
:1012D0007180882351F00E94BF8060933402709324
:1012E0003502809336029093370286E40E94718023
:1012F000882369F00E94BF8060933C0270933D0296
:1013000080933E0290933F0281E0809335060E94D5
:10131000D29A0FB6F89480904C1190904D11A090F5
:101320004E11B0904F110FBE2091C90D022F10E049
:101330007724000F111FF801ED56F04F6081718185
:10134000882777FD8095982F0E942FDC000F111FB2
:101350000F55104FF80120813181428153810E9445
:101360009BDD181614F477247394CC24CA94DC2CD7
:101370007601ECECF7E04490E8ECF7E05490E4EC14
:10138000F7E064903CC1642D0CEC17E008C085E5E3
:1013900091E10E94777A0F5F1F4FF80164916623F5
:1013A000B1F7E091C90DF0E0EE0FFF1FEE0FFF1F48
:1013B000EF55F04F408151816281738185E591E164
:1013C00021E00E94F2D7652D08EC17E008C085E502
:1013D00091E10E94777A0F5F1F4FF80164916623B5
:1013E000B1F74091C90D50E0662757FD6095762F03
:1013F00085E591E10E94E1D7662D04EC17E008C075
:1014000085E591E10E94777A0F5F1F4FF8016491A3
:101410006623B1F7F7FC24C00FB6F89420914C1165
:1014200030914D1140914E1150914F110FBEC70197
:10143000B601605F784D8F4F9F4F621B730B840B1B
:10144000950B28EE33E040E050E00E9485DF85E513
:1014500091E1BA01A9012AE000E00E9456D706C036
:1014600085E591E16DE571E00E94973385E591E1B5
:101470006AE00E94777A0FB6F89480904C119090B1
:101480004D11A0904E11B0904F110FBE0E945AA066
:101490000E94487C0E941E6FFFEFCF16FFEFDF0611
:1014A000FFEFEF06FFEFFF0609F050C0E091C90D16
:1014B000772031F1F0E08F01000F111F000F111F95
:1014C0000F55104FEE0FFF1FED56F04F60817181E9
:1014D000882777FD8095982F0E942FDC20E030E050
:1014E00040E85FE30E94B3DA9B01AC01F801608140
:1014F0007181828193810E949BDD87FF58C062C009
:10150000F0E08F01000F111F000F111F0F55104F3A
:10151000EE0FFF1FED56F04F60817181882777FD38
:101520008095982F0E942FDC20E030E040E85FE3B8
:101530000E94B4DA9B01AC01F80160817181828163
:1015400093810E948DDB181694F53CC0F7FC3AC0DD
:10155000E091C90DF0E08F01000F111F000F111F66
:101560000F55104FEE0FFF1FED56F04F6081718148
:10157000882777FD8095982F0E942FDC9B01AC0176
:10158000F80160817181828193810E94B3DA0E94A7
:10159000FCDB97FF07C090958095709561957F4F14
:1015A0008F4F9F4F64307105810591055CF00FB638
:1015B000F894C0904C11D0904D11E0904E11F090E5
:1015C0004F110FBEFFEFCF16FFEFDF06FFEFEF0665
:1015D000FFEFFF06A1F0F7FE01C093C70FB6F89426
:1015E00080914C1190914D11A0914E11B0914F11DD
:1015F0000FBE8C199D098051974208F082C70FB623
:10160000F89480914C1190914D11A0914E11B09190
:101610004F110FBE88199909AA09BB09895E934029
:10162000A040B04008F0AFCE31CF89EA97E00E94E9
:10163000ED6E83E50E947180882341F00E94BF8097
:101640000E94FCDB70939A0F6093990F0FB6F89489
:10165000E0904C11F0904D1100914E1110914F11EE
:101660000FBEE6EAF7E09490E2EAF7E0A490EEE934
:10167000F7E0B49087C00FB6F89480914C11909128
:101680004D11A0914E11B0914F110FBE8E199F09AF
:10169000A00BB10B895E9340A040B04008F46CC031
:1016A000E091B10DF0E0EE0FFF1FEE0FFF1FEF55C1
:1016B000F04FC080D180E280F380692D06EA17E008
:1016C00008C085E591E10E94777A0F5F1F4FF8010E
:1016D00064916623B1F785E591E1B701A60122E0A7
:1016E0000E94F2D76A2D02EA17E008C085E591E171
:1016F0000E94777A0F5F1F4FF80164916623B1F75C
:101700004091B10D50E0662757FD6095762F85E535
:1017100091E10E94E1D76B2D0EE917E008C085E545
:1017200091E10E94777A0F5F1F4FF8016491662361
:10173000B1F74091AF0F5091B00F6091B10F709120
:10174000B20F85E591E121E00E94F2D785E591E1B4
:101750006CE571E00E94973385E591E16AE00E94B3
:10176000777A0FB6F894E0904C11F0904D110091FB
:101770004E1110914F110FBE0E945AA00E94487C3A
:101780000E941E6F6091990F70919A0F882777FDC4
:101790008095982F0E942FDC2091AF0F3091B00FD1
:1017A0004091B10F5091B20F0E949BDD18160CF4BE
:1017B00062CF84E997E00E94ED6EBAC683E50E948D
:1017C0007180882319F10E94BF8020E030E040E062
:1017D00050E00E948DDB88231CF460E070E011C0B3
:1017E0000E94BF8020E030E04FE753E40E949BDD81
:1017F00018161CF46FEF70E004C00E94BF800E94B6
:10180000FCDB7093B30D6093B20D78C68FEF90E060
:101810009093B30D8093B20D71C61092B30D1092D8
:10182000B20D6CC610926E0D69C681E080936E0D8C
:1018300065C683E50E947180882399F00E94BF806D
:1018400020E030E04AE754E40E946DDE0E9401DCB3
:10185000609388027093890280938A0290938B022E
:101860004DC688E50E947180882309F075C689E518
:101870000E947180882309F06FC68AE50E947180FA
:10188000882309F069C685E40E947180882309F0E5
:1018900063C60E945AA8439A8C9A8D9A0E9468A89F
:1018A0002DC6779A89E50E9471808111769A8AE522
:1018B0000E9471808111479A85E40E94718088237B
:1018C00009F41CC6439A8C9A8D9A18C683E50E9427
:1018D00071800E94BF8020E030E04AE754E40E941B
:1018E0006DDE0E9401DC6093D60D7093D70D80935E
:1018F000D80D9093D90D02C6F9ED6F2EF5E07F2E2D
:10190000E9EC2E2EE5E03E2E75E1472E76E0572ECF
:1019100088249924F401E450FD4F80810E94718055
:10192000882309F45DC0F3E08F1609F052C00E94CD
:10193000BF805B016C0120E030E040EA51E40E948E
:101940008DDB88230CF03FC0F301608171818281BF
:101950009381A60195010E9494DB7B018C0160912B
:101960000D0670910E0680910F0690911006A80149
:1019700097010E946DDE60930D0670930E068093B2
:101980000F0690931006F10160817181828193812D
:10199000A80197010E946DDEF1016083718382834B
:1019A0009383F20160817181828193810E942DDC99
:1019B000A80197010E946DDE0E9401DCF2016083A4
:1019C000718382839383F301A082B182C282D38226
:1019D00007C00E94BF80F301608371838283938379
:1019E0000894811C911C44E050E0640E751E240E86
:1019F000351E440E551E54E08516910409F08ACF19
:101A00007DC5E9EFF6E064918F0108C085E591E1BD
:101A10000E94777A0F5F1F4FF80164916623B1F738
:101A20006DC58091050E9091060E05966AE270E0F4
:101A30000E94DC10FC01009711F031971082809118
:101A4000050E9091060E05960E940F6F57C5E6EFA2
:101A5000F6E064918F0108C085E591E10E94777AF4
:101A60000F5F1F4FF80164916623B1F74091710D2C
:101A70005091720D6091730D7091740D85E591E137
:101A800022E00E94F2D7E3EFF6E064918F0108C0F4
:101A900085E591E10E94777A0F5F1F4FF80164910D
:101AA0006623B1F74091750D5091760D6091770DD9
:101AB0007091780D85E591E122E00E94F2D7E0EF88
:101AC000F6E064918F0108C085E591E10E94777A84
:101AD0000F5F1F4FF80164916623B1F74091790DB4
:101AE00050917A0D60917B0D70917C0D85E591E1AF
:101AF00022E00E94F2D7EDEEF6E064918F0108C07B
:101B000085E591E10E94777A0F5F1F4FF80164919C
:101B10006623B1F740917D0D50917E0D60917F0D50
:101B20007091800D85E591E122E00E94F2D7E2EE0E
:101B3000F6E064918F0108C085E591E10E94777A13
:101B40000F5F1F4FF80164916623B1F780E00E9498
:101B500025A80E942FDC2091D9053091DA0540910B
:101B6000DB055091DC050E9494DBAB01BC0185E5EF
:101B700091E122E00E94F2D7EFEDF6E064918F014F
:101B800008C085E591E10E94777A0F5F1F4FF80149
:101B900064916623B1F781E00E9425A80E942FDCA2
:101BA0002091DD053091DE054091DF055091E00583
:101BB0000E9494DBAB01BC0185E591E122E00E942B
:101BC000F2D7ECEDF6E064918F0108C085E591E174
:101BD0000E94777A0F5F1F4FF80164916623B1F777
:101BE00082E00E9425A80E942FDC2091E10530911F
:101BF000E2054091E3055091E4050E9494DBAB01BE
:101C0000BC01C3C280E001C081E00E9479A776C414
